:020000040800F2
:100000000000052031380008E5300008F330000812
:10001000F9300008FF30000805310008000000003A
:10002000000000000000000000000000410801087E
:100030000B31000800000000510A0108B90A01084C
:1000400081380008813800088138000881380008AC
:10005000813800088138000881380008813800089C
:10006000813800088138000881380008813800088C
:10007000813800088138000881380008813800087C
:10008000813800088138000881380008813800086C
:10009000813800088138000881380008813800085C
:1000A000813800088138000881380008813800084C
:1000B00081380008193100088138000881380008AB
:1000C000813800088138000881380008813800082C
:1000D000813800088138000881380008813800081C
:1000E000813800088138000881380008813800080C
:1000F00081380008813800088138000881380008FC
:10010000813800083931000881380008813800083A
:1001100081380008813800084D3100088138000816
:1001200081380008813800088138000861310008F2
:1001300081380008813800088138000881380008BB
:1001400081380008813800088138000881380008AB
:1001500081380008753100088138000881380008AE
:10016000813800088138000881380008813800088B
:10017000813800088138000881380008000000003C
:10018000813800088138000881380008813800086B
:10019000813800088138000881380008813800085B
:1001A00089310008813800089D3100088138000835
:1001B000813800088138000881380008813800083B
:0801C0008138000881380008B5
:1001D00010B5054C237833B9044B13B10448AFF381
:1001E00000800123237010BD3C01002000000000AE
:1001F00054C4020808B5034B1BB103490348AFF3CD
:10020000008008BD000000004001002054C4020826
:10021000034613F8012B002AFBD1181A0138704746
:1002200001F0FF01102A2BDB10F0070F08D010F8A7
:10023000013B013A8B422DD010F0070F42B3F6D1AB
:10024000F0B441EA012141EA014122F007047FF0C4
:1002500000070023F0E80256083C85EA010586EA1B
:10026000010685FA47F5A3FA87F586FA47F6A5FA57
:1002700087F68EB9EED1F0BC01F0FF0102F0070263
:1002800032B110F8013B013A83EA010313B1F8D10E
:100290000020704701387047002D06BF35460338EF
:1002A000073815F0010F07D1013015F4807F02BF28
:1002B000013015F4C03F0130F0BC0138704700BF79
:1002C00053B94AB9002908BF00281CBF4FF0FF31BD
:1002D0004FF0FF3000F06EB9ADF1080C6DE904CEBF
:1002E00000F006F8DDF804E0DDE9022304B0704711
:1002F0002DE9F047089D04468C46002B40F0838092
:100300008A42174647D9B2FA82F242B1C2F12000BE
:1003100024FA00F09140974040EA010C94404FEAE3
:100320001748230CBCFBF8F61FFA87FE08FB16C122
:1003300043EA014306FB0EF1994209D9FB1806F185
:10034000FF3080F01981994240F21681023E3B4411
:100350005B1AA4B2B3FBF8F008FB103344EA034481
:1003600000FB0EFEA64509D93C1900F1FF3380F0D1
:100370000581A64540F2028102383C4440EA06402D
:10038000A4EB0E0400261DB1D4400023C5E90043B0
:100390003146BDE8F08702B9FFDEB2FA82F2002AE8
:1003A00050D1CB1B4FEA174E1FFA87F80126B3FB3B
:1003B000FEFC210C0EFB1C3341EA034108FB0CF34D
:1003C0008B4207D979180CF1FF3002D28B4200F230
:1003D000E9808446C91AA3B2B1FBFEF00EFB1011EE
:1003E00043EA014408FB00F8A04507D93C1900F195
:1003F000FF3302D2A04500F2D9801846A4EB0804CE
:1004000040EA0C40BFE78B4209D9002D00F0B180D3
:100410000026C5E9000130463146BDE8F087B3FA51
:1004200083F6002E4AD18B4202D3824200F2B8807A
:10043000841A61EB030101208C46002DA8D0C5E988
:10044000004CA5E7C2F1200320FA03F6974001FA19
:1004500002F04FEA174ED9403043030CB1FBFEF6D1
:100460001FFA87F80EFB161143EA014306FB08F159
:10047000994204FA02F409D9FB1806F1FF3C80F016
:100480008D80994240F28A80023E3B445B1A81B2E1
:10049000B3FBFEF00EFB103341EA034100FB08F30F
:1004A0008B4207D9791800F1FF3C73D28B4271D986
:1004B00002383944CB1A40EA064678E7C6F1200CE8
:1004C00003FA06F422FA0CF31C4320FA0CF701FAA3
:1004D00006F34FEA144E21FA0CF11F433B0CB1FB1B
:1004E000FEF91FFA84F80EFB191143EA014109FBDA
:1004F00008FA8A4502FA06F200FA06F308D96118EA
:1005000009F1FF3048D28A4546D9A9F102092144B0
:10051000A1EB0A01BFB2B1FBFEF00EFB101147EADE
:10052000014700FB08F8B84507D9E71900F1FF318A
:100530002ED2B8452CD90238274440EA0940A7EB0F
:100540000807A0FB02894F45C64649461AD317D073
:100550005DB1B3EB0E0267EB010707FA0CFCF2404A
:100560004CEA0202F740C5E9002700263146BDE803
:10057000F0872E4628460BE70646E9E61846FDE6D4
:100580004345E5D2B8EB020E69EB04010138DFE721
:100590000846D2E760468DE78146B9E7664675E7CB
:1005A00030464AE7ACF1020C394413E702383C44C8
:1005B00024E700BF704700BF80B500AF10216A4834
:1005C00009F02AFB03469AB2684B1A80402168481A
:1005D00009F022FB03469AB2664B1A80634B1B88D4
:1005E000002B11D1644B1B7883F00103DBB2002B8D
:1005F00002D0624B01221A705F4B1B78002B14D083
:100600005F4B01221A7010E05B4B1B7883F00103F3
:10061000DBB2002B02D0594B00221A70564B1B78CC
:10062000002B02D0564B00221A70524B1B88002B15
:1006300011D1514B1B7883F00103DBB2002B02D0A8
:100640004F4B01221A704C4B1B78002B14D04B4B94
:1006500001221A7010E0484B1B7883F00103DBB2D3
:10066000002B02D0464B00221A70434B1B78002B04
:1006700002D0424B00221A70414B1B78002B03D151
:100680003E4B1B78002B02D03E4B00221A603E4BA3
:100690001B88032B03D03C4B1B88052B62D1374BA7
:1006A0001B78002B09D0394B1B7883F00103DBB298
:1006B000002B02D0364B01221A70314B1B78002BD5
:1006C00009D0344B1B7883F00103DBB2002B02D03E
:1006D0002F4B02221A70294B1B7883F00103DBB2E7
:1006E000002B0AD0294B1B78002B06D0244B1B78FB
:1006F000002B02D0264B02221A70214B1B7883F06C
:100700000103DBB2002B0AD0224B1B78002B06D052
:100710001A4B1B78002B02D01D4B01221A70174B6D
:100720001B7883F00103DBB2002B09D0144B1B783C
:1007300083F00103DBB2002B02D0154B00221A70AC
:100740000F4B1A78134B1A700C4B1A780F4B1A7008
:100750000A4B1B7883F00103DBB2002B02D00E4B57
:1007600000221A7000BF80BD000402400600002075
:100770000018024004000020630100205C010020FA
:100780005D01002030040020120000205E010020E6
:10079000600100205F0100206101002080B500AFF2
:1007A00000F02AFE034B00221A8000F005F800BF7B
:1007B00080BD00BF6E01002080B400AF444B1B8899
:1007C00042F6E062B2FBF3F39AB2424B1A80414B1D
:1007D0001B885B009AB2404B1A803E4B1B8807EE89
:1007E000903AB8EEE77A3D4B1B8807EE903AF8EE68
:1007F000677AF0EE086A67EEA66AB3EE0E6AC6EE96
:10080000867A67EE277AFCEEE77A17EE903A9AB28C
:10081000334B1A802F4B1B8807EE903AB8EEE77ADD
:10082000304B1B8807EE903AF8EE676A9FED2E6A10
:10083000C6EE267A67EE277AFCEEE77A17EE903A54
:100840009AB22A4B1A80234B1B8807EE903AB8EED7
:10085000E77A244B1B8807EE903AF8EE676A9FED23
:10086000226AC6EE867A67EE277AFCEEE77A17EE02
:10087000903A9AB2174B1A80164B1B881A461B4B9C
:100880001B8813441A4A128802FB03F3194A82FB9D
:1008900003125211DB17D31A1A46174B1A60104B6A
:1008A0001B881A46114B1B881344144A128802FBFA
:1008B00003F3104A82FB03125211DB17D31A1A46B4
:1008C0000F4B1A6000BFBD465DF8047B704700BF48
:1008D0000A0000206A010020680100200E000020AC
:1008E0006C0100201000002000004842660100203A
:1008F000160000201F85EB51C4570120180000206E
:10090000C057012080B582B000AF0346FB71FB7970
:10091000002B0ED00E4B1B78002B14D0012280210F
:100920000C4809F091F9012202210B4809F08CF9D9
:1009300009E000228021074809F086F900220221FF
:10094000054809F081F900BF0837BD4680BD00BFEA
:100950000C000020001802400020024080B500AFCB
:10096000104B1B78002B03D00120FFF7CBFF02E0D8
:100970000020FFF7C7FFFFF71FFEFFF71DFF0A4B21
:100980001B88042B00F2FB8301A252F823F000BF66
:10099000AD090008A90C0008050E0008F90F0008B1
:1009A000B3100008620100206E0100209A4B1B78F2
:1009B000002B0AD0994B1B88002B06D1984B1B8823
:1009C000032B02D0954B02221A80964B1B78002BEA
:1009D0000AD0924B1B88002B06D1914B1B88032B0E
:1009E00002D08E4B01221A808B4B1B78002B0AD031
:1009F0008D4B1B78022B06D1894B1B88032B02D110
:100A0000864B02221A80874B1B78002B0AD0864B1C
:100A10001B78012B06D1824B1B88032B02D17F4B05
:100A200001221A807C4B1B78002B0AD07E4B1B784E
:100A3000022B06D17A4B1B88052B02D1774B022261
:100A40001A80784B1B78002B11D0774B1B78012B29
:100A50000DD1764B1B7883F00103DBB2002B06D05F
:100A60006F4B1B88052B02D16C4B01221A80704BF7
:100A70001B88022B03D06E4B1B88012B0AD1674BBE
:100A80001B88002B06D16B4B1B78002B02D0634BCD
:100A900003221A80664B1B88022B03D0644B1B88F1
:100AA000012B0CD1634B1B7883F00103DBB2002BCD
:100AB00005D05A4B1B88002B01D100F083FB5E4B05
:100AC0001B685E4A128892009A1A5D4B1B689A4214
:100AD00011D95C4B1B7883F00103DBB2002B0AD0E9
:100AE000594B1B78002B06D04C4B1B88002B02D196
:100AF0004A4B04221A80504B1B68504A12889200BD
:100B00009A1A4F4B1B689A4213D94E4B1B7883F0AD
:100B10000103DBB2002B0CD04B4B1B7883F001039D
:100B2000DBB2002B05D03D4B1B88002B01D100F020
:100B30006DFB414B1B68414A12889A1A404B1B6857
:100B40009A4202D9414B04221A703B4B1B683B4A24
:100B5000128852009A1A3A4B1B689A4202D93B4BB0
:100B600005221A70344B1A68344B1B8819460B4601
:100B70005B000B44D21A324B1B689A4202D9334BAA
:100B800006221A702C4B1B682C4A128892009A1A63
:100B90002B4B1B689A4202D92C4B07221A70264B0A
:100BA0001A68264B1B8819460B469B000B44D21A29
:100BB000234B1B689A4202D9244B08221A701E4B01
:100BC0001A681E4B1B8819460B465B000B445B00E2
:100BD000D21A1B4B1B689A4202D91C4B09221A706D
:100BE000154B1A68154B1B8819460B46DB005B1A20
:100BF000D21A134B1B689A4202D9144B0A221A705C
:100C00000D4B1B680D4A1288D2009A1A0C4B1B68B8
:100C10009A4220D91CE000BF5D0100207001002035
:100C2000120000205C010020600100206101002012
:100C3000140000200D000020580100206A0100204F
:100C4000705701201A00002064010020720100206A
:100C50007C4B0B221A707C4B1A687C4B1B88194604
:100C60000B46DB000B44D21A794B1B689A4202D91F
:100C7000744B0C221A70744B1A68744B1B881946FB
:100C80000B469B000B445B00D21A714B1B689A42C7
:100C900002D96C4B0D221A706E4B1868002300228B
:100CA000684910F0EDF86AE26B4B01221A70694B4B
:100CB000186800230022634910F0E2F8674B1B8894
:100CC000002B02D1654B01221A80654B00221A804D
:100CD0000120FFF717FE634B00221A70624B0022BF
:100CE0001A70594B1B68614A13606FE0FFF764FC90
:100CF000564B1B881A465D4B1B681A44524B1B68A7
:100D00009A4294BF01230023DBB21A46554B1B784D
:100D100083F00103DBB21340002B18D00020FFF753
:100D2000F1FD4E4B1B885B009AB24C4B1A804B4B2B
:100D30001B8801339AB2494B1A80484B1B88FF2B02
:100D400002D9464B00221A80464B01221A70484BAA
:100D50001B88012B0BD0464B1B88022B07D0444B22
:100D60001B88032B03D0424B1B88052B2AD13F4BFA
:100D70001A68404B1B681A44334B1B689A4221D8AF
:100D80003D4B1B78002B0AD0394B1B88012B03D01D
:100D9000374B1B88022B02D1314B02221A80364B73
:100DA0001B78002B0ED0354B1B78022B0AD1304B11
:100DB0001B88032B03D02E4B1B88052B02D1284BFD
:100DC00002221A80204B1B681F4A13601F4B1B888E
:100DD0001A46264B1B681344294A12881A441A4B98
:100DE0001B689A4282D2184B1B68194A1360154B34
:100DF00000221A70174B186800230022114910F0C6
:100E00003FF8BCE1134B1868002300220D4910F095
:100E100037F8124B1B88002B02D1104B01221A808D
:100E20000F4B00221A800120FFF76CFD0D4B0022B2
:100E30001A700D4B00221A70034B1B680B4A13608B
:100E400098E000BF72010020580100206A010020D4
:100E500070570120A45A0120610100207401002074
:100E600070010020760100201A000020CC570120DC
:100E700012000020C45701205D0100206001002005
:100E800066010020FFF798FB8E4B1B881A468E4B9D
:100E90001B681A448D4B1B689A4294BF01230023A0
:100EA000DBB21A468A4B1B7883F00103DBB2134096
:100EB000002B12D00020FFF725FD864B1B885B001E
:100EC0009AB2844B1A80834B1B88FF2B02D9814B2B
:100ED00000221A807E4B01221A707F4B1B88012B47
:100EE0000BD07D4B1B88022B07D07B4B1B88032B21
:100EF00003D0794B1B88052B3CD1734B1A68774B79
:100F00001B681A44714B1B689A4233D8744B1B7888
:100F1000002B0AD0704B1B88012B03D06E4B1B8813
:100F2000022B02D16F4B01221A806D4B1B78002BD4
:100F30000AD06D4B1B78012B06D1674B1B88032B06
:100F400002D1684B01221A80654B1B78002B11D00F
:100F5000654B1B78012B0DD1644B1B7883F001038B
:100F6000DBB2002B06D05C4B1B88052B02D15D4BFE
:100F700001221A80534B1B881A46534B1B6813449B
:100F80005B4A12881A44514B1B689A4204D3524B55
:100F90001B88042B7FF476AF4F4B1B88042B19D191
:100FA00001E0FFF709FB534B1B78002BF9D1002020
:100FB000FFF7A8FC474B1B885B009AB2454B1A8091
:100FC000444B1B88FF2B02D9424B00221A80404B16
:100FD00001221A700020FFF795FC3C4B1B68464A23
:100FE0001360464B00221A70454B186800230022FC
:100FF00042490FF045FFC2E0404B01221A70404BBE
:101000001868002300223D490FF03AFF384B1B8837
:101010001A462D4B1B681A442C4B1B689A4202D966
:10102000364B02221A70364B1868002300223349CF
:101030000FF026FF334B1B78002B01D000F0C2F8D5
:10104000284B00221A80214B1B681F4A136017E0AF
:10105000FFF7B2FA274B1B78002B06D0214B1B88D9
:10106000002B02D11F4B02221A801D4B1B78002B34
:1010700006D01C4B1B88002B02D11A4B01221A8070
:10108000214B1B881A46104B1B681A440F4B1B68D8
:101090009A4203D31D4B1B78002BD9D1174B032247
:1010A0001A70174B18680023002214490FF0E8FE4D
:1010B00065E00C4B00221A80044B1B68024A136047
:1010C0003EE000BF6C010020CC57012058010020F9
:1010D000760100207401002012000020C05701207A
:1010E0005C010020700100206001002061010020EF
:1010F000660100205D010020705701207201002070
:10110000A45A012008000020680100200D000020E2
:10111000FFF752FA204B1B78002B06D01F4B1B8881
:10112000002B02D11D4B02221A801D4B1B78002B75
:1011300006D01A4B1B88002B02D1184B01221A80B3
:10114000184B1B885B001A46174B1B681A44174B39
:101150001B689A42DCD2164B1B7883F00103DBB28A
:10116000002B0BD000F052F8124B07221A70124BD2
:101170001868002300220F490FF082FE00BF0F4BBA
:101180001A880F4B1A80054B1A880C4B1A800120C5
:101190000EF0B4FE00BF80BD5D0100207001002094
:1011A0005C01002068010020CC570120580100207C
:1011B0001A00002072010020A45A01206E010020B4
:1011C0001400002080B582B000AF0C4B1B881A467B
:1011D0000B4B9B5CFB710B4B1B78002B06D00A4B17
:1011E0001868F91D002300220FF04AFE034B00226D
:1011F0001A8000BF0837BD4680BD00BF74010020C3
:10120000B8C5020808000020D859012080B582B076
:1012100000AF0A4B1B78FB71094B1B78002B06D0E3
:10122000084B1868F91D002300220FF029FE064B19
:1012300001221A7000BF0837BD4680BDB8C502083C
:1012400008000020D85901201A00002080B586B07F
:1012500004AF6723FB716423029301230193FB1DF9
:10126000009302230122A021574808F0C7FD052062
:1012700007F07AF96423029301230193534B0093FF
:1012800002230222A021504808F0B8FD052007F0F3
:101290006BF964230293012301934D4B00930223C6
:1012A0000322A021484808F0A9FD052007F05CF9B9
:1012B0006423029301230193464B009302230422EB
:1012C000A021414808F09AFD052007F04DF964235C
:1012D000029301230193404B009302230522A02196
:1012E000394808F08BFD052007F03EF9642302938E
:1012F00001230193394B009302230622A021324897
:1013000008F07CFD052007F02FF9642302930123E8
:101310000193334B009302230722A0212A4808F0AF
:101320006DFD052007F020F964230293012301934A
:101330002C4B009302230822A021234808F05EFDD5
:10134000052007F011F96423029301230193264B32
:10135000009302230922A0211B4808F04FFD05201D
:1013600007F002F964230293012301931F4B0093BA
:1013700002230A22A021144808F040FD052007F0AE
:10138000F3F86423029301230193194B0093022382
:101390000B22A0210C4808F031FD052007F0E4F8ED
:1013A0006423029301230193124B009302230C2226
:1013B000A021054808F022FD052007F0D5F800BF60
:1013C0000837BD4680BD00BF745701200A000020C9
:1013D000630100200D0000206401002016000020A1
:1013E000180000200E00002008000020100000203F
:1013F0000C0000201200002080B586B004AF00234E
:10140000FB716423029301230193FB1D00930223CC
:101410000122A021594808F005FE052007F0A4F894
:10142000FB79672B40F0A58064230293012301938D
:10143000534B009302230222A021504808F0F2FDF2
:10144000052007F091F864230293012301934D4B8B
:10145000009302230322A021484808F0E3FD052061
:1014600007F082F86423029301230193464B009313
:1014700002230422A021414808F0D4FD052007F0F2
:1014800073F86423029301230193404B00930223DA
:101490000522A021394808F0C5FD052007F064F8B1
:1014A0006423029301230193394B00930223062204
:1014B000A021324808F0B6FD052007F055F8642356
:1014C000029301230193334B009302230722A021AF
:1014D0002A4808F0A7FD052007F046F86423029388
:1014E000012301932C4B009302230822A0212348BF
:1014F00008F098FD052007F037F8642302930123D4
:101500000193264B009302230922A0211B4808F0D7
:1015100089FD052007F028F8642302930123019335
:101520001F4B009302230A22A021144808F07AFDE1
:10153000052007F019F86423029301230193194B46
:10154000009302230B22A0210C4808F06BFD05201C
:1015500007F00AF86423029301230193124B0093CE
:1015600002230C22A021054808F05CFD052006F0AE
:10157000FBFF00BF0837BD4680BD00BF7457012088
:101580000A000020630100200D00002064010020FB
:1015900016000020180000200E0000200800002087
:1015A000100000200C0000201200002080B500AFC9
:1015B0000249002010F030FE00BF80BDA13B0008B2
:1015C00080B485B000AFF860B9607A60FB68074A04
:1015D0001A60BB68064A1A607B6880221A6000BFE6
:1015E0001437BD465DF8047B704700BF78010020CA
:1015F0003002002080B400AFBFF34F8F00BFBFF3B5
:101600006F8F00BF0D4B0022C3F85022BFF34F8FE6
:1016100000BFBFF36F8F00BF084B5B69074A43F4FD
:1016200000335361BFF34F8F00BFBFF36F8F00BF15
:1016300000BFBD465DF8047B704700BF00ED00E0D1
:1016400080B485B000AF1F4B0022C3F88420BFF3E5
:101650004F8F00BF1B4BD3F880307B607B685B0BE8
:10166000C3F30E03FB607B68DB08C3F30903BB60B5
:10167000FB685A0143F6E0731340BA6892071149B8
:101680001343C1F86032BB685A1EBA60002BEFD119
:10169000FB685A1EFA60002BE5D1BFF34F8F00BFE5
:1016A000084B5B69074A43F480335361BFF34F8FA4
:1016B00000BFBFF36F8F00BF00BF1437BD465DF89A
:1016C000047B704700ED00E0B0B5DAB000AF00F089
:1016D00081FFFFF78FFFFFF7B3FF06F00FFF00F06A
:1016E000A3F900F0E1FC00F00DFA00F02DFA00F093
:1016F0002FFC00F09BFA00F0D9FA00F059FB00F043
:10170000ABFB00F0FFFB00F087FB01F017FE00F0E1
:101710004DFA02F0B6F8A9480CF012FE0023C7F803
:1017200060310023C7F8643107F5B0730121184612
:101730000EF0F8FB0346A24A13600023C7F85831A5
:101740000023C7F85C3107F5AC73012118460EF091
:10175000E9FB03469B4A13609B4B07F5A4740FCB30
:1017600084E80F0007F5A473002118460EF090FCE2
:101770000346964A1360944B07F59C740FCB84E89C
:101780000F0007F59C73002118460EF081FC0346FC
:101790008F4A13608C4B07F594740FCB84E80F00CD
:1017A00007F59473002118460EF072FC0346894A2F
:1017B0001360854B07F58C740FCB84E80F0007F599
:1017C0008C73002118460EF063FC0346824A1360B6
:1017D0007D4B07F584740FCB84E80F0007F5847305
:1017E000002118460EF054FC03467C4A1360764BE9
:1017F00007F1F8040FCB84E80F0007F1F80300218C
:1018000018460EF045FC0346754A1360754B07F108
:10181000E8040FCB84E80F0007F1E8030021184625
:101820000EF036FC0346704A1360674B07F1D8048C
:101830000FCB84E80F0007F1D803002118460EF003
:1018400027FC0346694A13605F4B07F1C8040FCBBE
:1018500084E80F0007F1C803002118460EF018FCB9
:101860000346634A1360584B07F1B8040FCB84E872
:101870000F0007F1B803002118460EF009FC0346DB
:101880005C4A1360504B07F1A8040FCB84E80F00AB
:1018900007F1A803002118460EF0FAFB0346564A4A
:1018A0001360494B07F198040FCB84E80F0007F150
:1018B0009803002118460EF0EBFB03464F4A1360D5
:1018C000414B07F188040FCB84E80F0007F1880330
:1018D000002118460EF0DCFB0346494A13603A4BE0
:1018E00007F178040FCB84E80F0007F1780300219B
:1018F00018460EF0CDFB0346424A136007F1680319
:10190000314A1C4613460FCB84E80F0007F16803E9
:10191000002118460EF0BCFB03463B4A136007F15A
:101920005803294A1C4613460FCB84E80F0007F1E1
:101930005803002118460EF0ABFB0346334A1360F0
:1019400007F13C03324A1C4615460FCD0FC495E8FB
:10195000070084E8070007F13C03002118460EF059
:101960006FFA03462B4A136007F120032A4A1C46EC
:1019700015460FCD0FC495E8070084E8070007F16E
:101980002003002118460EF05BFA0346234A136039
:101990003B1D234A1C4615460FCD0FC495E8070092
:1019A00084E807003B1D002118460EF049FA034663
:1019B0001C4A13600EF021FAFEE700BFE458012034
:1019C000EC5901209C5A012094C40208E0590120DE
:1019D000E8590120DC580120A05A0120505801206C
:1019E000D8590120A4C40208A45A0120E4590120B6
:1019F00028580120D8580120D4570120585A0120D6
:101A00003C5B0120E0580120F0590120545A01208C
:101A1000B4C40208D8570120D0C40208DC59012000
:101A2000ECC40208D057012080B594B000AF07F194
:101A3000200330220021184629F0D8FB07F10C03BF
:101A400000221A605A609A60DA601A612B4B1B6C94
:101A50002A4A43F080531364284B1B6C03F08053D5
:101A6000BB60BB68264B1B68254A43F440431360A8
:101A7000234B1B6803F440437B607B6801233B627C
:101A80004FF480337B620223BB634FF48003FB631C
:101A900019233B644FF4D8737B640223BB640F2388
:101AA000FB6407F12003184609F0BAFF0346002B38
:101AB00001D000F0D9FD09F01BFA0346002B01D03C
:101AC00000F0D2FD0F23FB6002233B6100237B610A
:101AD0004FF4A053BB614FF48053FB6107F10C033B
:101AE000072118460AF040FA0346002B01D000F007
:101AF000BBFD00BF5037BD4680BD00BF003802406F
:101B00000070004080B500AF0D4B0E4A1A600C4BC0
:101B100000221A710A4B00225A71094B00225A61A5
:101B2000074B00229A61064B01221A62044806F014
:101B3000CFFE0346002B01D000F096FD00BF80BD14
:101B40002C5801200030024080B500AF154B164ADA
:101B50001A60144B00225A60124B00229A60114BFB
:101B60000022DA600F4B00229A620E4B0022DA62EA
:101B70000C4B00221A630B4B00225A63094807F0F2
:101B8000A7FB0346002B01D000F06EFD01210548A4
:101B900007F0F8FC0346002B01D000F065FD00BF04
:101BA00080BD00BF5C5A012000B0024080B500AF8C
:101BB0001B4B1C4A1A601A4B1B4A5A60184B0022D6
:101BC0009A60174B0122DA60154B00221A61144B00
:101BD00000225A61124B00229A61114B0022DA61F5
:101BE0000F4B00221A620E4808F048F80346002BFB
:101BF00001D000F039FD0021094808F049FD0346F5
:101C0000002B01D000F030FD0021054808F08BFDCD
:101C10000346002B01D000F027FD00BF80BD00BFB0
:101C200074570120005400406847402080B500AF41
:101C30001B4B1C4A1A601A4B1B4A5A60184B002255
:101C40009A60174B0122DA60154B00221A61144B7F
:101C500000225A61124B00229A61114B0022DA6174
:101C60000F4B00221A620E4808F008F80346002BBA
:101C700001D000F0F9FC0021094808F009FD0346F5
:101C8000002B01D000F0F0FC0021054808F04BFDCE
:101C90000346002B01D000F0E7FC00BF80BD00BF71
:101CA000DC570120005C00406847402080B58EB0C2
:101CB00000AF3B1D34220021184629F097FA3A4B19
:101CC0003A4A1A60384B00225A60374B00229A6019
:101CD000354B0022DA60344B00221A61324B282245
:101CE0005A61314B09229A612F4B3522DA612E4B12
:101CF0000B221A622C4B40F215225A622A4B40F2F8
:101D00001B129A62284B40F23522DA62264B40F2CF
:101D10001D121A63244B002283F83420224B002228
:101D200083F83520204B002283F836201E4808F027
:101D300047FD0346002B01D000F096FC00237B609A
:101D40004FF4F073BB600023FB604FF488733B617A
:101D500002237B61FF23BB610023FB614FF480639F
:101D60003B6205237B624FF04043BB624FF4F0734C
:101D7000FB624FF488733B63002387F83430002301
:101D800087F83530002387F836303B1D002219468E
:101D9000054808F09DFE0346002B01D000F064FCCE
:101DA00000BF3837BD4680BD305901200068014072
:101DB00080B500AF164B174A1A60154B01225A60C6
:101DC000134B04229A60124B1022DA60104B182237
:101DD0001A610F4B4FF4A0625A610D4B00229A61B9
:101DE0000B4B0022DA610A4B00221A62084809F004
:101DF000CFF80346002B01D000F036FC05F0EEFED4
:101E000005F044FF5C2006F0D9FC00BF80BD00BF98
:101E1000405B0120001000A080B400AF0C4B0D4AC5
:101E20001A600B4B00225A60094B00229A60084B43
:101E30000022DA60064B00221A61054B00225A612B
:101E4000034B00229A6100BFBD465DF8047B7047DA
:101E500054580120002C014080B58AB000AF07F132
:101E60001C0300221A605A609A603B4600221A60E6
:101E70005A609A60DA601A615A619A611F4B204A6F
:101E80001A601E4B64225A601C4B00229A601B4B46
:101E90006922DA60194B00221A61184B00229A61FC
:101EA00016480CF0C5FA0346002B01D000F0DCFB0D
:101EB0002023FB6100237B6207F11C0319460F48B6
:101EC0000CF0C8FF0346002B01D000F0CDFB00232F
:101ED0003B6000237B600023BB6000233B613B46EB
:101EE0000022194605480CF019FC0346002B01D0CE
:101EF00000F0BAFB00BF2837BD4680BDE458012082
:101F00000004004080B582B000AF104B1B6B0F4A3D
:101F100043F4800313630D4B1B6B03F480037B605E
:101F20007B68002205213B2006F01EFC3B2006F0CA
:101F300037FC00220521452006F016FC452006F05E
:101F40002FFC00BF0837BD4680BD00BF00380240EF
:101F500080B588B000AF3B1D00221A605A609A60BD
:101F6000DA601A615A619A614C4B4D4A1A604B4BC8
:101F700000225A60494B00229A60484B0422DA60E2
:101F8000464B10221A61454B40225A61434B4FF495
:101F9000C0729A61414B0022DA61404B4FF40062FB
:101FA0001A623E4B4FF480525A623C4B00229A62B6
:101FB00002237B600723BB600423FB6007233B6194
:101FC00003237B610223BB610223FB613B1D194696
:101FD00032480CF0D4F80346002B01D000F044FB4B
:101FE00000233B602F4B01221A602E4B10225A60B7
:101FF0002C4B01229A602B4B0022DA604FF6FF72C5
:10200000284926480CF0EFF8012006F0ADFA254BE0
:1020100002221A60234B10225A60224B01229A603E
:10202000204B0022DA604FF6FF721E491B480CF06D
:10203000DAF81C4B03221A601A4B10225A60194B13
:1020400008229A60174B0022DA604FF6FF7215499A
:1020500012480CF0C8F84FF40C733B60114B04228B
:102060001A60104B10225A600E4B01229A603B6896
:102070000C4AD3604FF6FF720A4908480CF0B3F8D7
:1020800040F22B7105480CF0D9F84FF0204343F291
:10209000D2021A6000BF2037BD4680BDA85A012079
:1020A000400100A03404002080B590B000AF07F1DB
:1020B0002C0300221A605A609A60DA601A61824B1F
:1020C0001B6B814A43F0100313637F4B1B6B03F0C0
:1020D0001003BB62BB6A7C4B1B6B7B4A43F0020361
:1020E0001363794B1B6B03F002037B627B6A764BB5
:1020F0001B6B754A43F004031363734B1B6B03F0B4
:1021000004033B623B6A704B1B6B6F4A43F0010355
:1021100013636D4B1B6B03F00103FB61FB696A4B9F
:102120001B6B694A43F040031363674B1B6B03F05F
:102130004003BB61BB69644B1B6B634A43F4007390
:102140001363614B1B6B03F400737B617B695E4B14
:102150001B6B5D4A43F0080313635B4B1B6B03F07F
:1021600008033B613B69584B1B6B574A43F4806340
:102170001363554B1B6B03F48063FB60FB68524B8E
:102180001B6B514A43F0200313634F4B1B6B03F04F
:102190002003BB60BB684C4B1B6B4B4A43F4807302
:1021A0001363494B1B6B03F480737B607B68464B66
:1021B0001B6B454A43F080031363434B1B6B03F0D7
:1021C00080033B603B6801220821404807F03CFD4A
:1021D000002202213E4807F037FD01224FF48051D2
:1021E0003B4807F031FD002280213A4807F02CFDE2
:1021F0001023FB6200233B6301237B6307F12C0365
:102200001946354807F050FA4FF40053FB6200239B
:102210003B6300237B6307F12C0319462F4807F02B
:1022200043FA0823FB6201233B6300237B63002303
:10223000BB6307F12C031946244807F035FA41F235
:102240000203FB6201233B6300237B630023BB6328
:1022500007F12C0319461E4807F026FA0123FB62FA
:1022600000233B6301237B6307F12C0319461848C5
:1022700007F01AFA8023FB6201233B6300237B6390
:102280000023BB6307F12C031946124807F00CFA30
:102290004023FB6200233B6301237B6307F12C0394
:1022A00019460C4807F000FA4023FB6200233B6309
:1022B00001237B6307F12C031946094807F0F4F961
:1022C00000BF4037BD4680BD0038024000280240B4
:1022D00000200240001802400004024000080240B2
:1022E000001C024080B500AF094B1B68782B04D955
:1022F00000220821074807F0A7FC054B1B68002BAC
:1023000004D101220821034807F09EFC00BF80BDD4
:10231000300400200028024080B582B000AF786011
:102320004FF47A700DF0EAFD024B1B680133014A4D
:102330001360F5E73004002080B584B000AF78600A
:10234000FEF70CFBFFF7CEFF874B1B78012B13D159
:10235000FFF752F8FEF722FA0123BB81834B18687E
:1023600007F10C01002300220EF08AFD0A200DF077
:10237000C5FD7D4B00221A707D4B1B78012B04D1CB
:10238000FEF764FF7A4B00221A707A4B1B88FB81A0
:10239000794B1B6807F10E01002218460EF0ACFFC6
:1023A0000346012B05D1FA89724B1A80704B01222A
:1023B0001A70724B1B6807F10E01002218460EF0CE
:1023C0009BFF0346012B0AD1FB89002B14BF01237D
:1023D0000023DAB26A4B1A70654B01221A70694BFE
:1023E0001B6807F10E01002218460EF085FF034618
:1023F000012B0AD1FB89002B14BF01230023DAB281
:10240000614B1A705A4B01221A70604B1B6807F11E
:102410000E01002218460EF06FFF0346012B0AD171
:10242000FB89002B14BF01230023DAB2584B1A702A
:102430004F4B01221A70574B1B6807F10E01002207
:1024400018460EF059FF0346012B05D1FA89524B6D
:102450001A80474B01221A70504B1B6807F10E017E
:10246000002218460EF048FF0346012B05D1FA89D9
:102470004B4B1A803E4B01221A704A4B1B6807F1E6
:102480000E01002218460EF037FF0346012B05D13E
:10249000FA89454B1A80364B01221A70434B1B6850
:1024A00007F10E01002218460EF026FF0346012B0D
:1024B00005D1FA893E4B1A802D4B01221A703D4BF3
:1024C0001B6807F10E01002218460EF015FF0346A7
:1024D000012B0AD1FB89002B14BF01230023DAB2A0
:1024E000354B1A70224B01221A70344B1B6807F1CE
:1024F0000E01002218460EF0FFFE0346012B0AD102
:10250000FB89002B14BF01230023DAB22C4B1A7075
:10251000174B01221A702B4B1B6807F10E0100228A
:1025200018460EF0E9FE0346012B07D1FB89002B6C
:1025300014BF01230023DAB2234B1A70234B1B680C
:1025400007F10E01002218460EF0D6FE0346012BBD
:1025500005D1FA891E4B1A80054B01221A70012001
:102560000DF0CCFCECE600BF1B000020D45701208E
:10257000440400200A000020E0590120E85901200D
:1025800064010020DC5801200D000020A05A012029
:10259000630100202858012016000020D85801208F
:1025A00018000020585A01200E0000203C5B01203A
:1025B000100000205058012008000020E0580120A1
:1025C0000C000020F059012062010020545A012023
:1025D0001200002080B584B000AF3B4600221A6094
:1025E0005A609A60DA6006F0F7F801233B70002326
:1025F0007B704FF010437B601B233B7200237B7288
:102600000023BB720323FB7200233B7300237B7305
:102610000023BB730023FB733B46184606F014F9F6
:1026200001237B7017233B720123BB733B46184683
:1026300006F00AF9042006F0E7F800BF1037BD469F
:1026400080BD000080B582B000AF78607B681B68F9
:10265000044A934201D105F067FF00BF0837BD4629
:1026600080BD00BF0010004080B400AF00BFBD4679
:102670005DF8047B7047000080B582B000AF114B5D
:102680001B6C104A43F0805313640E4B1B6C03F019
:1026900080537B607B680B4B5B6C0A4A43F480433E
:1026A0005364084B5B6C03F480433B603B6800223F
:1026B0000F216FF0010006F057F800BF0837BD4644
:1026C00080BD00BF0038024080B485B000AF7860A4
:1026D0007B681B680A4A93420BD10A4B1B6B094A61
:1026E00043F480531363074B1B6B03F48053FB606D
:1026F000FB6800BF1437BD465DF8047B704700BF20
:10270000003002400038024080B584B000AF7860ED
:102710007B681B680D4A934213D10D4B1B6B0C4A0F
:1027200043F4000313630A4B1B6B03F40003FB60C9
:10273000FB68002205215A2006F016F85A2006F000
:102740002FF800BF1037BD4680BD00BF00B002406B
:102750000038024080B5ACB000AF786007F19C0350
:1027600000221A605A609A60DA601A6107F1180351
:1027700084220021184628F039FD7B681B68444AF2
:1027800093423DD14FF48043BB610023FB6707F1C7
:102790001803184609F0DCFD0346002B01D0FFF7B3
:1027A00063FF3C4B1B6B3B4A43F002031363394B03
:1027B0001B6B03F002037B617B694FF44073C7F826
:1027C0009C301223C7F8A0300023C7F8A43003239D
:1027D000C7F8A8300423C7F8AC3007F19C031946AA
:1027E0002D4806F061FF2B4B1B6C2A4A43F4001363
:1027F0001364284B1B6C03F400133B613B6942E0FC
:102800007B681B68254A93423DD14FF48033BB61FE
:102810000023C7F8843007F11803184609F098FD23
:102820000346002B01D0FFF71FFF1A4B1B6B194A01
:1028300043F080031363174B1B6B03F08003FB60B3
:10284000FB684FF4C073C7F89C301223C7F8A03060
:102850000123C7F8A4300323C7F8A8300423C7F81E
:10286000AC3007F19C0319460D4806F01DFF094BDB
:102870001B6C084A43F400031364064B1B6C03F4FF
:102880000003BB60BB6800BFB037BD4680BD00BF62
:10289000005400400038024000040240005C004048
:1028A000001C024080B582B000AF78607B681B6876
:1028B000154A934210D1154B1B6C144A23F4001394
:1028C00013644FF48071124807F09AF84FF40071C6
:1028D0000F4807F095F813E07B681B680D4A934298
:1028E0000ED10A4B1B6C094A23F4000313648021A8
:1028F000094807F085F84FF48071074807F080F821
:1029000000BF0837BD4680BD00540040003802407B
:1029100000040240005C0040001C024080B5AEB0E4
:1029200000AF786007F1A40300221A605A609A6031
:10293000DA601A6107F1200384220021184628F08A
:1029400055FC7B681B686F4A934240F0D680082391
:102950003B624FF4C0737B630523FB630223BB63BD
:1029600000233B640123BB644FF40033FB6407F195
:102970002003184609F0ECFC0346002B01D0FFF7BA
:1029800073FE614B5B6C604A43F0806353645E4B43
:102990005B6C03F08063FB61FB695B4B1B6B5A4A0A
:1029A00043F010031363584B1B6B03F01003BB6120
:1029B000BB69554B1B6B544A43F400731363524B72
:1029C0001B6B03F400737B617B694F4B1B6B4E4A9F
:1029D00043F4806313634C4B1B6B03F480633B61D4
:1029E0003B69494B1B6B484A43F040031363464B1A
:1029F0001B6B03F04003FB60FB68434B1B6B424ABD
:102A000043F480731363404B1B6B03F48073BB6010
:102A1000BB681023C7F8A4300223C7F8A8300023EE
:102A2000C7F8AC300023C7F8B0300E23C7F8B43075
:102A300007F1A4031946354806F036FE4EF6FF733B
:102A4000C7F8A4300223C7F8A8300023C7F8AC3079
:102A50000023C7F8B0300E23C7F8B43007F1A40341
:102A600019462B4806F020FEF723C7F8A4300223AE
:102A7000C7F8A8300023C7F8AC300023C7F8B0303F
:102A80000E23C7F8B43007F1A4031946214806F015
:102A90000BFE4FF48053C7F8A4300223C7F8A830C8
:102AA0000023C7F8AC300023C7F8B0300923C7F8BB
:102AB000B43007F1A4031946174806F0F5FD4FF4AA
:102AC0004643C7F8A4300223C7F8A8300023C7F84C
:102AD000AC300023C7F8B0300E23C7F8B43007F18C
:102AE000A40319460D4806F0DFFD002205215820F9
:102AF00005F03AFE582005F053FE00BFB837BD463A
:102B000080BD00BF00680140003802400010024054
:102B10000024024000280240001802400020024029
:102B200080B58CB000AF786007F11C0300221A60FA
:102B30005A609A60DA601A617B681B683B4A93426C
:102B400070D13B4B9B6B3A4A43F002039363384B83
:102B50009B6B03F00203BB61BB69354B1B6B344AB3
:102B600043F010031363324B1B6B03F010037B61C4
:102B70007B692F4B1B6B2E4A43F0020313632C4BD4
:102B80001B6B03F002033B613B69294B1B6B284A1B
:102B900043F008031363264B1B6B03F00803FB6031
:102BA000FB680423FB6102233B6200237B62032357
:102BB000BB620923FB6207F11C0319461D4806F09E
:102BC00073FD4023FB6102233B6200237B620323EE
:102BD000BB620A23FB6207F11C031946164806F084
:102BE00063FD0423FB6102233B6200237B6203231A
:102BF000BB620923FB6207F11C0319460E4806F06D
:102C000053FD4FF46053FB6102233B6200237B6260
:102C10000323BB620923FB6207F11C031946074823
:102C200006F042FD00BF3037BD4680BD001000A059
:102C3000003802400010024000040240000C024034
:102C400080B582B000AF78607B681B680C4A934205
:102C500012D10C4B9B6B0B4A23F0020393630421AC
:102C6000094806F0CDFE4421084806F0C9FE4FF49D
:102C70006051074806F0C4FE00BF0837BD4680BD5E
:102C8000001000A000380240001002400004024082
:102C9000000C024080B5ACB000AF786007F19C0337
:102CA00000221A605A609A60DA601A6107F118030C
:102CB00084220021184628F099FA7B681B68754A1F
:102CC000934240F0E2804FF42003BB610023C7F839
:102CD00094300023C7F8983007F11803184609F01C
:102CE00037FB0346002B01D0FFF7BEFC6A4B5B6C41
:102CF000694A43F400635364674B5B6C03F40063FD
:102D00007B617B69644B1B6B634A43F00403136371
:102D1000614B1B6B03F004033B613B695E4B1B6B18
:102D20005D4A43F0080313635B4B1B6B03F008031E
:102D3000FB60FB684FF4F853C7F89C300223C7F8D8
:102D4000A0300023C7F8A4300323C7F8A8300C2311
:102D5000C7F8AC3007F19C031946504806F0A4FCB4
:102D60000423C7F89C300223C7F8A0300023C7F81B
:102D7000A4300323C7F8A8300C23C7F8AC3007F100
:102D80009C031946464806F08FFC464B464A1A609B
:102D9000444B4FF000625A60424B00229A60414B14
:102DA0000022DA603F4B4FF480621A613D4B4FF4D2
:102DB00080525A613B4B4FF480429A61394B20223A
:102DC000DA61384B4FF400321A62364B04225A62F1
:102DD000344B03229A62334B4FF40002DA62314BD8
:102DE0004FF400121A632F4805F05CFE0346002BD7
:102DF00001D0FFF739FC7B682A4A1A64294A7B68AC
:102E000093632A4B2A4A1A60284B4FF000625A609B
:102E1000264B40229A60254B0022DA60234B4FF468
:102E200080621A61214B4FF480525A611F4B4FF45C
:102E300080429A611D4B2022DA611C4B4FF4003214
:102E40001A621A4B04225A62184B03229A62174BD9
:102E50004FF40002DA62154B4FF400121A63134864
:102E600005F020FE0346002B01D0FFF7FDFB7B6839
:102E70000E4ADA630D4A7B689363002205213120F4
:102E800005F072FC312005F08BFC00BFB037BD4669
:102E900080BD00BF002C0140003802400008024005
:102EA000000C0240F459012058640240DC5A012011
:102EB000A064024080B584B000AF78607B681B6876
:102EC0000D4A934213D10D4B1B6C0C4A43F0020385
:102ED00013640A4B1B6C03F00203FB60FB680022C7
:102EE00005211D2005F040FC1D2005F059FC00BF08
:102EF0001037BD4680BD00BF0004004000380240CE
:102F000080B586B000AF3B1D00221A605A609A60FF
:102F1000DA601A613A4B1B68002B6DD1384B0122E5
:102F20001A60384B9B6B374A43F001039363354B70
:102F30009B6B03F001033B603B684FF683737B6040
:102F40000223BB600023FB6003233B610C237B61F6
:102F50003B1D19462C4806F0A7FB48F233137B6053
:102F60000223BB600023FB6003233B610C237B61D6
:102F70003B1D1946254806F097FB4CF203737B6016
:102F80000223BB600023FB6003233B610C237B61B6
:102F90003B1D19461E4806F087FB4FF63F037B603A
:102FA0000223BB600023FB6003233B610C237B6196
:102FB0003B1D1946174806F077FB28237B60022348
:102FC000BB600023FB6003233B610C237B613B1D43
:102FD0001946114806F068FB08237B600223BB609A
:102FE0000023FB6003233B610C237B613B1D1946DF
:102FF0000A4806F059FB00E000BF1837BD4680BD07
:10300000480400200038024000100240001802402E
:10301000000C024000140240001C02400008024064
:1030200080B582B000AF7860FFF76AFF00BF083755
:10303000BD4680BD80B58CB000AF78600023FB62D8
:103040000023BB6200227968362005F08DFB362014
:1030500005F0A6FB1F4B1B6C1E4A43F010031364C4
:103060001C4B1B6C03F01003FB60FB6807F11002A4
:1030700007F114031146184609F038F909F022F94E
:1030800003465B00FB62FB6A134AA2FB03239B0C13
:10309000013BBB62114B124A1A60104B40F2E732FF
:1030A000DA600E4ABB6A53600C4B00221A610B4B6C
:1030B00000229A6009480BF0E1F80346002B04D186
:1030C00006480BF03DF9034600E00123184630376F
:1030D000BD4680BD0038024083DE1B438C5B01206F
:1030E0000010004080B400AF00BFBD465DF8047B17
:1030F000704780B400AFFEE780B400AFFEE780B455
:1031000000AFFEE780B400AFFEE780B400AF00BFC1
:10311000BD465DF8047B704780B500AF04480BF0F6
:10312000DEF9044B1B680133024A136000BF80BD07
:10313000E45801205801002080B500AF024809F092
:1031400075FF00BF80BD00BF5458012080B500AF9F
:1031500002480BF0C4F900BF80BD00BF8C5B0120AA
:1031600080B500AF024805F03DFE00BF80BD00BF46
:10317000F459012080B500AF024805F033FE00BFCE
:1031800080BD00BFDC5A012080B500AF024807F0C7
:10319000E7FB00BF80BD00BF3059012080B500AF04
:1031A000024806F0DFF800BF80BD00BF5C5A012076
:1031B00080B400AF01231846BD465DF8047B70471C
:1031C00080B582B000AF7860396027F0BBFE03465F
:1031D00016221A604FF0FF3318460837BD4680BDEF
:1031E00080B582B000AF78604FF0FF317868FFF7AC
:1031F000E7FFFEE780B586B000AFF860B9607A609F
:1032000000237B610AE0AFF300800146BB685A1CD3
:10321000BA60CAB21A707B6901337B617A697B68D4
:103220009A42F0DB7B6818461837BD4680BD80B5F2
:1032300086B000AFF860B9607A6000237B6109E076
:10324000BB685A1CBA601B781846AFF300807B69D4
:1032500001337B617A697B689A42F1DB7B681846AF
:103260001837BD4680BD80B483B000AF78604FF0A2
:10327000FF3318460C37BD465DF8047B704780B4B9
:1032800083B000AF786039603B684FF400525A60F9
:10329000002318460C37BD465DF8047B704780B4A8
:1032A00083B000AF7860012318460C37BD465DF847
:1032B000047B704780B485B000AFF860B9607A6075
:1032C000002318461437BD465DF8047B70470000A4
:1032D00080B586B000AF7860144A154BD31A7B6175
:1032E0007B693B61134B1B68002B02D1114B124AC7
:1032F0001A60104B1A687B6813443A699A4207D2E5
:1033000027F020FE03460C221A604FF0FF3309E03D
:10331000084B1B68FB60074B1A687B681344054A1F
:103320001360FB6818461837BD4680BD00000520B5
:10333000000A00004C040020A860012080B500AF06
:10334000044905480CF020FD03461A46034B1A7049
:1033500000BF80BDDC5B0120B8C60208D85B01203D
:1033600080B582B000AF0023FB7100F096F80346F1
:10337000012B01D0022312E00B4809F0D9FB0346D0
:10338000FB71FB79002B09D14FF4006106480AF06C
:103390009DF90346002B01D00123FB71FB791846F0
:1033A0000837BD4680BD00BF5458012080B586B0A7
:1033B00000AFF860B9607A600023FB757B68BA687B
:1033C000F968064809F06AFC0346002B01D0012386
:1033D000FB75FB7D18461837BD4680BD545801204B
:1033E00080B586B000AFF860B9607A600023FB75E5
:1033F0007B68BA68F968064809F032FD0346002B7D
:1034000001D00123FB75FB7D18461837BD4680BDF2
:103410005458012080B500AF05480AF0F1F9034681
:10342000042B14BF01230023DBB2184680BD00BF6C
:103430005458012080B582B000AF786079680348A5
:103440000AF018F900BF0837BD4680BD5458012066
:1034500080B582B000AF786000F018F800BF083780
:10346000BD4680BD80B582B000AF786000F0C4F981
:1034700000BF0837BD4680BD80B582B000AF786020
:1034800000F0C8F900BF0837BD4680BD80B400AF6A
:1034900000BFBD465DF8047B704780B582B000AFC9
:1034A0000123FB7100F00CF80346002B01D100232F
:1034B000FB71FB79DBB218460837BD4680BD0000C2
:1034C00080B582B000AF0123FB714FF40051064874
:1034D00006F0A2FB0346002B01D00023FB71FB7911
:1034E00018460837BD4680BD0008024080B584B04C
:1034F00000AF78600CF094FCF86006E0FFF78AFFFC
:103500000346002B01D1002309E00CF089FC0246A0
:10351000FB68D31A7A689A42F0D84FF0FF33184606
:103520001037BD4680BD000080B582B000AF0346B5
:10353000FB710B4B01221A70FFF76CFF0346002B47
:1035400007D1074B1B78DBB223F00103DAB2044B3F
:103550001A70034B1B78DBB218460837BD4680BD96
:103560001C00002090B587B000AF0346FB71204BD4
:1035700001221A700CF048FC0346002B30D0FFF7F4
:10358000EFFE0346002B07D1FB791846FFF7CCFF6F
:1035900003461A46164B1A70154B1B78DBB2012BEB
:1035A0001ED0144B1B68002B0ED1134B07F10804DF
:1035B0000FCB84E80F0007F10803002118460CF038
:1035C00067FD03460B4A13600A4B1B68002B07D1AB
:1035D000074B1B78DBB243F00103DAB2044B1A70DD
:1035E000034B1B78DBB218461C37BD4690BD00BFAD
:1035F0001C0000205004002008C5020880B582B0DD
:1036000000AF0346FB71FB791846FFF78DFF0346B9
:1036100018460837BD4680BD80B58AB000AFB96096
:103620007A603B600346FB73012387F8273047F23B
:103630003050FFF75BFF0346002B02DA97F8273084
:1036400032E03A687968B868FFF7B0FE034687F859
:10365000263097F82630002B24D1154B196807F136
:10366000140347F2305218460CF07AFD7B69102B98
:1036700018D1BB69012B15D10CF0D2FB386208E0E0
:10368000FFF7C8FE0346002B03D1002387F827303D
:1036900008E00CF0C5FB02463B6AD31A47F22F52F2
:1036A0009342EDD997F8273018462837BD4680BD9C
:1036B0005004002080B58AB000AFB9607A603B60EA
:1036C0000346FB73012387F8273047F23050FFF79A
:1036D0000DFF0346002B02DA97F827302EE03A68F8
:1036E0007968B868FFF77CFE0346002B24D1154BA0
:1036F000196807F1140347F2305218460CF030FDF8
:103700007B69102B18D1BB69022B15D10CF088FBFB
:10371000386208E0FFF77EFE0346002B03D100234A
:1037200087F8273008E00CF07BFB02463B6AD31A8F
:1037300047F22F529342EDD997F827301846283791
:10374000BD4680BD5004002080B58CB000AF03465C
:103750003A60FB710B46BB71012387F82F30254B74
:103760001B78DBB203F00103002B01D003233CE004
:10377000BB79032B34D801A252F823F08D3700080F
:1037800095370008AD370008C7370008002387F8D1
:103790002F3028E007F10C031846FFF74BFE7A6A3A
:1037A0003B681A60002387F82F301CE007F10C03F8
:1037B0001846FFF73FFEBB6A9AB23B681A800023A7
:1037C00087F82F300FE007F10C031846FFF732FEA1
:1037D000BB6A5A0A3B681A60002387F82F3002E060
:1037E000042387F82F3097F82F3018463037BD461E
:1037F00080BD00BF1C00002080B500AF044B1B68DB
:103800000022022118460CF06BFC00BF80BD00BFF7
:103810005004002080B500AF044B1B68002201213A
:1038200018460CF05DFC00BF80BD00BF50040020B6
:10383000DFF834D0002103E00C4B5B5843500431D7
:103840000B480C4B42189A42F6D30B4A02E0002375
:1038500042F8043B094B9A42F9D304F041FC27F0AB
:103860007FFCFDF731FF7047000005201823030897
:10387000000000203C0100203C010020A460012049
:10388000FEE780B500AF00F053FC00BF80BD80B5FF
:1038900082B000AF786000F0BBFC00BF0837BD46C7
:1038A00080BD40687047416070470000094A136856
:1038B00043F080731360A2F54E42074B52F84C1C44
:1038C0004C3A0B431360A2F57B62136843F001038B
:1038D00013607047FCED00E055CEACC5511A01EB0A
:1038E0005301B1FBF3F07047014B1868704700BFFC
:1038F000041000E0704710B504460C2127F0C1FA0F
:10390000204610BD036810B51B69044631B19847C5
:10391000A26863689B1A1844606010BD9847A06055
:10392000FBE70000024B7020024A1360DB68184777
:103930002800002054040020704710B504460421DC
:1039400027F09FFA204610BD37B50A4D0C462B686C
:1039500013B9002003B030BD1B6970200192984755
:1039600001990028F5D02B68702022465B699847A2
:103970000120EFE7540400207FB501238DF81720C4
:103980004FF47A72CDE901320DF1170200920A4626
:103990000146054806F032FA10B1034806F0FEF978
:1039A00007B05DF804FB00BFDC5701207FB50023A2
:1039B0000A464FF47A718DF817300123CDE90131B1
:1039C0000DF1170100910146054806F02BFB10B1DF
:1039D000034806F0E3F99DF8170007B05DF804FB13
:1039E000DC570120704770477047012380F874103E
:1039F00080F8753070470020704700207047836B57
:103A00000BB10846184770474FF6FF707047406883
:103A100003689B691847704738B5044600F0C8FC36
:103A20000A4A4FF0404123682046D3F88050084BA3
:103A3000A8470023074D84F84A302846FFF736FF91
:103A40000123256184F86C3038BD00BF00FC03C041
:103A500000F807C05804002008B531B90A4B4FF4EC
:103A600025710A4A0A4827F03BFAC0E90F12003ACA
:103A70000849436418BF0122003B0A7018BF0123A4
:103A8000054A137008BD00BF0CC7020844C70208EE
:103A900092C70208AE540120AF54012000F070BC60
:103AA00000F074BC70B500F0A1FC104A0023C2F80D
:103AB0008430BFF34F8FD2F8803043F6E074C3F305
:103AC000C900C3F34E335B0103EA0406014646EA2C
:103AD00081750139C2F87452F9D2203B13F1200FDD
:103AE000F2D1BFF34F8FBFF36F8F70BD00ED00E0D9
:103AF00000F08ABC00F020BC00F088BC00F090BC54
:103B000000F024BC10B5044613F0D4F92368204615
:103B1000D3F8A030BDE81040184712F090BB10B5A4
:103B200004467C2127F0ADF9204610BD90F877308F
:103B30001BB1406803681B681847184670470000AF
:103B400090F83410114B30B590F874401A788C42CC
:103B50000DD05AB90E4A0F4914880F480C800188BD
:103B60000E4D11800122298004801A7030BD002A78
:103B7000FCD00948074A0188084D1180044A14887E
:103B8000118000222C800480EFE700BFA8540120A0
:103B9000A4540120AA540120A6540120AC540120B1
:103BA000014608B5034B186801B1012113F09CF9D7
:103BB000012008BDB0540120034B00225A609A60D6
:103BC000024A1A60704700BF58040020D4C6020899
:103BD00008B501210B480CF0A5F90B4B186028B96A
:103BE0000A4B25210A4A0B4827F07AF901210A4895
:103BF0000CF098F9094B186018B9094B2821044AB0
:103C0000F1E708BDA8C9020864040020A4C802089E
:103C1000EDC802081CC90208A0C9020868040020F7
:103C200064C90208024B4FF0FF3118680CF0ACB9C0
:103C300064040020014B18680CF0F4B964040020FF
:103C4000024B002118680CF09FB900BF64040020EB
:103C5000FFF7F0BF014B18680CF0E4B968040020CE
:103C600010B5064C002120680CF08EF920684FF04A
:103C7000FF31BDE810400CF087B900BF6804002098
:103C80000CF02AB903685B6C184701207047036881
:103C90009B6A18470D4B82B01A6B42F400021A63FC
:103CA0001A6B02F400020192019A1A6942F40002AE
:103CB0001A611A6922F400021A61054B054A1A6159
:103CC0004FF08062044B9A6002B0704700380240A7
:103CD0005C5A0120E53C000800E100E040F2EF30D2
:103CE00070470000024B1B68586803685B691847FF
:103CF000B054012008B50B280BD8DFE800F01206FD
:103D0000100A0A0A0A0808080808012008BD052048
:103D1000FCE7054B6421054A054827F0E1F800203F
:103D2000F4E70220F2E700BFB0C90208CBC90208DD
:103D300017CA020808B50A2809D8DFE800F01006FB
:103D40000E080808080606060600012008BD054BF7
:103D50008521054A054827F0C3F80020F6E7022030
:103D6000F4E700BFB0C902085DCA020817CA02081A
:103D70002DE9F84391F81D800C464046FFF7BAFF45
:103D8000A77F05463846FFF7B5FF06463846FFF7DA
:103D9000D1FFA18A628B534B521A9E461A649A61D4
:103DA000228B521A1A61E28A586342EA014221695F
:103DB0005A646268D963DA60D4F800C094F81C9041
:103DC000BCF1800F4FEA09623BD015D8BCF1200F3F
:103DD00045EA02007AD0BCF1400F77D0BCF1040F65
:103DE0002BD02A43B8453F4B42F40032DA610CBF76
:103DF00040F201223C4A1EE0BCF5807F07D0BCF5B2
:103E0000007FEED142F4003242F0090203E042F4B6
:103E1000003242F00A02DA61E0680202440102F470
:103E20007802C00004F47C44C0B2224302431A6208
:103E30002E4A5E6259611A6044E040F40030D86155
:103E4000F6E7A0682A43041D42F40032DC62DA611E
:103E500002785E62596142B1012A1CD0244B40F2C3
:103E60000F11244A244827F03BF842880125D969DC
:103E7000501E21F47F4222F0100242EA0022DA6151
:103E8000184CE36943F02003E361E3699B0614D512
:103E9000FFF7F6FEF9E74288B9F1FF05D96902F1AB
:103EA000FF3018BF012521F47F4222F0100242EAC0
:103EB000002242F01002DA61E2E71023A3601DB194
:103EC0000A4B2360BDE8F883074BFAE740F4003063
:103ED000064BCEF81C00CEF82460CEF81410CEF8B5
:103EE0000030EFE700B002400102010001020200D1
:103EF000AACA0208C4CA020817CA0208F8B58E7F07
:103F00000C463046FFF716FFA78AE18A628B1E4BEC
:103F100041EA07412569D21B58635964DD631A647D
:103F20002168082918D19A611A615862174A217FBD
:103F300042EA0162DA61E1680A02480102F47802A9
:103F4000C90000F47C40C9B202430A431A62104A15
:103F50005D61DD601A60F8BD0022D8611A61E16818
:103F60001EB99963084B0B4AF4E70A02480102F4B0
:103F70007802C90000F47C40C9B202430A43217FA1
:103F800042EA01629A63EDE700B0024009000100D5
:103F90000102020001020300054B4FF08062036042
:103FA000044BC3F88820BFF34F8FBFF36F8F704768
:103FB0000CCB020800E100E010B50446FFF7ECFF6F
:103FC0004FF44261204626F05CFF204610BD000001
:103FD00070B504460A4B0C3000262546602260600E
:103FE0002672667245F8203B294613F0E9F804F57D
:103FF0004263EE602035AB42FBD1204670BD00BF6E
:104000000CCB0208012070470C2070470C2303FBE7
:104010000100083070470C2303FB01000830704793
:104020000120704743F67C40704743F67C4303FB16
:1040300001000830704743F67C4303FB0100083061
:104040007047012070471020704700EB01100830C6
:10405000704700EB011008307047084600F00CBBB9
:10406000034B10B5044603600EF036FE204610BD2B
:10407000C4CB020810B50446FFF7F2FF1421204616
:1040800026F0FFFE204610BD034B10B5044603602A
:104090000EF022FE204610BD90CB020810B504465B
:1040A000FFF7F2FF43F68441204626F0EAFE204661
:1040B00010BD0000034B10B5044603600EF00CFE6B
:1040C000204610BD5CCB020810B50446FFF7F2FF96
:1040D0001821204626F0D5FE204610BD094B10B50C
:1040E0000446036000F572503030FFF7B9FF04F169
:1040F0002C00FFF7C9FF04F11400FFF7DBFF204697
:1041000010BD00BFF8CB020808B50248FFF7E6FF74
:1041100008BD00BF7004002010B50446FFF7DEFFA5
:1041200043F62861204626F0ACFE204610BD000074
:104130002DE9F34100F0E2F90024054600F0E2F930
:104140002346014622462846009419F0BDFB244B25
:10415000244A2046244D1A6002F028FE234819F014
:10416000F5FA2B78BFF35B8FDB0733D4284626F0B4
:104170008AFE78B31E4C1F4F1F4B04F1140007F149
:10418000200604F12C0823606060C4F80880E76012
:1041900026610EF0A3FD194B404663610EF09EFDB3
:1041A000174B3846E3620EF099FD164B07F11400E9
:1041B0003B6003F0B9F8224607F11401304602F0E3
:1041C000F1FF304600F058FA284626F068FE0E4807
:1041D00026F0A4FE0D4802B0BDE8F041FFF71CBC7C
:1041E0002C550120384F00206C04002020000020B6
:1041F0007004002020410020F8CB02085CCB0208AC
:1042000090CB0208C4CB020809410008BC4E002034
:10421000014812F078B800BFBC4E002070B5244BA6
:10422000244C254E254D23603046FFF7D1FE28460D
:104230001CF0D0FB224B00224FF480714FF4F07041
:10424000DC60204C1A8583F82A20DA621A861A6606
:1042500083F86C201A67C3E912121B49C3E91912CB
:104260004FF080715967012183F8781017490B606E
:10427000174908804FF48871C3E90422C3E9062274
:10428000C3E90822C3E90E22C3E91022C3E91422BC
:10429000C3E91622C3E9016521800E4C83F834205E
:1042A00022700D4C0D4A20800D481A60018070BDAF
:1042B000FCC60208984200209C4200203C4F00208F
:1042C000BC4E0020A654012001000001B054012082
:1042D000A4540120A8540120AA540120E0C70208D8
:1042E000AC5401200148FFF757BE00BF9C4200209C
:1042F000104A002370B5C2F88430BFF34F8FD2F854
:10430000803043F6E074C3F3C900C3F34E335B015E
:1043100003EA0406014646EA81750139C2F874527F
:10432000F9D2203B13F1200FF2D1BFF34F8FBFF32F
:104330006F8F70BD00ED00E0034B902283F85A238D
:1043400083F85823704700BF00E100E0094A0A499A
:10435000D3680A48C3F30A03013B9BB20B8011697F
:10436000C1F30A01013901801364536B43F0010367
:104370005363704700680140B64F0020B44F0020DF
:10438000014B986A704700BF84680140024B0122CC
:10439000996243F8602C704784680140034B5B6965
:1043A000DB0301D5FFF7A4BF704700BF00ED00E0BD
:1043B00070B5044611F095FF2368DD6D16F086F8A0
:1043C00001462046A84723682046054AD3F8805076
:1043D0004FF040410023AC46BDE87040604700BF4D
:1043E00000FC03C011F064BF11F06EBF08B511F0FE
:1043F0002CFF044B5B69DB0303D5BDE80840FFF7E6
:1044000077BF08BD00ED00E012F087B8034B4FF016
:1044100080629A604FF080729A60704700E100E01D
:10442000084B4FF08062C3F88820BFF34F8FBFF373
:104430006F8F4FF08072C3F88820BFF34F8FBFF3A8
:104440006F8F704700E100E0134B144A1B6C11881A
:104450008B4210B5124C13D1124B198806F076FB23
:10446000226892F86630013382F86630FFF7F2FB7B
:10447000206812F01FFD0020BDE81040FFF7B2BA1F
:1044800006F064FB0020FFF7AEFA20680368BDE881
:104490001040DB69184700BF00680140B64F00209C
:1044A000B0540120B44F0020704710B504460421D9
:1044B00026F0E7FC204610BD08B505291CD8DFE82A
:1044C00001F003070B0F131702F0BCFC006808BDD6
:1044D00002F0B8FC4068FAE702F0B4FC8068F6E746
:1044E00002F0B0FCC068F2E702F0ACFC0069EEE755
:1044F00002F0A8FC4069EAE70020E8E700487047BE
:1045000018CC02081020704713B5002451B103687D
:1045100001AA01948DF803409C680DF10303A047A4
:1045200002B010BD0846FBE740897047808970479C
:104530008088704783798088184480B27047C0793A
:1045400000F07F007047C079C0097047704710B510
:104550000446082126F095FC204610BD704700F562
:1045600096730868496803C3704770477047416095
:10457000704770470123037270477047704710B44B
:1045800041680346C2689B68541001EB6200D20781
:1045900048BF0A595DF8044B48BFD35818474368D1
:1045A0002BB183682BB9C06800F001007047184632
:1045B00070470120704710B504460C2126F061FCBD
:1045C000204610BD10B50446102126F05AFC2046A6
:1045D00010BD10B504464FF4AC7126F052FC2046D5
:1045E00010BD10B515F072FF0368BDE810401B6BDD
:1045F000184710B50446D0F83C0158B10368DB6891
:10460000984738B1D4F83C0103689B689847002369
:10461000C4F83C3110BD0000F8B5044617460E46FC
:1046200015F0BEFF104B00251C6029460F4BC4E956
:1046300054760F4E236030680E4BC4E95255C4E9DE
:1046400050350368C4E94E559B689847284602F0E8
:10465000ADFB336893F876200AB1D86C00B998683E
:104660001DF0E9FE2046F8BD1C550120A8D0020827
:10467000B054012090D00208064BC0F84401C0F8A5
:1046800048310023C0F84C3100F5A073C0F83C312C
:10469000704700BFD94700082DE9F84F07469068DA
:1046A0009946884603681446DDF828A01B6A984797
:1046B00043F67B43984205D8414BA321414A4248E7
:1046C00026F00EFC606803681B6A98470F2803D821
:1046D0003E4BA4213B4AF2E7E06803681B6A984717
:1046E0000B2803D83A4BA521364AE8E715F0EEFE31
:1046F00015F03AFFD9F8000010B10368DB6898475D
:10470000D9F8000010B103681B689847386810B1E9
:1047100003685B699847D8F8000010B103685B68CC
:104720009847386810B103681B689847D8F80000AC
:1047300010B103689B689847E06800214FF0000BB8
:1047400003685B6A9847234B0546C0F804B00360D2
:10475000594680F808B0A06803685B6A9847064627
:1047600003F038F96068594603685B6A9847044665
:10477000314602F06BFEC9F80050C8F800403E60B8
:10478000E4B1231DCAF8043030463368C4F808A0E9
:10479000DB68F4639847236820461B6898472946DE
:1047A000304617F0ACFB2B6828461B6998472B68EE
:1047B00028465B6998472046BDE8F88F2346E1E725
:1047C00068CD0208F6CD0208FACE020841CF0208F1
:1047D000E4CF0208ECD00208D0F8543107B500F558
:1047E0009C710093044BD0F850210448FFF754FF0C
:1047F00003B05DF804FB00BF105501200C550120EB
:10480000006A7047406A704770478B888069DB0A8E
:104810000A6850F823001044704710B5C2B1137BEA
:10482000B3B1547BD27A240204F4E0641443C26925
:1048300098B202EB840213888B4202D192F90200F3
:1048400010BD05D80138043280B20028F3D1F7E753
:104850000020F5E710B50446282126F012FB20467B
:1048600010BD000030B589B00446BDF85050069523
:10487000BDF84C5005959DF8405004959DF83C506E
:1048800003959DF8385002959DF8345001959DF898
:104890003050009516F098FE064B20462360119B81
:1048A000A361129BE361159B2362169B636209B0AF
:1048B00030BD00BF10D102080020704781807047D2
:1048C000C1807047018170474181704770477047D0
:1048D00070477047704710B4C4880368121B8488FF
:1048E0001B6D091B12B25DF8044B09B218474FF655
:1048F000FF7383814FF0FF3303621368C36110605D
:104900007047806A704770477047704770477047BC
:1049100090F825201AB190F8242002B11860704751
:104920000022028042808280C2807047036870B596
:104930000446DB6A15469847236820462946DB6D06
:10494000BDE87040184770B50D79044690F82C30DA
:104950003DB93BB123682046D3F88030BDE87040B4
:1049600018477BB1B5FA85F320465B0984F82C30F3
:104970002368D3F884309847236820465B699847BA
:10498000002DE7D070BD7047704770477047704783
:10499000704770477047704770477047704770475F
:1049A000704770477047704770477047704770474F
:1049B0007047072070470220704790F82C302BB1C9
:1049C000C26EC26523B1436F03667047826EF8E71B
:1049D000036FF9E708B590F82C3033B1D0F8B83050
:1049E000C0F8A830FFF7E9FF08BDD0F8B430F7E70A
:1049F000704770477047704738B50546064B044608
:104A0000C03045F8043B03681B6898476368284634
:104A10001B689847204638BD54D9020838B5074B63
:104A200004464FF47175036063596019A03D1B681B
:104A3000984715F19C0FF7D1204638BD3CD90208A4
:104A4000704770477047F0B446680446C568A4686C
:104A50006F1006EB6500ED0744BFF5592C59A446CD
:104A6000F0BC604743682BB183682BB9C06800F085
:104A700001007047184670470120704770B44568C0
:104A80000346C4689B68661005EB6400E40744BFF6
:104A9000AC59E35870BC184743682BB183682BB9F5
:104AA000C06800F001007047184670470120704749
:104AB00030B444680346C2689B68551004EB62003A
:104AC000D20748BF625930BC48BFD3581847436823
:104AD0002BB183682BB9C06800F0010070471846FD
:104AE00070470120704730B444680346C2689B6831
:104AF000551004EB6200D20748BF625930BC48BF72
:104B0000D358184743682BB183682BB9C06800F0AD
:104B1000010070471846704701207047838B8B4215
:104B200086BF00EB810148680020704710B5031D67
:104B3000848B002291B28C4208D953F8041B104692
:104B4000013291F837100029F4D010BD4FF0FF303A
:104B5000FBE7036810B51B6904469847011E06DB96
:104B60002368204689B2DB68BDE810401847002062
:104B700010BD10B50430048B00239AB2944205D9BD
:104B800050F8042B013382F83810F6E710BD838B00
:104B90001BB1436893F8380070471846704730B42B
:104BA00044680346C2689B68551004EB6200D20754
:104BB00048BF625930BC48BFD358184743682BB12F
:104BC00083682BB9C06800F0010070471846704731
:104BD00001207047A0F878117047B0F8780170474D
:104BE00090F82D3080F8AE3080F85A30704790F849
:104BF0002D3080F85A307047A0F844107047B0F854
:104C00004400704770B50D4604460121284613F054
:104C10003FFF2368294620465B6ABDE8704018477D
:104C200010B50446FFF7FAFE40F26441204626F034
:104C300028F9204610BD10B50446FFF7DDFE4FF4FD
:104C4000BE71204626F01DF9204610BD10B5044661
:104C5000782126F016F9204610BD10B50446BC2177
:104C600026F00FF9204610BD10B504465C2126F051
:104C700008F9204610BD10B504464FF4C87126F05F
:104C800000F9204610BD10B50446482126F0F9F879
:104C9000204610BD10B50446102126F0F2F820463B
:104CA00010BD10B50446102126F0EBF8204610BDCB
:104CB00010B50446102126F0E4F8204610BD10B5CA
:104CC0000446102126F0DDF8204610BD10B504463C
:104CD000102126F0D6F8204610BD0000034B10B579
:104CE000044603600FF032FF204610BD88D602084C
:104CF00010B50446FFF7F2FFFC21204626F0C1F86C
:104D0000204610BD094B10B50446036000F5A750BE
:104D10000830FFF771FE04F584500430FFF77EFE83
:104D200004F19800FFF7DAFF204610BD18DA0208F8
:104D300010B50446FFF7E6FF43F66C41204626F027
:104D4000A0F8204610BD000008B58BB2062B05D98F
:104D5000054B5421054A064826F0C2F8A02301FB62
:104D60000300043008BD00BF60D102087BD10208F7
:104D700007D2020808B58BB2012B05D9054B542187
:104D8000054A064826F0ACF8BC2301FB03000430BA
:104D900008BD00BF60D1020866D2020807D202082F
:104DA0000368828D70B51E6B0446114B8DB21B6873
:104DB0002BB9104BAE21104A104826F091F810493B
:104DC0000988914203D80F4BAF210B4AF4E713F83F
:104DD00012200D4B1B6853F822000368DB6A9847CA
:104DE000281A334601B22046BDE87040184700BF7C
:104DF00020550120FBD202083DD302086BD30208E4
:104E000024550120B2D302082855012008B5838B10
:104E1000052B05D9084B4121084A094826F060F8BE
:104E200000F120028A6200F13002CA635A1C8283B8
:104E300000EB8300416008BD04D402083DD40208A1
:104E4000ABD4020810B504462C300EF065FB04F11B
:104E5000C4000EF061FB04F58870BDE810400EF050
:104E60005BBB70B541F2880541F2E846044600F6A6
:104E7000F460FFF7E7FF63596019A035D3F880307D
:104E80009847B542F7D12C44201D02F094FED4F887
:104E9000C03004F1C000D3F88030BDE8704018473E
:104EA000F7B54FF6FF73818D044699422AD0164B11
:104EB0001B682BB9154BAE21154A164826F010F881
:104EC000154A12888A4203D8144BAF21104AF4E7DE
:104ED00003EB410213F81100114B55781B68C5F321
:104EE000810553F820603368DF690E4B186801F0C4
:104EF00099FF00230246294600933046E36BB847EA
:104F000003B0F0BD0020FBE720550120FBD20208D2
:104F10003DD302086BD3020824550120B2D3020806
:104F2000285501202C550120818D4FF6FF739942A1
:104F300070B504461ED00368DD6E0F4B1B682BB99D
:104F40000E4BAE210E4A0F4825F0CAFF0E4B1B88B0
:104F50008B4203D80D4BAF21094AF4E70C4B18687C
:104F600001F060FFE26B0146AC4620460023BDE83D
:104F700070406047002070BD20550120FBD2020820
:104F80003DD302086BD3020824550120B2D3020896
:104F90002C55012010B50446006B50B10368DB6846
:104FA000984730B1206B21460368BDE810409B68EC
:104FB000184710BD00F52A72914202D103689B6D1B
:104FC000184700F6B432914202D103685B6CF7E7F0
:104FD00000F62842914202D103681B6CF0E700F60C
:104FE0009C42914202D10368DB6BE9E700F5516214
:104FF000914202D103689B6BE2E7704700F5F672BD
:105000008A4202D10368DB6D1847704710B40C4622
:10501000114600F5DB62944204D103681B6D5DF814
:10502000044B184700F2D472944202D103689B6C7F
:10503000F5E700F50D62944202D10368DB6CEEE700
:1050400000F64C22944202D103685B6DE7E75DF8FD
:10505000044B704700F58162914202D103681B6ED8
:10506000184700F56272914202D103685B6EF7E760
:1050700000F57272914202D103689B6EF0E700F571
:105080009162914202D10368DB6EE9E700F552724A
:10509000914202D103681B6FE2E700F589629142F9
:1050A00002D103685B6FDBE7704713B5044608461F
:1050B00011461A4604F58453043398420CD1036810
:1050C00001929B689847236801461B6B019A204612
:1050D00002B0BDE81040184704F5A75308339842C2
:1050E00007D1036801929B689847236801465B6B70
:1050F000ECE702B010BD13B50446406C019158B105
:105100000368DB68984738B1606C019903689B6855
:1051100002B0BDE81040184702B010BD70B504469B
:105120000D460026A28BB3B29A420CD904EB83033E
:105130005868A84205D090F8373013B1002113F019
:10514000A7FC0136EEE7206C50B10368DB68984796
:1051500030B1206C29460368BDE870409B68184751
:1051600070BD2DE9F04104460EF078FF94F87431DB
:10517000002B53D0B4F87631B4F8785101339BB298
:10518000AB42A4F8763149D35B1BB4F88021D4F844
:10519000846100219DB2B4F87C31D21A2846B4F85B
:1051A0007A3112B2B047B4F87E31B4F882210646A3
:1051B0000021D4F88871D21A2846B4F87A3112B294
:1051C000B847B4F87E21B4F87C110244204631443B
:1051D00012B209B2FFF77FFBB4F87831B4F87A1154
:1051E000B4F876210B449A4218D3002384F8743122
:1051F000A4F8763115F06AF9214615F09FF9D4F834
:105200008C0158B10368DB68984738B1D4F88C0139
:1052100021460368BDE8F0419B681847BDE8F0816E
:1052200090F840302DE9F0410446002B4FD0B0F803
:105230004230B0F8445001339BB2AB42A0F8423048
:1052400045D35B1BB0F84C20066D00219DB2B0F831
:105250004830D21AB0F84630284612B2B047B4F8F7
:105260004A30B4F84E2006460021676DD21A28460F
:10527000B4F8463012B2B847B4F84A20B4F848102F
:1052800002442046314412B209B2FFF724FBB4F8BD
:105290004430B4F84610B4F842200B449A4216D376
:1052A000002384F84030A4F8423015F00FF921466D
:1052B00015F044F9A06D50B10368DB68984730B130
:1052C000A06D21460368BDE8F0419B681847BDE822
:1052D000F0810000074A02600022C0E90122C0E913
:1052E0000322C0E90522C0E907224FF480728284BC
:1052F000704700BF4C060308036870B50446DB6ABC
:10530000154698472368204629461B6BBDE8704028
:10531000184770B504461D46BDF91060FFF7ECFF55
:105320002368294620465B6B984723683146204610
:105330009B6BBDE87040184710B50446FFF7CAFFE5
:10534000024B204623600023A36210BD94E90208AB
:1053500010B504462622002125F048FF2046FFF71D
:10536000B9FF044B20462360FF2384F82630002336
:10537000A36210BD2000030838B504460D4626225E
:10538000002125F033FF2046FFF7A4FF064B2046FF
:10539000294623602B88E384FF2384F8283013F008
:1053A00059FA204638BD00BF4402030810B5044630
:1053B0002622002125F01AFF2046FFF78BFF074B1E
:1053C0004FF47F0220462360054BA3624FF6FF7324
:1053D000A3850023C4E90C32238710BD78FF02089F
:1053E00060CD020810B504462622002125F0FEFEFD
:1053F0002046FFF76FFF054B204623600023A36282
:1054000084F82C30012384F8243010BD68FE020893
:1054100010B50446FFF7E6FF084B4FF0FF32204679
:1054200023604FF6FF73E3856FF07F43C4E90C23DD
:10543000002384F83830E36310BD00BFAC020308DA
:10544000FF22002370B502720446124A124E026017
:105450003268436092F87610C0E9033309B1D06C2A
:1054600000B9906803685B6A98473368B0FA80F5C2
:10547000D86C6D0928B103685B6A9847002808BF9B
:1054800001252DB9054B2C21054A064825F028FD9C
:10549000204670BDD8FA0208B054012001D5020898
:1054A0005FD5020898D5020810B50446FFF79AFFA9
:1054B0004FF6FF73044A2046E385238684F8323092
:1054C0002260A38610BD00BFD4FE020870B504465A
:1054D000FFF732FF4FF47F4300252646A3850123C3
:1054E000256384F82430134B46F8343B3046FFF7ED
:1054F0002FFF114B2A462946636330462566A4F8E0
:105500006450C4E91A55C4E91C55FFF7F5FE31464D
:10551000204626460EF000FF084B46F8783B304602
:10552000FFF744FF20463146C4E92D550EF0F4FE46
:10553000204670BD14D70208E0010308A8D702086E
:105540002DE9F04F04460025DFF8B8B304F5E07606
:1055500004F5F67904F52A7804F5387A04F54777E6
:105560002DED108BB5B016F04DFB2346DE4AE563FA
:1055700043F8402B18462593FFF7EAFE04F16C032D
:105580004FF6FF7232A91846ADF8C8200F93FFF707
:10559000F3FE04F19803184608EE903A0FF0EAFB88
:1055A000D24A04F5CA73C4F89051C4F89820012275
:1055B0001846289384F8BC20FFF7BEFE3046FFF75C
:1055C000BBFE4846FFF782FF4046FFF76DFF50469F
:1055D000FFF7ECFE3846FFF7AFFE04F552731846AE
:1055E0000293FFF715FF04F5627318460393FFF764
:1055F0000FFF04F5727318460493FFF709FF04F5D3
:10560000816318460593FFF703FF04F58963184685
:105610000693FFF7FDFE04F5916318460793FFF725
:10562000F7FE04F5996318461093FFF7BFFE04F2E6
:10563000045318461193FFF7B9FE04F5A863184602
:105640001293FFF7B3FE04F27C5318461393FFF74F
:10565000ADFE04F5B76318461493FFF7A7FE04F2F6
:10566000F45318461593FFF7A1FE04F5C6631846D8
:1056700009EE903AFFF760FE04F25C631846169359
:10568000FFF794FE04F5D36318461793FFF78EFED9
:1056900004F5DB63C4F898B61846C4F8D4560CEE8B
:1056A000103A0FF0AFF904F2D47318460CEE903AAA
:1056B0000FF0A8F904F50D6318460DEE103A0FF03F
:1056C000A1F904F6CC1318461893FFF76FFE04F601
:1056D0000C23C4F8CCB91846C4F8085A1993FFF73C
:1056E00065FE04F64C23C4F80CBAC4F8485A1846B0
:1056F0000DEE903A0FF086F904F6483318461A93E7
:10570000FFF754FE04F68833C4F848BB04F6F46B84
:105710001846C4F8845B0AEE903AFFF70DFE04F6D3
:10572000B43318461B93FFF7BFFE04F6EC3318465C
:105730001C93FFF73BFE04F6284318460B93FFF734
:10574000B3FE04F5466318461D93FFF72FFE04F6DB
:105750009C4318461E93FFF7A7FE04F6D443184651
:105760001F93FFF723FE04F5516318462093FFF7BC
:105770009BFE04F6485318462193FFF717FE04F6E4
:10578000845318460BEE103AFFF7D6FD04F55B6321
:1057900018460EEE103A10F065F904F66C631846E0
:1057A0002693FFF7D5FD04F6986318462293FFF77A
:1057B000FDFD4F4AC4F8D45E5846C4F8982E84F8CC
:1057C000D85EA4F8DA5EC4F8DC5EC4F8E05EC4F823
:1057D000E45EC4F8E85EC4F8EC5EC4F8F05E0EF077
:1057E00073F9444A41F28403C4F8F42E41F268028A
:1057F000A55441F26A02A55241F26C02A55041F251
:105800007002A55041F27402A55041F27802A550F1
:1058100041F27C02A55004F584521560E21804F5AB
:1058200084552C92344A0835E25004F5A7530833C6
:1058300024932846A03502F0B3F9249B9D42F8D169
:105840002E4A41F2E843281D41F2D475E25002F09D
:10585000BBF904F5AD50083002F0B6F904F5B353C6
:10586000043318460EEE903AFFF7A0FD04F5B55349
:10587000184609EE103A0DF0D3FA631918462D9325
:10588000FFF7DEFD1E4A41F2E87362510025E55044
:1058900004F5BF530C3318460C93FFF759FD04F57C
:1058A000C053183318460D93FFF752FD41F64403D9
:1058B000E21810460892FFF779FD124941F64403B9
:1058C000E150089BDD6304F5C4530433184608EE29
:1058D000103A0DF0A5FA41F6B813E21810462992D5
:1058E000FFF7AEFD10E000BF18DA020888D6020804
:1058F00008D602083CD802083CD9020854D902084C
:10590000B8FA020838010308CE4A41F6B813E2504B
:1059100041F6CC13E55004F5CE53103318460BEE88
:10592000903AFFF709FD04F5CF5332A91C330993D0
:105930004FF6FF730998ADF8C830FFF71DFD04F569
:10594000D153083318460FEE103AFFF72FFD04F538
:10595000D353043318460FEE903AFFF727FD04F5B2
:10596000D55318462393FFF721FD41F6DC2304F5B8
:105970000150E2180C300AEE102AB34AE2501AEE37
:10598000103AB24A9D8341F6FC23E118E25041F6F9
:10599000043381ED01AA2421E15041F608330121AD
:1059A000E15041F60C33E250E118282241F614335D
:1059B00081ED01AAE25041F618330122A449E250D8
:1059C0001AEE103AC3E9105541F6FC73E2180A9238
:1059D000A04AE2500A9B5C6042F20403E15042F2AA
:1059E0000803E55042F20C03E1182A919A49E1506C
:1059F0002A9B9A495C6042F21403E15042F2180378
:105A0000E55042F21C03E1180E919549E1500E9BBE
:105A100094495C6042F22403E15042F22803E550CD
:105A200042F22C03E118E25042F234038E4A2B91E9
:105A30004C604FF4E151E25042F23803E55042F23B
:105A40003C03E2182792894AE250279B884A5C600F
:105A500042F24403E25042F24803E55013F060F88A
:105A60004FF488732A462946259800934FF4F07323
:105A7000FFF74FFC4FF07F432A462946A3660F9855
:105A8000FFF73AFC32A90F98ADF8C85012F0E2FEC9
:105A90002A46294618EE900AFFF72EFC322118EE0E
:105AA000900A0FF049F8322118EE900A0FF0B2F880
:105AB000704B289918EE900AC4F89C310FF008FA40
:105AC0006C4B5A212A4604F50870C4F8C83100917D
:105AD000C9232946FFF71DFC674A4FF00A01674BAF
:105AE0004846A4F850126649C4E99523654BC4E9B9
:105AF0009713D4F8EC31D3F884309847624B04F50F
:105B0000197032A932931A232890ADF8CC3012F0D4
:105B1000B4FAB4F9F6315A21B4F8F4212898A4F86B
:105B20006C222022A4F86E32C92300910121FFF7D4
:105B3000F0FB4FF0FF314846C4E9A811FEF74AFFD9
:105B40005A21C9239A2248460091FF21FFF7E1FB21
:105B50002A993046C4F81C1249460EF0DDFB404637
:105B60004D2240F22311FFF7C7FB4FF0080131A887
:105B700032AAADF8C4104FF009014FF00609ADF894
:105B8000C810A4F8DC120146404612F089FC4046D9
:105B9000012112F0B1F80A993046C4F8D0124146FA
:105BA0000EF0BAFB2B2250464FF49171FFF7A4FB85
:105BB0004FF0FF30344B4FF00408C4F810034FF09F
:105BC0001900A4F81453ADF8CC0032A83293014662
:105BD000504612F052FA514630464FF0030A0EF08A
:105BE0009BFB314618EE900A05260FF071F9214A09
:105BF000F9210298C4F824233222FFF77DFB31A853
:105C000032A9ADF8BC80034630A8009102462FA807
:105C1000ADF8C4A001460298ADF8C890ADF8C060D8
:105C200012F08DFE2946029812F032FF3846029992
:105C300084F880530EF070FB642216210398FFF75E
:105C40005BFB23E0B8FA020884D902086CD9020889
:105C5000B54F0008B8D90208D0D90208FD4F000896
:105C6000E8D902080D5000085550000800DA020873
:105C7000AB500008E0011001524F4BFFCFCABEFFEE
:105C80002E2B28FFA39484FF60CD020831A832A9EF
:105C9000ADF8BC80034630A8009102462FA8ADF8AD
:105CA000C4A001460398ADF8C890ADF8C06012F0EA
:105CB00046FE2946039812F0EBFE3846039984F815
:105CC000C0530EF029FB962216210498FFF714FB0F
:105CD00031A832A9ADF8BC80034630A80091024635
:105CE0002FA8ADF8C4A001460498ADF8C890ADF84F
:105CF000C06012F024FE0121049812F0C9FE38465B
:105D0000049984F800540EF007FB322216210598FE
:105D1000FFF7F2FA31A832A9ADF8BC80034630A8EB
:105D2000009102462FA8ADF8C4A001460598ADF831
:105D3000C890ADF8C06012F002FE2946059812F036
:105D4000A7FE3846059984F840540EF0E5FA64221F
:105D5000F9210698FFF7D0FA31A832A9ADF8BC8036
:105D6000034630A8009102462FA8ADF8C4A0014612
:105D70000698ADF8C890ADF8C06012F0E0FD294675
:105D8000069812F085FE3846069984F880540EF085
:105D9000C3FAC82216210798FFF7AEFA31A832A934
:105DA000ADF8BC80034630A800914FF007080246CA
:105DB0002FA8ADF8C4A04FF0230A01460798ADF80C
:105DC000C890ADF8C06012F0BAFD2946079812F0ED
:105DD0005FFE3846079984F8C0540EF09DFA3B22C6
:105DE000722357211098CDF800A0FFF792FA4FF0D8
:105DF000FF304FF00901704BC4F8F80432A8ADF839
:105E0000CC10A4F8FC5401461098329312F035F9E6
:105E1000384610990EF080FA1D206C226423592117
:105E200000901198FFF775FA4FF0FF304FF008011E
:105E3000614BC4F83405ADF8CC1032A91198A4F820
:105E40003855329312F019F9384611990EF064FA68
:105E50001F239D225921129800937223FFF759FAAC
:105E60004FF0FF31544B1298C4F8701532A9A4F8C2
:105E700074553293ADF8CC8012F0FFF83846129981
:105E80000EF04AFA1B21D122712313980091582158
:105E9000FFF73FFA4FF0FF31474B1398C4F8AC15AA
:105EA00032A9A4F8B0553293ADF8CC9012F0E5F8D1
:105EB000384613990EF030FA3B2272234FF49D714D
:105EC000149804F5D959CDF800A0FFF722FA4FF045
:105ED000FF31394B09F10409C4F8E8154FF01B01F3
:105EE0001498ADF8CC1032A9A4F8EC55329312F006
:105EF000C4F8384614990EF00FFA6B2272234FF44F
:105F00009D711598CDF800A0FFF703FA2A4B4FF0CA
:105F1000FF31159832931C23C4F8241632A9A4F833
:105F20002856ADF8CC3012F0A8F8384615990EF086
:105F3000F3F9394618EE900A16270EF0C9FF1F4AEA
:105F4000B3231621C4F838261D2216980092EA229F
:105F5000FFF7DFF94FF0FF32174B32A9C4F88C2658
:105F60001698A4F890563293ADF8CC7012F085F8DC
:105F7000169919EE900A0EF0CFF920233322E22170
:105F80000093F2231798FFF7C4F90D4BA4F8CC56F1
:105F9000C4F8C8360B4B1B682BB90B4BAE210B4A10
:105FA0000B4824F09DFF0B4B1B880A2B16D80A4B7D
:105FB000AF21064AF4E700BF60CD0208E0011001FE
:105FC0002DF705FF20550120FBD202083DD3020822
:105FD0006BD3020824550120B2D30208E04B0A21FA
:105FE0004FF07D0A186800F01DFFDE4A03460421C9
:105FF000484617F09DFB4FF00401DB4B1798C4F89F
:10600000D4964FF00109ADF8CC1032A9329312F0BA
:1060100034F8179919EE900A0EF07EF939463222BB
:106020001CEE100AFFF768F932A84FF0020131AAFE
:10603000034630A8ADF8C41001461CEE100AADF8B6
:10604000C090ADF8C8800EF039FD2B46424631466F
:106050001CEE100ACDE9005A0EF0A4FB32221421E6
:106060001CEE100A0EF00BFB1E211CEE100A0EF0A7
:1060700092FA0E9919EE900AC4F8D0171CEE101A75
:106080000EF04AF9394696221CEE900AFFF734F9D1
:106090000DF1C80C4FF0020131AA63460DF1C00C9E
:1060A0001CEE900AADF8C4106146ADF8C090ADF892
:1060B000C8800EF003FD2B46424631461CEE900A86
:1060C000CDE9005A0EF06EFB632229461CEE900AC1
:1060D0000EF0D5FA0A211CEE900A0EF05CFA0E9929
:1060E00019EE900AC4F8CC181CEE901A0EF014F9B0
:1060F0003946C8221DEE100AFFF7FEF80DF1C80C54
:106100004FF0020031AA63460DF1C00CADF8C40097
:106110001DEE100A6146ADF8C090ADF8C8800EF0D3
:10612000CDFC2B46424631461DEE100A4FF01409B5
:10613000CDE9005A0EF036FB632229461DEE100A07
:106140000EF09DFA0A211DEE100A0EF024FA0E99A7
:1061500019EE900AC4F8C8191DEE101A0EF0DCF8FA
:106160004FF01B0CDF239A22E2211898CDF800C0D3
:10617000FFF7CFF841F62C334FF0FF3CA4F8005A5C
:10618000E2181898C4F8FCC90DF1C80CE552764B1A
:106190006146C4F8082A3293ADF8CC9011F06DFF37
:1061A000189919EE900A0EF0B7F84FF0190CDF238A
:1061B000CD22E2211998CDF800C0FFF7AAF841F6E8
:1061C00034334FF0FF3CA4F8405AE2181998C4F851
:1061D0003CCA0DF1C80CE552634B6146C4F8482A2D
:1061E00032931523ADF8CC3011F047FF199919EE11
:1061F000900A0EF091F8394632AF64221DEE900AF3
:10620000FFF77AF83B464FF001014FF0020030AF44
:1062100031AAADF8C010ADF8C40039461DEE900AA1
:10622000ADF8C8800EF04AFC2B46424631461DEEC2
:10623000900ACDF804A000954FF017080EF0B2FABE
:10624000502249461DEE900A0EF019FA32211DEE39
:10625000900A04F5D9570EF09EF90E9919EE900A9E
:10626000AA46C4F8441B1DEE901A0EF055F8F2230E
:10627000E2216A221A981C37CDF80080FFF749F80E
:106280003A49A4F87C5BC4F8781B39490B68002BA9
:106290003FF483AE37490B88182B7FF688AE304A1F
:1062A0001821106800F0BEFD2E4A0346042138462E
:1062B00017F03EFA32AA2C4B11461A98C4F8847B88
:1062C0004FF008073293ADF8CC8011F0D6FE1A9942
:1062D00019EE900A0EF020F819EE901A18EE900AB6
:1062E0004FF009080EF0F4FD234A1B983C21C4F836
:1062F000902B3222FFF700F80DF1C80E1B98724662
:106300000DF1C40EA4F8E88B7146ADF8C470ADF879
:10631000C88012F0C5F80A991E271AEE900AC4F830
:10632000DC1B1B990DF0F8FF9A221C98CA230097DA
:10633000E221FEF7EEFF4FF0FF3E0B4BC4F81CECE2
:106340004FF0030E1C98ADF8CCE00DF1C80EA4F888
:10635000205C7146329311F090FE1C990EE000BF54
:106360002C550120FAD5020860CD02082DF705FF53
:106370002055012024550120E00110011AEE900A59
:106380000DF0CAFF0B9864223D21FEF7B5FF0DF119
:10639000C80E4FF0080C0B9872460DF1C40EA4F80D
:1063A0005C8C7146ADF8C4C0ADF8C88012F078F8C6
:1063B0000B98012111F0A0FC0A991AEE900AC4F87A
:1063C000501C0B990DF0A8FF68221D988723009799
:1063D000E221FEF79EFF4FF002004FF0FF3EDB4B45
:1063E000ADF8CC0032A8C4F890EC0146A4F8945C57
:1063F0001D98329311F041FE1D991AEE900A0DF08E
:106400008BFF1E9896223C21FEF776FF32A84FF0B4
:10641000080CA4F8D08C024631A8ADF8C4C00146DF
:106420001E98ADF8C88012F03BF80A991AEE900A4F
:10643000C4F8C41C1E990DF06FFF36221F988723E5
:106440000097E221FEF765FF4FF0FF304FF00101AA
:10645000BE4BC4F8040DA4F8085D1F98ADF8CC102D
:1064600032A9329311F009FE1F991AEE900A0DF02D
:1064700053FF2098C8223C21FEF73EFF32A94FF07F
:10648000080C20980A46A4F8448D31A9ADF8C4C080
:10649000ADF8C88012F004F80A991AEE900A40F29A
:1064A0003528C4F8381D20990DF036FFCC222198EC
:1064B000CA230097E221FEF72CFF4FF0FF31A34BD8
:1064C0002198C4F8781D32A9A4F87C5D3293ADF808
:1064D000CC6011F0D2FD21991AEE900A0DF01CFF4C
:1064E0001AEE901A18EE900A0EF0F2FC984AAA21C1
:1064F0004FF49E731EEE100AC4F88C2D00915122A9
:106500000B21FEF706FF1EEE100A84F8545E914937
:106510000FF07CFE2A4629462698CDF800804FF4DD
:106520009E73FEF7F6FE8C4B4FF010011EEE100A24
:10653000C4F8943E84F8921E26990EF0C3FF2A46B2
:1065400029462298CDF800804FF49E73FEF7E1FEB5
:1065500041F644334FF0FF314FF00F08E218A4F832
:10656000CC5EC4F8C81E32A9E552784BC4F8D42ECC
:1065700022983293ADF8CC8011F07FFD22991EEE67
:10658000100A0EF09FFF1EEE100A01210FF043FECD
:106590001EEE101A1BEE100A0DF0BEFEAA21782383
:1065A00051225846009140F26311FEF7B2FE29468F
:1065B00058460DF07FFB294658460DF021FA584603
:1065C00066490DF0E0FC494658460DF0DFFC4946AF
:1065D00058460DF0DEFC584664210DF022FA58466C
:1065E0003C210DF07BFB2A46294658460DF07FFBE7
:1065F0002A46294658460DF080FB2A465846242153
:106600000DF081FB2799249B58460A4600912C994E
:106610000DF097FB2A46394658460DF0AAFB59461D
:106620001BEE100A0A270DF077FE1B232F221EEE09
:10663000900A009340F263117823FEF76AFE41F25C
:1066400094634FF0FF311EEE900AE1501EEE901A57
:106650003E4B8D864FF010013293ADF8CC1032A92D
:1066600011F00BFD1EEE901A1BEE100A0DF054FEF9
:1066700019EE100A07220B21FEF73EFE2A46294694
:1066800019EE100A4FF4AF7300970CF0B0FB3A46C6
:106690003B46294619EE100A00950CF089FC0B23A5
:1066A00032A919EE100AADF8C8300CF029FD41F2FC
:1066B000E8732B4A2D9919EE100AE2500CF03EFBBC
:1066C000324619EE100A02210CF03BFB324619EE5D
:1066D000100A4FF4AF710CF016FB19EE100A0621E8
:1066E0000CF036FB19EE100A01210CF03CFB394688
:1066F00019EE100A0CF04DFB19EE101A1BEE100AE1
:106700000DF00AFE434632460C98F821CDF8008081
:10671000FEF7FFFD41F61403124A1BEE100A0C9916
:10672000E2500DF0F9FD32460D9810236C21CDF8A2
:106730000080FEF7EEFD04F5C2530B4A1BEE100A73
:106740000D991A600DF0E8FD1D230FE060CD0208E1
:10675000E0011001C5C5D1FF2B2B36FF8DBF01080D
:1067600000FF48FF303036FF2A2A2EFF0898062205
:10677000009340F26D116E23FEF7CBFD41F66903E5
:106780004FF0FF31D522E55441F674030898E150EB
:1067900041F67A0308998D8632A9E25441F6F473E2
:1067A000E218E55204F5C4531A60844B3293132364
:1067B000ADF8CC3011F061FC08991BEE100A0DF019
:1067C000ABFD18EE100A072240F26911FEF794FDA6
:1067D0002A46294618EE100A4B2300970CF007FBB7
:1067E0002B460322294618EE100A00950CF0E0FB18
:1067F0000C2332A918EE100AADF8C8300CF080FC5A
:1068000041F6CC136E4A299918EE100AE2500CF0AA
:1068100095FA3246294618EE100A0CF092FA3246E2
:1068200018EE100A46210CF06EFA18EE100A062136
:106830000CF08EFA18EE100A01210CF094FA18EE02
:10684000100A03210CF0A5FA18EE101A1BEE100A1C
:106850000DF062FD1BEE101A18EE900A0EF038FBD8
:1068600041F6D813574A29460998E2502A46FEF7BE
:1068700043FD32A90998ADF8C87011F0EBFF41F65D
:106880002423912209991BEE900AE2540DF044FD55
:106890001FEE100AD9228C21FEF72EFD41F6582357
:1068A0004FF0FF3232A91FEE100AE2501FEE102AFD
:1068B00012239586414DADF8CC30329511F0DDFBB9
:1068C0001FEE101A1BEE900A0DF026FD1FEE900A27
:1068D000B022B721FEF710FD4FF0FF3241F69423AE
:1068E00032A91FEE900A3295E2501FEE903AA3F8BB
:1068F00034A01123ADF8CC3011F0BFFB1FEE901A7D
:106900001BEE900A0DF008FD239870223F21FEF740
:10691000F3FC2D4A41F6D02332A92398E25004F526
:10692000D5533295A3F834A0ADF8CCA011F0A5FB57
:1069300023991BEE900A0DF0EFFC1BEE901A18EE57
:10694000900A0EF0C5FA314618EE900A0EF06AFA77
:10695000201D259908900DF0DFFC0F9908980DF087
:10696000DBFC18EE901A08980DF0D6FC02991AEE8E
:10697000100AFEF74BFA03991AEE100AFEF746FAD0
:1069800004991AEE100AFEF741FA05991AEE100A58
:10699000FEF73CFA06991AEE100AFEF737FA1AEEDD
:1069A000100A0799FEF732FA41F61C332B9A20465B
:1069B000E25035B0BDEC108BBDE8F08F60CD020821
:1069C0000000FFFFE0011001F7F7FCFF70B504467F
:1069D0000D460EF0D3F8D4F8F80060B10368DB6818
:1069E000984740B1D4F8F8002A4621460368BDE82C
:1069F00070409B68184770BD7047000030B5164D59
:106A00008DB02C78BFF35B8F14F0010420D12846A1
:106A100024F039FAE0B13F23022210490793104BCA
:106A200010480693104B0894059301230294CDE976
:106A300003330523CDE90944CDE900321423BE22F6
:106A4000FDF710FF284624F02AFA084824F066FAD9
:106A500004480DB030BD00BFB84F00208C740A90C0
:106A6000E01C0308BC4F002090DA0208F969000816
:106A70007047000030B5164D8DB02C78BFF35B8F9A
:106A800014F0010420D1284624F0FDF9E0B13F23A1
:106A9000022210490793104B10480693104B08949C
:106AA000059301230294CDE903330523CDE909447D
:106AB000CDE900321423BF22FDF7D4FE284624F08E
:106AC000EEF9084824F02AFA04480DB030BD00BFA2
:106AD000E44F0020F07E0A90E41C0308E84F0020F9
:106AE00094DA0208716A00087047000030B5164D4C
:106AF0008DB02C78BFF35B8F14F0010420D12846B1
:106B000024F0C1F9E0B13F23042210490793104B50
:106B100010480693104B089405930123CDE90333E5
:106B200002930523CDE90944CDE900321423BF22A5
:106B3000FDF798FE284624F0B2F9084824F0EEF953
:106B400004480DB030BD00BF1050002064890A9089
:106B50007C1F03081450002098DA0208E96A000834
:106B60007047000030B5154D8DB02C78BFF35B8FAA
:106B700014F001041FD1284624F085F9D8B13F2331
:106B800001220F4907930F4B0F4806930F4B0894B0
:106B900003940094CDE904430423CDE90944CDE9ED
:106BA00001320A230B22FDF75DFE284624F077F917
:106BB000074824F0B3F904480DB030BD3C50002024
:106BC000D8930A9014220308405000209CDA02084F
:106BD000616B00087047000030B5154D8DB02C7802
:106BE000BFF35B8F14F001041FD1284624F04BF94A
:106BF000D8B13F2336220F4907930F4B0F48069316
:106C00000F4B089405930123CDE90343029304231A
:106C1000CDE90944CDE900331423FDF723FE2846CE
:106C200024F03DF9074824F079F904480DB030BD4F
:106C30006850002074940A90182203086C500020B9
:106C4000A0DA0208D56B00087047000030B5164D79
:106C50008DB02C78BFF35B8F14F0010420D128464F
:106C600024F011F9E0B13F23042210490793104B9F
:106C700010480693104B089405930123CDE9034374
:106C800002930823CDE90944CDE9003228231722D5
:106C9000FDF7E8FD284624F002F9084824F03EF903
:106CA00004480DB030BD00BF9450002068970A9092
:106CB000B822030898500020A4DA0208496C0008A2
:106CC00000207047002070470EB403B503AB0021CD
:106CD00053F8042B019314F095FA02B05DF804EB1D
:106CE00003B070470CB407B504AB53F8042B019301
:106CF00014F088FA03B05DF804EB02B070470000AE
:106D0000C36B10B5044673B3038E2BB9184BBF2168
:106D1000184A194824F0E4F8C38D00EB43035B8B59
:106D20000BB315F04DFF238E012B03D8134BC42159
:106D3000134AEEE7E28D40F63F10531C9BB2092B3D
:106D4000194688BFA3F10A0104EB4101498B814236
:106D500009D10A2B04EB420228BF0023508B04EB1D
:106D60004303588351832046BDE8104015F00CBE04
:106D7000A8DA0208B1DA02085CDB0208A6DB020826
:106D8000B4DB020815F0BABD10B586B002AC84E8D9
:106D900006001A460AAB214605930193099B00930E
:106DA000089B12F07FFF06B010BD000038B518BB7D
:106DB000124B13481B681349B3B11A689C681A44F4
:106DC0001C4402605A681A440A600F4B00221A8061
:106DD00000F038F8054600F033F80C4B1C600C4B03
:106DE0001D600C4B188007E00B4B03600B4B0B60D6
:106DF0000B4B1C68002CE8D138BD00BFC0500020F0
:106E0000C4500020C8500020CC5000202055012044
:106E1000285501202455012020990A90AC980A9009
:106E2000989B0A90044B1B6853F82100034B1B6886
:106E300003EB4000704700BFC8500020C450002042
:106E40001D20704700487047D050002010B50A4CF4
:106E5000FFF7C2FE2060FFF7F9FE6060FFF782FED9
:106E6000A060FFF743FEE060FFF704FE2061FFF73C
:106E7000C5FD606110BD00BFD05000207047704755
:106E800010B50446A02123F0FCFF204610BD036886
:106E900070B504465B6B1546984723682046294623
:106EA0009B6BBDE8704018472DE9F341044600256F
:106EB000FEF710FA434B264629462622A56246F8DD
:106EC0002C3B304624F092F93046FEF703FA3E4B55
:106ED00004F158072622E362FF232946656584F8FA
:106EE0005230384624F082F93846FEF7F3F94FF66F
:106EF000FF73DFF808812946A4F884304FF47F033C
:106F00003046C4F88850C4F88C30304BA4F8905008
:106F1000A3652F4BC4F89450A360C4F88080FDF79C
:106F2000CDFC29463046FDF7CBFC242278213046A3
:106F3000FFF7ADFF274B16227821636511233846F2
:106F400084F852304FF4E023E365FFF7A0FF224BB3
:106F5000A4F88C5004F19805C4F888301F4B1B68C6
:106F60002BB91F4BAE211F4A1F4823F0B9FF1F4BFF
:106F70001B880C2B03D81E4BAF211A4AF4E71D4B7C
:106F80000C211868FFF74EFF1B4A034604212846D0
:106F900016F0CEFB0B2369463846C4F89450ADF882
:106FA0000430CDF8008011F068F8314620460DF02D
:106FB000B3F9204639460DF0AFF9204602B0BDE8DE
:106FC000F08100BF90DC02082000030838010308AC
:106FD000780024003C3C47FFACACB5FF20550120B5
:106FE000FBD202083DD302086BD3020824550120CE
:106FF000B2D302082C550120FAD5020860CD020850
:107000007047704710B50446BC2123F03AFF204674
:1070100010BD00002DE9F34104460025FEF75AF9A2
:10702000484B264629462622A56246F82C3B304688
:1070300024F0DCF83046FEF74DF9434B04F15807D5
:107040002622E362FF232946656584F852303846DC
:1070500024F0CCF83846FEF73DF94FF6FF73DFF821
:1070600018812946A4F884304FF47F033046C4F8D1
:107070008850C4F88C30354BA4F89050A365344B3D
:10708000C4F89450A36084F89850A4F89A50C4F8B7
:107090008080C4E92755C4E92955C4E92B55FDF77B
:1070A0000DFC29463046FDF70BFC242278213046A2
:1070B000FFF7EDFE274B1622782163651D23384626
:1070C00084F852304FF4E023E365FFF7E0FE4FF021
:1070D000FF33A4F88C5004F1B405C4F888301E4B7B
:1070E0001B682BB91D4BAE211D4A1E4823F0F8FE2C
:1070F0001D4B1B880E2B03D81C4BAF21184AF4E7FD
:107100001B4B0E211868FFF78DFE1A4A0346042117
:10711000284616F00DFB0D2369463846C4F89450F6
:10712000ADF80430CDF8008010F0A7FF31462046BE
:107130000DF0F2F8204639460DF0EEF8204602B088
:10714000BDE8F0811CDD02082000030808D6020813
:107150007800240014141CFF20550120FBD20208E3
:107160003DD302086BD3020824550120B2D3020894
:107170002C550120FAD5020860CD0208704710B5E1
:1071800004464FF4AC7123F07CFE204610BD10B5D0
:107190000446D0F8540100F0CFF82046BDE8104076
:1071A00013F0D4B810B50446FDF736FA014B20466B
:1071B000236010BDA8DD0208002307B505481A4664
:1071C000ADF806100DF10601006809F059FE03B094
:1071D0005DF804FB545A0120002307B505481A4600
:1071E000ADF806100DF10601006809F049FE03B084
:1071F0005DF804FBF0590120002307B505481A4645
:10720000ADF806100DF10601006809F039FE03B073
:107210005DF804FBE0580120002307B505481A4635
:10722000ADF806100DF10601006809F029FE03B063
:107230005DF804FBE0590120002307B504481A4615
:10724000019101A9006809F01BFE03B05DF804FB81
:10725000E8590120002307B504481A46019101A905
:10726000006809F00DFE03B05DF804FBDC58012056
:10727000002307B504481A46019101A9006809F0E6
:10728000FFFD03B05DF804FBA05A0120002307B501
:1072900004481A46019101A9006809F0F1FD03B004
:1072A0005DF804FB50580120002307B505481A4635
:1072B000ADF806100DF10601006809F0E1FD03B01C
:1072C0005DF804FB28580120002307B505481A463D
:1072D000ADF806100DF10601006809F0D1FD03B00C
:1072E0005DF804FBD8580120002307B505481A466D
:1072F000ADF806100DF10601006809F0C1FD03B0FC
:107300005DF804FB585A0120002307B505481A46CA
:10731000ADF806100DF10601006809F0B1FD03B0EB
:107320005DF804FB3C5B0120024A026000224260DF
:10733000704700BFECDD02081FB5214B0022044658
:107340000DF1030118688DF8032009F0D5FF01281D
:1073500006D1606820B103689DF803109B689847C8
:10736000184B002201A91868019209F0C5FF0128F5
:1073700005D1606818B103680199DB689847124B22
:10738000002202A91868029209F0B6FF012805D16F
:10739000606818B1036802991B6998470B4B00227B
:1073A00003A91868039209F0A7FF012805D16068B6
:1073B00018B1036803995B69984704B010BD00BF1A
:1073C000D8590120A45A0120E4590120D4570120A2
:1073D000704704387047704707B5C068019101A92C
:1073E0000368D3F88030984703B05DF804FBA0F140
:1073F0000400FFF7F1BF07B5C0688DF807100DF165
:10740000070103689B6F984703B05DF804FBA0F188
:107410000400FFF7F0BFC0680368DB6F1847A0F1F6
:107420000400FFF7F8BFC0680368D3F8843018473A
:10743000A0F10400FFF7F7BF10B50446102123F0B8
:1074400020FD204610BDA0F10400F5E70022C16038
:107450008260044A10B502F10804303204604260D0
:1074600010BD00BF1CDE020800F571532C33C0F8BC
:1074700090317047704700009830884202BF024B3D
:1074800000221A60704700BF30040020704770B4BB
:1074900045680346C4689B68661005EB6400E40712
:1074A00044BFAC59E35870BC184743682BB183689C
:1074B0002BB9C06800F001007047184670470120E2
:1074C000704710B50446102123F0DBFC204610BDA8
:1074D00038B50C4D04460A460B49284624F0E4FA18
:1074E0002846F8F795FE294682B204F5FF5014307D
:1074F00015F0B9FD04F5C250BDE83840043013F072
:10750000A3BF00BF4053002064DE020838B5044624
:107510000D6800F5B55004F5C4540A2D04F10404B7
:1075200008DC29460BF035FC00212046BDE8384038
:107530000BF02FBC0A210BF02CFCA5F10A01F4E79B
:1075400010460A230422983115F0BCBD08B5034A41
:107550008721034B034823F0C3FC00BFA3DE0208CE
:1075600067DE0208D6DE02080368DB6A1847C36BD1
:1075700005219868FFF7F8BFC36B04219868FFF7EF
:10758000F3BFC36B03219868FFF7EEBFC36B002105
:107590009868FFF7E9BF10B504460A231046B431D6
:1075A000042215F08FFD04F6F4600CF06DF9E36B26
:1075B00081B29B681A6818461268BDE810401047EF
:1075C00003685B6918470000C36B37B50D46044676
:1075D00089B29868FFF7F4FF2A460A4901A824F007
:1075E00063FA01A8F8F714FE01A982B204F5D95094
:1075F0000C3015F038FD04F6CC1013F025FF03B065
:1076000030BD00BF1ADF020803689B6918470000FD
:1076100030B5044685B000F2D4700021234D0190AE
:107620000CF0B9FF019813F00FFF04F50D60002175
:1076300001900CF0B0FF019813F006FFE36B0021FE
:107640009868FFF7BDFF2946002202A824F02CFA13
:1076500002A8F8F7DDFD02A982B204F5D9500C307A
:1076600015F001FD04F6CC1013F0EEFEE36B0021E3
:107670009868FFF7C9FF2946002203A824F014FAEE
:1076800003A8F8F7C5FD03A982B204F5D950143058
:1076900015F0E9FC04F60C2013F0D6FEE36B022192
:1076A0009868FFF761FF05B030BD00BF1ADF020820
:1076B00030B5044685B000F2D4706421234D0190AA
:1076C0000CF069FF019813F0BFFE04F50D60642112
:1076D00001900CF060FF019813F0B6FEE36B64219B
:1076E0009868FFF76DFF2946642202A824F0DCF9B0
:1076F00002A8F8F78DFD02A982B204F5D9500C302A
:1077000015F0B1FC04F6CC1013F09EFEE36B64217F
:107710009868FFF779FF2946642203A824F0C4F98A
:1077200003A8F8F775FD03A982B204F5D950143007
:1077300015F099FC04F60C2013F086FEE36B012192
:107740009868FFF711FF05B030BD00BF1ADF0208CF
:10775000C36B37B50D46044689B29868FFF754FFEE
:107760002A460A4901A824F09FF901A8F8F750FD1C
:1077700001A982B204F5D950143015F074FC04F656
:107780000C2013F061FE03B030BD00BF1ADF020809
:10779000C36B37B5044698680D4689B20368DB6948
:1077A00098472A460D4901A824F07EF901A8F8F768
:1077B0002FFD01A982B204F5D950043015F053FC15
:1077C0001E2D074B04F5D36018BF4FF0FF33C4F8EC
:1077D000C83613F039FE03B030BD00BF64DE0208C6
:1077E0002DF705FFC36B37B5044698680D4689B27F
:1077F00003681B6A98472A460D4901A824F054F9EA
:1078000001A8F8F705FD01A982B204F5D9501C3092
:1078100015F029FC322D074B04F6483018BF4FF005
:10782000FF33C4F8783B13F00FFE03B030BD00BF48
:1078300064DE02082DF705FFC26B0346906893F8DB
:1078400018120268926A01B1012110472DE9F04136
:10785000044629480E46F8F7DBFC04F5DA55B0F586
:10786000967FDFF8948005F104051DD104F5EC53F3
:1078700041462A4600271C3301F8017B22F8027B8F
:107880009A42F9D11C48F8F7C3FC1B4982B228463A
:1078900015F0E9FB04F69860A4F89E7E13F0D4FD81
:1078A0004FF0000388F8003001223146124824F0DE
:1078B0005EF91148F8F7ACFC0F4982B2284615F082
:1078C000D2FB04F698650123284684F8D13E13F0D4
:1078D000BBFD2846FDF728FB95280BDD2846FDF764
:1078E00023FBC0F19600A4F89E0E2846BDE8F041A7
:1078F00013F0AABDBDE8F081E850002008B5054BA3
:107900001B680BB9FFF722FE828EC08D131A5842F6
:10791000584108BD5855012010B5044600F52A709D
:10792000FFF7ECFFE36B81B29B681A681846526A56
:10793000BDE81040104710B5044600F6B430FFF71C
:10794000DDFF0146E36B98680268BDE810405268AD
:10795000104710B5044600F62840FFF7CFFF014658
:10796000E36B98680268BDE810409268104710B554
:10797000044600F69C40FFF7C1FF0146E36B9868A0
:107980000268BDE810401269104710B5044600F5C2
:107990005160FFF7B3FF0146E36B98680268BDE8EA
:1079A0001040D26810470000034B10B50446036036
:1079B000FDF7A8F9204610BD40DF020810B50446C7
:1079C000FFF7F2FF43F67C41204623F05AFA2046A7
:1079D00010BD000010B50446FDF7B2FD084B094983
:1079E0002046236043F66C43E218E15043F67443AB
:1079F0005460054AE25043F678430022E25010BD3D
:107A000040DF020828DF02087974000837B5044611
:107A1000FDF727FA524B04F2D470524D19880190A9
:107A20000CF0B9FD019813F00FFD4F4B04F50D60FC
:107A3000198801900CF0AFFD019813F005FD4B4B38
:107A400004F5DB60198801900CF0A5FD019813F096
:107A5000FBFC474B04F69C401978019010F04CF960
:107A6000019813F0F1FC434B04F6B43019780190FF
:107A700010F042F9019813F0E7FC3F4B04F6284060
:107A80001978019010F038F9019813F0DDFC3B4BA8
:107A900004F551601978019010F02EF9019813F057
:107AA000D3FC374B04F6F4604FF0FF32B3F900100B
:107AB00001900CF05EF9019813F0C6FC314B04F60E
:107AC0004C20198801900CF066FD019813F0BCFC65
:107AD0002D4B04F52A701978019010F00DF90198DA
:107AE00013F0B2FC2B8833B904F5D65004F581614C
:107AF0001C30FDF787F82B88012B06D104F5D650F2
:107B000004F562711C30FDF77DF82B88022B06D13D
:107B100004F5D65004F572711C30FDF773F82B880C
:107B2000032B06D104F5D65004F591611C30FDF706
:107B300069F82B88042B06D104F5D65004F5527150
:107B40001C30FDF75FF82B88052B06D104F5D650C5
:107B500004F589611C30FDF755F803B030BD00BF56
:107B60001600002012000020180000200E00002047
:107B700008000020640100200D00002063010020A7
:107B80000A000020100000200C0000207047FFF7C2
:107B900076B910B50446A02123F073F9204610BD34
:107BA00010B50446FFF780F9014B2046236010BD55
:107BB000D0DF02087047FFF724BA10B50446BC2195
:107BC00023F05FF9204610BD10B50446FFF722FAF6
:107BD000014B2046236010BD5CE0020880B582B0F6
:107BE00000AF284B284A1A60264803F04DFA034696
:107BF000002B01D0012341E00021224800F078F859
:107C0000204B01225A601F4B04229A601D4B102208
:107C1000DA604FF080737B607B6893FAA3F33B607C
:107C20003B68B3FA83F3DBB2013B1A46154B1A618A
:107C3000144B4FF4A0625A61124B00229A61114B0F
:107C40000022DA610F4B00221A620E4803F0A0F9FD
:107C50000346002B01D0012310E00A4800F008F988
:107C60000346002B01D0042308E0064800F042F947
:107C70000346002B01D0042300E0002318460837F8
:107C8000BD4680BD44600120001000A080B590B0CA
:107C900000AF4FF480733B62EB23BB604FF4406353
:107CA0007B624FF400537B610023BB624FF0407353
:107CB000FB620A23FB6100237B630023BB63002379
:107CC000FB6300237B6000233B603A4607F1080317
:107CD0001946064803F00AFC0346002B01D0012395
:107CE00000E0002318464037BD4680BD44600120B7
:107CF00080B58EB000AF78603960594B9B6B584AA5
:107D000043F002039363564B9B6B03F002033B6209
:107D10003B6A534B9B69524A43F002039361504BB9
:107D20009B694F4A23F0020393614D4B1B6B4C4AF6
:107D300043F0020313634A4B1B6B03F00203FB6126
:107D4000FB69474B1B6B464A43F002031363444BEA
:107D50001B6B03F00203BB61BB69414B1B6B404AC9
:107D600043F0080313633E4B1B6B03F008037B6176
:107D70007B693B4B1B6B3A4A43F008031363384B58
:107D80001B6B03F008033B613B69354B1B6B344AAB
:107D900043F010031363324B1B6B03F01003FB60C3
:107DA000FB682F4B1B6B2E4A43F0080313632C4BCD
:107DB0001B6B03F00803BB60BB6840237B6202239C
:107DC000BB620123FB6203233B630A237B6307F14E
:107DD00024031946234801F067FC04237B62002337
:107DE000FB6209237B6307F1240319461D4801F058
:107DF0005BFC4FF400637B6209237B6307F1240380
:107E00001946194801F050FC4FF480537B62092356
:107E10007B6307F124031946134801F045FC042352
:107E20007B6209237B6307F1240319460F4801F0A5
:107E30003BFC4FF400537B6209237B6307F124036F
:107E40001946094801F030FC00220F215C2000F0A7
:107E50008BFC5C2000F0A4FC00BF3837BD4680BD21
:107E60000038024000040240000C024000100240B2
:107E700080B590B000AF78604FF480733B626623AA
:107E8000BB6000237B620023BB620023FB620023F4
:107E9000FB6100237B630023BB630023FB6307F1CB
:107EA000080341F288321946786803F011F9034655
:107EB000002B01D0012319E09923BB6007F10803CF
:107EC00041F288321946786803F002F90346002B24
:107ED00001D001230AE041F28831786800F0C7F848
:107EE0000346002B01D0012300E000231846403751
:107EF000BD4680BD80B594B000AF78604FF480730C
:107F0000BB6285233B610023FB6200233B634FF090
:107F100080737B6300237B620123BB630023FB63CD
:107F200000233B6400237B6407F1100341F2883295
:107F30001946786803F0CCF80346002B01D00123E2
:107F400048E007F10F0341F288321946786803F0E0
:107F5000B4F90346002B01D001233BE0786800F020
:107F60003DF80346002B01D0012333E081233B6120
:107F7000FB7B5BB203F00F035AB2F023FB64FB6C94
:107F800093FAA3F3BB64BB6CB3FA83F3DBB2194679
:107F90000A238B405BB213435BB2DBB2FB7307F186
:107FA000100341F288321946786803F091F80346CD
:107FB000002B01D001230DE007F10F0341F28832BD
:107FC0001946786803F0E2F80346002B01D001233C
:107FD00000E0002318465037BD4680BD80B596B0FE
:107FE00000AF78604FF48073BB6306233B620023CD
:107FF000FB6300233B6400237B6400237B6300233B
:10800000FB6400233B6500237B6507F1200341F2FD
:1080100088321946786803F05BF80346002B01D0DC
:10802000012320E00223BB600223FB600023BB612D
:1080300001237B6110233B614FF48003FB61052327
:108040003B624FF080737B6407F1080207F1200167
:1080500041F28833786803F0D2F90346002B01D04F
:10806000012300E0002318465837BD4680BD80B587
:1080700096B000AF786039604FF48073BB6305231E
:108080003B620023FB6300233B644FF080737B64FF
:1080900000237B630023FB6400233B6500237B6597
:1080A0000023BB600123FB600023BB6101237B61D4
:1080B00010233B614FF48003FB6107F1080207F1D5
:1080C00020013B68786803F09AF90346002B01D041
:1080D000012300E0002318465837BD4680BD00004C
:1080E00080B400AF154BD3F88830144A43F47003C2
:1080F000C2F88830124B1B68114A43F00103136029
:108100000F4B00229A600E4B1A680D490D4B13401D
:108110000B600B4B0C4A5A60094B1B68084A23F44E
:1081200080231360064B0022DA60044B4FF000629C
:108130009A6000BFBD465DF8047B704700ED00E02B
:1081400000380240FFFFF6FE1030002480B582B0F8
:1081500000AF0346FB8000F0B5F900BF0837BD460D
:1081600080BD80B483B000AF0346FB8000BF0C37F6
:10817000BD465DF8047B704780B584B000AF034610
:10818000FB8000237B730023FB730023BB7300F091
:1081900099F90023FB7310E0FB88DBB2A821184695
:1081A000FBF704FC03467B737B7BDBB2512B01D1D5
:1081B0000123BB73FB7B0133FB73FB7B022B02D8D8
:1081C000BB7B002BE8D07B7BDBB29BB21846103721
:1081D000BD4680BD80B582B000AF0346FB80FB8802
:1081E000184600F07DF9FB88184600F033F900BF0F
:1081F0000837BD4680BD000080B584B000AF03469F
:10820000FB800023FB73FB88DBB202211846FBF7DF
:10821000CDFB0346FB73FB7BDBB203F00F03DBB24A
:10822000FB73FB7BDBB2052B01D90023FB73FB7BCC
:10823000DAB2054B5A70044B00229A70FB7BDBB21A
:1082400018461037BD4680BD4453002080B586B027
:1082500000AF0346B9607A60FB810023FB74002302
:10826000FB750023BB7500237B7500233B756D4BAD
:108270009A786C4B5B789A4280F0CF80694B9B7800
:10828000092B71D801A252F823F000BFB582000873
:10829000C7820008D9820008EB820008FD8200082E
:1082A0000F830008218300083383000845830008FA
:1082B000578300080423FB750323BB7506237B75D6
:1082C00005233B7551E00A23FB750923BB750C237D
:1082D0007B750B233B7548E01023FB750F23BB75A3
:1082E00012237B7511233B753FE01623FB75152385
:1082F000BB7518237B7517233B7536E01C23FB7574
:108300001B23BB751E237B751D233B752DE022238C
:10831000FB752123BB7524237B7523233B7524E048
:108320002823FB752723BB752A237B7529233B75DF
:108330001BE02E23FB752D23BB7530237B752F236C
:108340003B7512E03423FB753323BB7536237B75F5
:1083500035233B7509E03A23FB753923BB753C2374
:108360007B753B233B7500E000BFFB89DBB2FA7DE8
:1083700011461846FBF71AFB0346FB74FB7CDBB285
:108380009AB2294B1A80FB89DBB2BA7D1146184696
:10839000FBF70CFB0346FB74FB7CDBB21B0203F414
:1083A00070631AB2204B1B881BB213431BB29AB2E4
:1083B0001D4B1A801C4B1A88BB681A80FB89DBB2E4
:1083C0007A7D11461846FBF7F1FA0346FB74FB7CF5
:1083D000DBB29AB2144B1A80FB89DBB23A7D1146AC
:1083E0001846FBF7E3FA0346FB74FB7CDBB21B0287
:1083F00003F470631AB20C4B1B881BB213431BB2FD
:108400009AB2094B1A80084B1A887B681A80054B70
:108410009B780133DAB2034B9A7000BF1837BD4620
:1084200080BD00BF445300204853002080B584B075
:1084300000AF0346FB800023FB730123FB73FB8823
:10844000DBB2FA7BA4211846FBF796FA00BF10377F
:10845000BD4680BD80B584B000AF0346FB800023DD
:10846000FB730023FB73FB88DBB2FA7BA421184665
:10847000FBF782FA00BF1037BD4680BD80B483B0E1
:1084800000AF0346FB80002318460C37BD465DF85D
:10849000047B704780B483B000AF0346FB8000BF0D
:1084A0000C37BD465DF8047B7047000080B400AF18
:1084B000034B1B781846BD465DF8047B704700BF30
:1084C0004453002080B500AFFFF7F0FF0346002BB8
:1084D00002D1024B01221A7000BF80BD445300201C
:1084E00080B485B000AF0346FB800023FB60FB68CF
:1084F00018461437BD465DF8047B704780B500AF61
:10850000084B1B68074A43F480731360032000F094
:1085100020F90020FAF78EFDFAF7AEF8002318468E
:1085200080BD00BF003C024080B400AF064B1B780A
:108530001A46064B1B681344044A136000BFBD462D
:108540005DF8047B704700BF54000020906001205C
:1085500080B400AF034B1B681846BD465DF8047B32
:10856000704700BF9060012080B584B000AF786094
:10857000FFF7EEFFB8607B68FB60FB68B3F1FF3F7D
:1085800005D00A4B1B781A46FB681344FB6000BFFA
:10859000FFF7DEFF0246BB68D31AFA689A42F7D8A3
:1085A00000BF00BF1037BD4680BD00BF5400002093
:1085B00080B485B000AF78607B6803F00703FB6090
:1085C0000B4BDB68BB60BA684FF6FF031340BB6020
:1085D000FB681A02BB681A43064B1343BB60044A8C
:1085E000BB68D36000BF1437BD465DF8047B70479D
:1085F00000ED00E00000FA0580B400AF044BDB683A
:108600001B0A03F007031846BD465DF8047B70475C
:1086100000ED00E080B483B000AF0346FB7197F932
:108620000730002B0BDBFB7903F01F02074997F99A
:1086300007305B09012000FA02F241F8232000BF55
:108640000C37BD465DF8047B704700BF00E100E0D9
:1086500080B483B000AF0346FB7197F90730002B5D
:1086600012DBFB7903F01F020A4997F907305B0917
:10867000012000FA02F2203341F82320BFF34F8F8C
:1086800000BFBFF36F8F00BF00BF0C37BD465DF862
:10869000047B704700E100E080B483B000AF034684
:1086A0003960FB7197F90730002B0ADB3B68DAB2BF
:1086B0000C4997F907301201D2B20B4483F800231A
:1086C0000AE03B68DAB20849FB7903F00F03043B88
:1086D0001201D2B20B441A7600BF0C37BD465DF8CA
:1086E000047B704700E100E000ED00E080B489B059
:1086F00000AFF860B9607A60FB6803F00703FB61C4
:10870000FB69C3F10703042B28BF0423BB61FB698A
:108710000433062B02D9FB69033B00E000237B6195
:108720004FF0FF32BB6902FA03F3DA43BB681A4029
:108730007B699A404FF0FF317B6901FA03F3D9431B
:108740007B680B40134318462437BD465DF8047B15
:10875000704780B582B000AF78607868FFF728FF77
:1087600000BF0837BD4680BD80B586B000AF034668
:10877000B9607A60FB7300237B61FFF73DFF78618E
:108780007A68B9687869FFF7B1FF024697F90F3048
:1087900011461846FFF780FF00BF1837BD4680BD61
:1087A00080B582B000AF0346FB7197F907301846D9
:1087B000FFF730FF00BF0837BD4680BD80B582B0EF
:1087C00000AF0346FB7197F907301846FFF740FFEB
:1087D00000BF0837BD4680BD80B400AFBFF35F8FD8
:1087E00000BF074B5B6A064A23F480335362054B94
:1087F00000225A6000BFBD465DF8047B704700BF91
:1088000000ED00E090ED00E080B483B000AF786050
:108810000B4A7B6843F0010353600A4B5B6A094AC9
:1088200043F480335362BFF34F8F00BFBFF36F8FAA
:1088300000BF00BF0C37BD465DF8047B704700BF2A
:1088400090ED00E000ED00E080B483B000AF786010
:108850007B685A781D4B9A607B681B78002B29D067
:108860001A4A7B685B68D3607B681B7B1A077B684E
:10887000DB7A1B061A437B689B7ADB041A437B680E
:108880005B7B9B041A437B689B7B5B041A437B687E
:10889000DB7B1B041A437B685B7A1B021A437B68F1
:1088A0001B7A5B0013437A6812781146074A0B4320
:1088B000136105E0054B0022DA60044B00221A61C7
:1088C00000BF0C37BD465DF8047B704790ED00E0BB
:1088D00080B582B000AF78607B68002B01D10123A6
:1088E00054E07B685B7FDBB2002B05D17B68002204
:1088F0001A777868F9F7E8FE7B6802225A777B6876
:108900001B79002B0CD17B681B68224A5A617B685B
:108910001B689A687B681B6822F018029A600CE05A
:108920007B6899687B68DB681A46786800F034F8E1
:108930000346002B01D0012328E07B685B79002BE4
:1089400005D17B681B684FF0FF321A6104E07B6839
:108950001B687A6812691A617B681B689B6823F040
:1089600060017B685A697B681B680A439A607B6870
:108970001B689B6823F080017B689A697B681B6891
:108980000A439A607B6801225A7700231846083709
:10899000BD4680BDB71DC10480B487B000AFF8608C
:1089A000B9607A600023FB751F233B6100BF3B6900
:1089B0005A1E3A61002B09D03B6903F01F03BA68C5
:1089C00022FA03F303F00103002BF0D07B68182B8D
:1089D00046D801A252F823F0678A0008618A00088D
:1089E000618A0008618A0008618A0008618A0008BB
:1089F000618A0008618A0008558A0008618A0008B7
:108A0000618A0008618A0008618A0008618A00089A
:108A1000618A0008618A0008498A0008618A0008A2
:108A2000618A0008618A0008618A0008618A00087A
:108A3000618A0008618A00083D8A00083B69062BAC
:108A400013D90123FB7510E03B69072B0FD90123D4
:108A5000FB750CE03B690F2B0BD90123FB7508E07C
:108A60000123FB7506E000BF04E000BF02E000BF89
:108A700000E000BFFB7D002B0DD1FB681B68BA68CE
:108A80005A61FB681B689B6823F01801FB681B6830
:108A90007A680A439A60FB7D18461C37BD465DF82C
:108AA000047B704780B586B000AF786000237B619F
:108AB000FFF74EFD38617B68002B01D1012399E05F
:108AC0007B68002283F834207B68022283F83520FB
:108AD0007B681B681A687B681B6822F001021A60B9
:108AE0000FE0FFF735FD02463B69D31A052B08D985
:108AF0007B6820225A657B68032283F83520032394
:108B000078E07B681B681B6803F00103002BE8D149
:108B10007B681B681B687B617A69384B13407B61FB
:108B20007B685A687B689B681A437B68DB681A43DA
:108B30007B681B691A437B685B691A437B689B6986
:108B40001A437B68DB691A437B681B6A13437A69A3
:108B500013437B617B685B6A042B07D17B68DA6A0D
:108B60007B681B6B13437A6913437B617B681B68CB
:108B70007A691A607B681B685B697B617B6923F09B
:108B800007037B617B685B6A7A6913437B617B685F
:108B90005B6A042B17D17B689B6A7A6913437B61FC
:108BA0007B68DB6A002B0ED0786800F015FB03466B
:108BB000002B08D07B6840225A657B68012283F82D
:108BC0003520012316E07B681B687A695A61786852
:108BD00000F0CCFA0346FB607B68DB6D3F229A40D5
:108BE000FB689A607B6800225A657B68012283F8E3
:108BF0003520002318461837BD4680BD3F8010F051
:108C000080B586B000AFF860B9607A603B60002341
:108C1000FB75FB689B6D3B61FB6893F83430012B5F
:108C200001D1022348E0FB68012283F83420FB686D
:108C300093F83530DBB2012B37D1FB68022283F881
:108C40003520FB6800225A653B687A68B968F86885
:108C500000F05EFAFB68DB6D3F229A403B699A6048
:108C6000FB681B681A68FB681B6842F016021A60F2
:108C7000FB681B685A69FB681B6842F080025A61F6
:108C8000FB681B6C002B07D0FB681B681A68FB682D
:108C90001B6842F008021A60FB681B681A68FB68D0
:108CA0001B6842F001021A6005E0FB68002283F8AD
:108CB00034200223FB75FB7D18461837BD4680BD66
:108CC00080B584B000AF78607B689B6DFB60FFF778
:108CD0003FFCB8607B6893F83530DBB2022B08D0DC
:108CE0007B6880225A657B68002283F83420012348
:108CF00052E07B681B681A687B681B6822F01602CA
:108D00001A607B681B685A697B681B6822F08002C6
:108D10005A617B681B6C002B03D17B689B6C002B1A
:108D200007D07B681B681A687B681B6822F0080202
:108D30001A607B681B681A687B681B6822F0010256
:108D40001A6013E0FFF704FC0246BB68D31A052B38
:108D50000CD97B6820225A657B68002283F8342076
:108D60007B68032283F83520032315E07B681B68AA
:108D70001B6803F00103002BE4D17B68DB6D3F220D
:108D80009A40FB689A607B68002283F834207B68F5
:108D9000012283F83520002318461037BD4680BDD8
:108DA00080B483B000AF78607B6893F83530DBB275
:108DB000022B04D07B6880225A6501230CE07B687B
:108DC000052283F835207B681B681A687B681B685E
:108DD00022F001021A60002318460C37BD465DF8E8
:108DE000047B704780B586B000AF78600023BB601D
:108DF000924B1B68924AA2FB03239B0A7B617B6810
:108E00009B6D3B613B691B68FB607B68DB6D0822E7
:108E10009A40FB681340002B1AD07B681B681B68C4
:108E200003F00403002B13D07B681B681A687B686F
:108E30001B6822F004021A607B68DB6D08229A40EE
:108E40003B699A607B685B6D43F001027B685A6501
:108E50007B68DB6D01229A40FB681340002B12D027
:108E60007B681B685B6903F08003002B0BD07B6879
:108E7000DB6D01229A403B699A607B685B6D43F031
:108E800002027B685A657B68DB6D04229A40FB68AE
:108E90001340002B12D07B681B681B6803F0020391
:108EA000002B0BD07B68DB6D04229A403B699A60F3
:108EB0007B685B6D43F004027B685A657B68DB6D01
:108EC00010229A40FB681340002B43D07B681B683C
:108ED0001B6803F00803002B3CD07B68DB6D10227D
:108EE0009A403B699A607B681B681B6803F4802387
:108EF000002B18D07B681B681B6803F40023002B31
:108F000008D17B681B6C002B24D07B681B6C7868B5
:108F100098471FE07B689B6C002B1BD07B689B6C89
:108F20007868984716E07B681B681B6803F48073B9
:108F3000002B07D17B681B681A687B681B6822F0CE
:108F400008021A607B681B6C002B03D07B681B6CCB
:108F5000786898477B68DB6D20229A40FB68134055
:108F6000002B00F08E807B681B681B6803F01003E9
:108F7000002B00F086807B68DB6D20229A403B69E5
:108F80009A607B6893F83530DBB2052B36D17B686D
:108F90001B681A687B681B6822F016021A607B68DF
:108FA0001B685A697B681B6822F080025A617B68E3
:108FB0001B6C002B03D17B689B6C002B07D07B685C
:108FC0001B681A687B681B6822F008021A607B68BD
:108FD000DB6D3F229A403B699A607B68002283F8F0
:108FE00034207B68012283F835207B681B6D002BC1
:108FF0007DD07B681B6D7868984778E07B681B683C
:109000001B6803F48023002B1CD07B681B681B6843
:1090100003F40023002B08D17B685B6C002B30D05D
:109020007B685B6C786898472BE07B68DB6B002B78
:1090300027D07B68DB6B7868984722E0240000200B
:10904000B5814E1B7B681B681B6803F48073002B83
:109050000FD17B681B681A687B681B6822F01002BE
:109060001A607B68002283F834207B68012283F831
:1090700035207B68DB6B002B03D07B68DB6B78686B
:1090800098477B685B6D002B32D07B685B6D03F08B
:109090000103002B22D07B68052283F835207B68F2
:1090A0001B681A687B681B6822F001021A60BB68A3
:1090B0000133BB607A699A4207D37B681B681B68DF
:1090C00003F00103002BF2D100E000BF7B68002217
:1090D00083F834207B68012283F835207B68DB6CC1
:1090E000002B05D07B68DB6C7868984700E000BFF8
:1090F0001837BD4680BD00BF80B483B000AF786034
:109100007B685B6D18460C37BD465DF8047B704785
:1091100080B485B000AFF860B9607A603B60FB68EE
:109120001B681A68FB681B6822F480221A60FB68BF
:109130001B683A685A60FB689B68402B08D1FB6843
:109140001B687A689A60FB681B68BA68DA6007E097
:10915000FB681B68BA689A60FB681B687A68DA600B
:1091600000BF1437BD465DF8047B704780B485B0FE
:1091700000AF78607B681B68DBB2103B134AA2FB30
:1091800003231B09FB60124AFB6813441B781A4631
:109190007B68DA65FB68032B08D97B681B681A4675
:1091A0000C4B13401A1D7B689A6506E07B681B68B0
:1091B0001A46084B13407A6893657B689B6D184686
:1091C0001437BD465DF8047B704700BFABAAAAAA5E
:1091D000F8E0020800FCFFFF80B485B000AF7860C3
:1091E0000023FB737B689B6ABB607B689B69002BD9
:1091F0001FD1BB68032B56D801A252F823F000BF41
:10920000119200082392000811920008A79200080A
:109210007B68DB6A03F08073002B46D00123FB736D
:1092200043E07B68DB6AB3F1C07F40D10123FB736D
:109230003DE07B689B69B3F5005F21D1BB68032BE0
:1092400037D801A252F823F0599200085F92000823
:1092500059920008719200080123FB7330E07B688B
:10926000DB6A03F08073002B25D00123FB7322E01F
:109270007B68DB6AB3F1C07F1FD10123FB731CE065
:10928000BB68022B03D9BB68032B03D018E0012372
:10929000FB7315E07B68DB6A03F08073002B0ED054
:1092A0000123FB730BE000BF0AE000BF08E000BF32
:1092B00006E000BF04E000BF02E000BF00E000BF26
:1092C000FB7B18461437BD465DF8047B704700BF32
:1092D00080B582B000AF78607B68002B01D101239C
:1092E00039E07B6893F83930DBB2002B06D17B681C
:1092F000002283F838207868F9F706FA7B680222A2
:1093000083F839207B681B681B6823F440317B6835
:109310005A687B681B680A431A607B681B685B6B32
:1093200023F007017B689A687B681B680A435A63CD
:109330007B681B681A6C0A4B13407A68D1687A689C
:1093400012680B4313647B680022DA637B68012296
:1093500083F83920002318460837BD4680BD00BF7A
:1093600000C0FFFF80B584B000AF78607B681B68E9
:109370005B68FB607B681B681B68BB60FB6803F075
:109380000103002B26D0BB6803F48073002B21D08F
:109390007B681B681A687B681B6822F480721A60FD
:1093A0007B68DB6B43F001027B68DA637B681B68D8
:1093B00001229A607B68042283F839207B680022AE
:1093C00083F838207B685B69002B03D07B685B697E
:1093D00078689847FB6803F02003002B26D0BB6811
:1093E00003F40053002B21D07B681B681A687B684C
:1093F0001B6822F400521A607B681B6820229A6066
:109400007B68DB6B43F002027B68DA637B680422D3
:1094100083F839207B68002283F838207B685B69F9
:10942000002B03D07B685B6978689847FB6803F082
:109430000803002B26D0BB6803F40063002B21D067
:109440007B681B681A687B681B6822F400621A60DC
:109450007B681B6808229A607B68DB6B43F0040220
:109460007B68DA637B68042283F839207B680022FA
:1094700083F838207B685B69002B03D07B685B69CD
:1094800078689847FB6803F00403002B13D0BB688F
:1094900003F48063002B0ED07B681B681A687B681E
:1094A0001B6822F480621A607B681B6804229A6041
:1094B000786800F053F8FB6803F00203002B24D017
:1094C000BB6803F40073002B1FD07B681B681A680D
:1094D0007B681B6822F400721A607B681B6802229A
:1094E0009A607B68DA6B7B68DA637B68012283F8B9
:1094F00039207B68002283F838207B681B69002BA9
:1095000003D07B681B6978689847FB6803F01003F9
:10951000002B1FD0BB6803F48053002B1AD07B684C
:109520001B681A687B681B6822F480521A607B688B
:109530001B6810229A607B68DA6B7B68DA637B6851
:10954000012283F839207B68002283F8382078686C
:1095500000F00EF800BF1037BD4680BD80B483B068
:1095600000AF786000BF0C37BD465DF8047B7047E4
:1095700080B483B000AF786000BF0C37BD465DF8A3
:10958000047B704780B487B000AF786039607B6837
:109590005B68B3F5403F7B6893F83830012B01D10D
:1095A000022379E07B68012283F838207B6802225D
:1095B00083F839203B681B0118337A6813443B61F8
:1095C0003B695A683B699B681B0413437B61354BBD
:1095D000FB603B695B680A2B03D03B695B68092B26
:1095E00007D13B69DB6803F07F437A6913437B61F2
:1095F00005E03B69DB681B067A6913437B613B68C6
:10960000002B20D17B681B685A6AFB68DB4302EAA7
:1096100003017B681B687A690A435A627B681B688E
:109620003A6912689A613B695B680A2B03D03B690F
:109630005B68092B27D13B69DA687B681B6822F0DD
:109640007F429A621FE07B681B68DA69FB68DB4334
:1096500002EA03017B681B687A690A43DA617B6866
:109660001B683A6912681A613B695B680A2B03D070
:109670003B695B68092B06D13B69DA687B681B682C
:1096800022F07F421A627B68012283F839207B68CE
:10969000002283F83820002318461C37BD465DF8A9
:1096A000047B70470F0003FF80B489B000AF78607F
:1096B00039600023FB6100237B6100233B610023B1
:1096C000BB610023FB6175E10122FB6902FA03F330
:1096D0007B613B681B687A6913403B613A697B692F
:1096E0009A4240F064813B685B68012B0BD03B6879
:1096F0005B68022B07D03B685B68112B03D03B688B
:109700005B68122B30D17B689B68BB61FB695B0097
:10971000032202FA03F3DB43BA691340BB613B68DF
:10972000DA68FB695B0002FA03F3BA691343BB61B1
:109730007B68BA699A607B685B68BB610122FB69E0
:1097400002FA03F3DB43BA691340BB613B685B6811
:109750001B0903F00102FB6902FA03F3BA69134320
:10976000BB617B68BA695A607B68DB68BB61FB6977
:109770005B00032202FA03F3DB43BA691340BB61C7
:109780003B689A68FB695B0002FA03F3BA6913430A
:10979000BB617B68BA69DA603B685B68022B03D007
:1097A0003B685B68122B23D1FB69DA087B680832BF
:1097B00053F82230BB61FB6903F007039B000F22C3
:1097C00002FA03F3DB43BA691340BB613B681A69D1
:1097D000FB6903F007039B0002FA03F3BA69134322
:1097E000BB61FB69DA087B680832B96943F822106B
:1097F0007B681B68BB61FB695B00032202FA03F311
:10980000DB43BA691340BB613B685B6803F003024A
:10981000FB695B0002FA03F3BA691343BB617B681F
:10982000BA691A603B685B6803F08053002B00F054
:10983000BE80664B5B6C654A43F480435364634B64
:109840005B6C03F48043FB60FB68614AFB699B0827
:10985000023352F82330BB61FB6903F003039B0022
:109860000F2202FA03F3DB43BA691340BB617B6842
:10987000584A934237D07B68574A934231D07B682D
:10988000564A93422BD07B68554A934225D07B6839
:10989000544A93421FD07B68534A934219D07B6845
:1098A000524A934213D07B68514A93420DD07B6851
:1098B000504A934207D07B684F4A934201D1092313
:1098C00012E00A2310E008230EE007230CE0062331
:1098D0000AE0052308E0042306E0032304E0022352
:1098E00002E0012300E00023FA6902F00302920083
:1098F0009340BA691343BB613549FB699B08023346
:10990000BA6941F823203D4B1B68BB613B69DB43CF
:10991000BA691340BB613B685B6803F48033002B7A
:1099200003D0BA693B691343BB61344ABB69136016
:10993000324B5B68BB613B69DB43BA691340BB6177
:109940003B685B6803F40033002B03D0BA693B69C2
:109950001343BB61294ABB695360284B9B68BB61B9
:109960003B69DB43BA691340BB613B685B6803F446
:109970008013002B03D0BA693B691343BB611F4AB4
:10998000BB6993601D4BDB68BB613B69DB43BA6914
:109990001340BB613B685B6803F40013002B03D0EA
:1099A000BA693B691343BB61144ABB69D360FB6965
:1099B0000133FB61FB690F2B7FF686AE00BF00BF52
:1099C0002437BD465DF8047B704700BF0038024075
:1099D000003801400000024000040240000802403C
:1099E000000C024000100240001402400018024027
:1099F000001C02400020024000240240003C0140C4
:109A000080B487B000AF7860396000233B610023E9
:109A1000FB600023BB6000237B61D9E001227B69EE
:109A200002FA03F33B613A683B691340FB60FA6852
:109A30003B699A4240F0C9806B4A7B699B080233BC
:109A400052F82330BB607B6903F003039B000F22B5
:109A500002FA03F3BA681340BB607B68634A93421F
:109A600037D07B68624A934231D07B68614A934227
:109A70002BD07B68604A934225D07B685F4A934233
:109A80001FD07B685E4A934219D07B685D4A93423F
:109A900013D07B685C4A93420DD07B685B4A93424B
:109AA00007D07B685A4A934201D1092312E00A2366
:109AB00010E008230EE007230CE006230AE005234C
:109AC00008E0042306E0032304E0022302E001236C
:109AD00000E000237A6902F0030292009340BA6822
:109AE0009A4232D14B4B1A68FB68DB434949134019
:109AF0000B60484B5A68FB68DB43464913404B6098
:109B0000444B9A68FB68DB43424913408B60414BEE
:109B1000DA68FB68DB433F491340CB607B6903F0A5
:109B200003039B000F2202FA03F3BB602E4A7B69FA
:109B30009B08023352F82310BB68DA432A487B693A
:109B40009B080A40023340F823207B681A687B692F
:109B50005B00032101FA03F3DB431A407B681A60C0
:109B60007B69DA087B68083253F822107B6903F0BE
:109B700007039B000F2202FA03F3DB437A69D20842
:109B800019407B68083243F822107B68DA687B69E9
:109B90005B00032101FA03F3DB431A407B68DA60C0
:109BA0007B685A6801217B6901FA03F3DB431A40A1
:109BB0007B685A607B689A687B695B00032101FAC5
:109BC00003F3DB431A407B689A607B6901337B6156
:109BD0007B690F2B7FF622AF00BF00BF1C37BD464D
:109BE0005DF8047B704700BF003801400000024070
:109BF0000004024000080240000C02400010024035
:109C00000014024000180240001C024000200240E4
:109C100000240240003C014080B485B000AF786071
:109C20000B467B807B681A697B881340002B02D02F
:109C30000123FB7301E00023FB73FB7B1846143701
:109C4000BD465DF8047B704780B483B000AF786098
:109C50000B467B8013467B707B78002B03D07A8881
:109C60007B689A6103E07B881A047B689A6100BF75
:109C70000C37BD465DF8047B7047000080B582B0AC
:109C800000AF78607B68002B01D101237FE07B6807
:109C900093F84130DBB2002B06D17B68002283F8B9
:109CA00040207868F8F756FD7B68242283F841202D
:109CB0007B681B681A687B681B6822F001021A60C7
:109CC0007B685A687B681B6822F070621A617B6847
:109CD0001B689A687B681B6822F400429A607B6864
:109CE000DB68012B07D17B689A687B681B6842F4AC
:109CF00000429A6006E07B689A687B681B6842F4C1
:109D000004429A607B68DB68022B04D17B681B6885
:109D10004FF400625A607B681B6859687B681A6858
:109D20001D4B0B4353607B681B68DA687B681B68BC
:109D300022F40042DA607B681A697B685B6942EA58
:109D400003017B689B691A027B681B680A43DA601F
:109D50007B68D9697B681A6A7B681B680A431A604A
:109D60007B681B681A687B681B6842F001021A60F6
:109D70007B6800225A647B68202283F841207B683C
:109D800000221A637B68002283F8422000231846D1
:109D90000837BD4680BD00BF0080000280B582B09C
:109DA00000AF78607B68002B01D1012321E07B6844
:109DB000242283F841207B681B681A687B681B6833
:109DC00022F001021A607868F8F76CFD7B680022C7
:109DD0005A647B68002283F841207B6800221A6362
:109DE0007B68002283F842207B68002283F84020B1
:109DF000002318460837BD4680BD000080B588B0F6
:109E000002AFF860084611461A4603467B810B46AE
:109E10003B811346FB80FB6893F84130DBB2202B7B
:109E200040F0F9803B6A002B02D0BB8C002B05D19F
:109E3000FB684FF400725A640123EDE0FB6893F86D
:109E40004030012B01D10223E6E0FB68012283F8B8
:109E50004020FEF77DFB78617B6900931923012286
:109E60004FF40041F86800F0C3FA0346002B01D01C
:109E70000123D1E0FB68212283F84120FB684022C6
:109E800083F84220FB6800225A64FB683A6A5A62EF
:109E9000FB68BA8C5A85FB6800225A63F8883A89B5
:109EA00079897B690193BB6A00930346F86800F0E7
:109EB000D3F90346002B05D0FB68002283F840202D
:109EC0000123A9E0FB685B8D9BB2FF2B0ED9FB68D9
:109ED000FF221A85FB681B8DDAB279890023009373
:109EE0004FF08073F86800F0A5FB0FE0FB685B8D16
:109EF0009AB2FB681A85FB681B8DDAB27989002358
:109F000000934FF00073F86800F094FB7A69B96A27
:109F1000F86800F0ADFA0346002B01D001237BE086
:109F2000FB685B6A1A78FB681B689A62FB685B6A6D
:109F30005A1CFB685A62FB685B8D9BB2013B9AB26C
:109F4000FB685A85FB681B8D013B9AB2FB681A853A
:109F5000FB685B8D9BB2002B34D0FB681B8D002B04
:109F600030D17B690093BB6A00228021F86800F041
:109F70003FFA0346002B01D001234DE0FB685B8DC7
:109F80009BB2FF2B0ED9FB68FF221A85FB681B8D45
:109F9000DAB27989002300934FF08073F86800F0FB
:109FA00049FB0FE0FB685B8D9AB2FB681A85FB6882
:109FB0001B8DDAB27989002300934FF00073F868A3
:109FC00000F038FBFB685B8D9BB2002B9ED17A6959
:109FD000B96AF86800F08CFA0346002B01D001231F
:109FE0001AE0FB681B682022DA61FB681B6859686D
:109FF000FB681A680A4B0B405360FB68202283F809
:10A000004120FB68002283F84220FB68002283F88D
:10A010004020002300E0022318461837BD4680BDCB
:10A0200000E800FE80B588B002AFF860084611462F
:10A030001A4603467B810B463B811346FB80FB6837
:10A0400093F84130DBB2202B40F0FD803B6A002BBF
:10A0500002D0BB8C002B05D1FB684FF400725A6410
:10A060000123F1E0FB6893F84030012B01D102237A
:10A07000EAE0FB68012283F84020FEF769FA786184
:10A080007B690093192301224FF40041F86800F026
:10A09000AFF90346002B01D00123D5E0FB68222253
:10A0A00083F84120FB68402283F84220FB680022AD
:10A0B0005A64FB683A6A5A62FB68BA8C5A85FB6834
:10A0C00000225A63F8883A8979897B690193BB6ACF
:10A0D00000930346F86800F013F90346002B05D0FF
:10A0E000FB68002283F840200123ADE0FB685B8D14
:10A0F0009BB2FF2B0ED9FB68FF221A85FB681B8DD4
:10A10000DAB27989524B00934FF08073F86800F00F
:10A1100091FA0FE0FB685B8D9AB2FB681A85FB68C9
:10A120001B8DDAB279894A4B00934FF00073F868BF
:10A1300000F080FA7B690093BB6A00220421F86872
:10A1400000F056F90346002B01D001237CE0FB68A8
:10A150001B685A6AFB685B6AD2B21A70FB685B6A5A
:10A160005A1CFB685A62FB681B8D013B9AB2FB6864
:10A170001A85FB685B8D9BB2013B9AB2FB685A85DE
:10A18000FB685B8D9BB2002B34D0FB681B8D002BD2
:10A1900030D17B690093BB6A00228021F86800F00F
:10A1A00027F90346002B01D001234DE0FB685B8DAE
:10A1B0009BB2FF2B0ED9FB68FF221A85FB681B8D13
:10A1C000DAB27989002300934FF08073F86800F0C9
:10A1D00031FA0FE0FB685B8D9AB2FB681A85FB6869
:10A1E0001B8DDAB27989002300934FF00073F86871
:10A1F00000F020FAFB685B8D9BB2002B9AD17A6944
:10A20000B96AF86800F074F90346002B01D0012305
:10A210001AE0FB681B682022DA61FB681B6859683A
:10A22000FB681A680B4B0B405360FB68202283F8D5
:10A230004120FB68002283F84220FB68002283F85B
:10A240004020002300E0022318461837BD4680BD99
:10A250000024008000E800FE80B586B002AFF86000
:10A26000084611461A4603467B810B463B8113463E
:10A27000FB80FB88DAB27989204B00934FF0807322
:10A28000F86800F0D7F9FA69B969F86800F0F0F8F1
:10A290000346002B01D001232CE0FB88012B05D1C4
:10A2A0003B89DAB2FB681B689A6215E03B891B0A9E
:10A2B0009BB2DAB2FB681B689A62FA69B969F868FE
:10A2C00000F0D6F80346002B01D0012312E03B89B1
:10A2D000DAB2FB681B689A62FB690093BB690022D3
:10A2E0008021F86800F084F80346002B01D0012398
:10A2F00000E0002318461037BD4680BD00200080D6
:10A3000080B586B002AFF860084611461A4603468B
:10A310007B810B463B811346FB80FB88DAB279894F
:10A32000204B00930023F86800F084F9FA69B969BA
:10A33000F86800F09DF80346002B01D001232CE0C3
:10A34000FB88012B05D13B89DAB2FB681B689A6256
:10A3500015E03B891B0A9BB2DAB2FB681B689A6264
:10A36000FA69B969F86800F083F80346002B01D058
:10A37000012312E03B89DAB2FB681B689A62FB6931
:10A380000093BB6900224021F86800F031F80346D1
:10A39000002B01D0012300E0002318461037BD46F2
:10A3A00080BD00BF0020008080B483B000AF786023
:10A3B0007B681B689B6903F00203022B03D17B6857
:10A3C0001B6800229A627B681B689B6903F001038B
:10A3D000012B07D07B681B689A697B681B6842F079
:10A3E00001029A6100BF0C37BD465DF8047B7047DF
:10A3F00080B584B000AFF860B9603B601346FB7174
:10A4000022E03B68B3F1FF3F1ED0FEF7A1F8024601
:10A41000BB69D31A3A689A4202D33B68002B13D126
:10A42000FB685B6C43F02002FB685A64FB682022E7
:10A4300083F84120FB68002283F84220FB68002259
:10A4400083F8402001230FE0FB681B689A69BB6812
:10A450001340BA689A420CBF01230023DBB21A46AC
:10A46000FB799A42CDD0002318461037BD4680BDF7
:10A4700080B584B000AFF860B9607A602CE07A688B
:10A48000B968F86800F070F80346002B01D001238A
:10A490002AE0BB68B3F1FF3F1ED0FEF759F8024631
:10A4A0007B68D31ABA689A4202D3BB68002B13D1D7
:10A4B000FB685B6C43F02002FB685A64FB68202257
:10A4C00083F84120FB68002283F84220FB680022C9
:10A4D00083F84020012307E0FB681B689B6903F0B9
:10A4E0000203022BCBD1002318461037BD4680BD96
:10A4F00080B584B000AFF860B9607A6028E07A680F
:10A50000B968F86800F030F80346002B01D0012349
:10A5100026E0FEF71DF802467B68D31ABA689A4215
:10A5200002D3BB68002B13D1FB685B6C43F02002A5
:10A53000FB685A64FB68202283F84120FB680022F4
:10A5400083F84220FB68002283F84020012307E0C3
:10A55000FB681B689B6903F02003202BCFD10023ED
:10A5600018461037BD4680BD80B584B000AFF86096
:10A57000B9607A60FB681B689B6903F01003102BBD
:10A5800051D122E0BB68B3F1FF3F1ED0FDF7E0FFE1
:10A5900002467B68D31ABA689A4202D3BB68002B82
:10A5A00013D1FB685B6C43F02002FB685A64FB68C4
:10A5B000202283F84120FB68002283F84220FB68B8
:10A5C000002283F8402001232EE0FB681B689B6972
:10A5D00003F02003202BD5D1FB681B681022DA6121
:10A5E000FB681B682022DA61F868FFF7DDFEFB6874
:10A5F0001B685968FB681A680D4B0B405360FB6879
:10A600005B6C43F00402FB685A64FB68202283F809
:10A610004120FB68002283F84220FB68002283F877
:10A620004020012300E0002318461037BD4680BDBE
:10A6300000E800FE80B485B000AFF8607B600B4698
:10A640007B8113467B72FB681B685A68BB695B0D94
:10A6500003F480610D4B0B43DB4302EA03017B896A
:10A66000C3F309027B7A1B0403F47F031A437B685C
:10A670001A43BB691A43FB681B680A435A6000BF50
:10A680001437BD465DF8047B704700BFFF63FF03CE
:10A6900080B483B000AF786039607B6893F8413054
:10A6A000DBB2202B38D17B6893F84030012B01D1ED
:10A6B000022332E07B68012283F840207B68242259
:10A6C00083F841207B681B681A687B681B6822F04E
:10A6D00001021A607B681B681A687B681B6822F499
:10A6E00080521A607B681B6819687B681B683A682F
:10A6F0000A431A607B681B681A687B681B6842F013
:10A7000001021A607B68202283F841207B680022C6
:10A7100083F84020002300E0022318460C37BD4692
:10A720005DF8047B704780B485B000AF7860396015
:10A730007B6893F84130DBB2202B39D17B6893F8EA
:10A740004030012B01D1022333E07B68012283F8E2
:10A7500040207B68242283F841207B681B681A68AC
:10A760007B681B6822F001021A607B681B681B680B
:10A77000FB60FB6823F47063FB603B681B02FA68B4
:10A780001343FB607B681B68FA681A607B681B6870
:10A790001A687B681B6842F001021A607B682022FD
:10A7A00083F841207B68002283F84020002300E0EA
:10A7B000022318461437BD465DF8047B704700003D
:10A7C00080B584B000AF78607B68002B01D1012395
:10A7D000BFE07B6893F8A130DBB2002B06D17B6829
:10A7E000002283F8A0207868F8F798F87B680222A6
:10A7F00083F8A1207B681B689A697B681B6822F03C
:10A8000070429A617B681B6899697B685A687B68AB
:10A810009B681A437B68DB681A437B681B691A4391
:10A820007B681B680A439A617B681B6899687B6830
:10A830001A684A4B0B4093607B685B691B04FB60A2
:10A840007B681B6899687B689A69FB681A437B6818
:10A850001B680A439A607B681B68D9687B681A6822
:10A860003E4B0B40D3607B68DB691B04FB607B685D
:10A870001B68D9687B681A6AFB681A437B681B6887
:10A880000A43DA607B681B6819697B681A68334B76
:10A890000B4013617B685B6A1B04FB607B681B6871
:10A8A00019697B689A6AFB681A437B681B680A43CC
:10A8B0001A617B681B6859697B681A68274B0B40D3
:10A8C00053617B68DB6A1B04FB607B681B6859690A
:10A8D0007B681A6BFB681A437B681B680A435A61E2
:10A8E0007B6893F835301B02FB607B6893F8363049
:10A8F0001B04BB607B681B68DA6A7B681B6802F01C
:10A900007F42DA627B681B68D96ABA68FB681343C6
:10A910007A6892F834201A437B681B680A43DA622B
:10A920007B681B685A6B7B681B6842F006025A639F
:10A930007B681B689A697B681B6842F001029A6118
:10A940007B680022C3F8A4207B68012283F8A12041
:10A95000002318461037BD4680BD00BF00F800F048
:10A9600080B584B000AF78607B681B689B6BFB6030
:10A970007B681B685B6BBB60FB6803F00403002B08
:10A9800023D0BB6803F00403002B1ED07B681B6838
:10A990005A6B7B681B6822F004025A637B681B6851
:10A9A0000422DA637B68D3F8A43043F001027B68A9
:10A9B000C3F8A4207B68042283F8A1207B680022CE
:10A9C00083F8A020786800F06FF8FB6803F00203BA
:10A9D000002B23D0BB6803F00203002B1ED07B6842
:10A9E0001B685A6B7B681B6822F002025A637B6803
:10A9F0001B680222DA637B68D3F8A43043F00202BA
:10AA00007B68C3F8A4207B68042283F8A1207B68BC
:10AA1000002283F8A020786800F046F8FB6803F075
:10AA20000103002B1BD0BB6803F00103002B16D0E1
:10AA30007B681B685A6B7B681B6822F001025A63B3
:10AA40007B681B680122DA637B68012283F8A120FE
:10AA50007B68002283F8A0207868F9F7F5FCFB6892
:10AA600003F00803002B1BD0BB6803F00803002B86
:10AA700016D07B681B685A6B7B681B6822F0080243
:10AA80005A637B681B680822DA637B68012283F8BB
:10AA9000A1207B68002283F8A020786800F00EF8DF
:10AAA00000BF1037BD4680BD80B483B000AF786072
:10AAB00000BF0C37BD465DF8047B704780B483B09F
:10AAC00000AF786000BF0C37BD465DF8047B70476F
:10AAD000B0B584B000AFF860B9607A60FB6893F8F5
:10AAE000A030012B01D102232CE0FB68012283F866
:10AAF000A020FB68022283F8A120FA687B68342139
:10AB000001FB03F3134403F13802BB6814461D46EE
:10AB10000FCD0FC40FCD0FC40FCD0FC42B68236012
:10AB20007A68B968F86800F049F8FB681B68012288
:10AB30005A62FB68012283F8A120FB68002283F897
:10AB4000A020002318461037BD46B0BD80B483B0A6
:10AB500000AF786039607B6893F8A030012B01D199
:10AB6000022323E07B68012283F8A0207B68022275
:10AB700083F8A1207B681B685A6B7B681B6822F0F6
:10AB800001025A630C4A3B6813647B681B685A6B6A
:10AB90007B681B6842F001025A637B68012283F8DC
:10ABA000A1207B68002283F8A020002318460C37E0
:10ABB000BD465DF8047B70470068014080B489B0F1
:10ABC00000AFF860B9607A60BB685A68FB681B68C0
:10ABD000DB681B0CC3F30B0313441B04FB61FB6812
:10ABE0001B681A467B68DB01134484335B68FA6890
:10ABF000126811467A68D2010A44843203F4704321
:10AC00005360BB681A68FB681B68DB681B0CC3F3E6
:10AC10000B0313445A1CFB681B6819467B68DB0155
:10AC20000B4484331946FB6913434B60BB68DA68F5
:10AC3000FB681B68DB68C3F30A0313441B04FB6156
:10AC4000FB681B681A467B68DB01134484339B68EE
:10AC5000FA68126811467A68D2010A44843203F411
:10AC600070439360BB689A68FB681B68DB68C3F33A
:10AC70000A0313445A1CFB681B6819467B68DB01F6
:10AC80000B4484331946FB6913438B60FB681B68D4
:10AC90001A467B68DB01134484331B69FA68126827
:10ACA00011467A68D2010A44843223F00703136103
:10ACB000FB681B681A467B68DB01134484331A4621
:10ACC000BB681B691361BB6893F831301B02FB61E1
:10ACD000BB6893F832301B04BB61BB689B691B06E1
:10ACE0007B61FB681B681A467B68DB011344843375
:10ACF0009B69FB681B681A467B68DB01134484333D
:10AD00001A4600239361BB6893F830301A46FB69FA
:10AD10001A43BB691A43FB681B6819467B68DB0151
:10AD20000B44843319467B6913438B61FB681B68B2
:10AD30001A467B68DB01134484335B69FA68126846
:10AD400011467A68D2010A44843223F0FF0353612A
:10AD5000FB681B681A467B68DB01134484331A4680
:10AD6000BB685B695361FB681B681A467B68DB0143
:10AD700013448433DA69FB681B6819467B68DB017E
:10AD80000B4484331946584B1340CB61BB68DA69D6
:10AD9000BB681B6AF968096808467968C9010144FB
:10ADA00084311343CB61FB681B681A467B68DB0167
:10ADB000134484339B6AFB681B681A467B68DB017B
:10ADC000134484331A4600239362FB681B681A46B7
:10ADD0007B68DB01134484331A46BB685B6A936269
:10ADE000BB681B69002B02D10423FB611BE0BB681D
:10ADF0001B69012B02D10323FB6114E0BB681B69B3
:10AE0000042B0BD0BB681B69022B07D0BB681B69E6
:10AE1000032B03D0BB681B69072B02D10223FB6104
:10AE200001E00123FB61FB681B681A467B68DB01BC
:10AE300013448433DB6AFA68126811467A68D201D7
:10AE40000A44843203F0E023D362BB689B6AFA6948
:10AE500002FB03F31A04BB685968BB681B68CB1A72
:10AE6000F96901FB03F30333F96809680846796857
:10AE7000C901014484311343CB62FB681B681A4645
:10AE80007B68DB01134484331A6BFB681B6819462B
:10AE90007B68DB010B4484331946144B13400B636E
:10AEA000FB681B681A467B68DB01134484331A462F
:10AEB000BB68DB6A1363FB681B681A467B68DB01AF
:10AEC000134484331B68FA68126811467A68D20109
:10AED0000A44843243F00103136000BF2437BD46A7
:10AEE0005DF8047B704700BFF8F8FFFF00F8FFFF34
:10AEF00080B582B000AF00237B60234B1B6C224ADD
:10AF000043F080531364204B1B6C03F080533B6071
:10AF10003B681E4B1B681D4A43F480331360FDF7EA
:10AF200017FB786009E0FDF713FB02467B68D31A34
:10AF3000B3F57A7F01D9032322E0144B5B6803F455
:10AF40008033B3F5803FEED1104B1B680F4A43F4BA
:10AF500000331360FDF7FCFA786009E0FDF7F8FABA
:10AF600002467B68D31AB3F57A7F01D9032307E041
:10AF7000064B5B6803F40033B3F5003FEED10023CA
:10AF800018460837BD4680BD0038024000700040BA
:10AF900080B586B002AF7860FDF7DAFAF8607B68BA
:10AFA000002B01D1012367E07B6893F84130DBB2CD
:10AFB000002B0BD17B68002283F840207868F7F7DC
:10AFC000AFFD41F28831786800F05FFB7B681B6859
:10AFD0001B6823F4F8517B689B68013B1A027B686D
:10AFE0001B680A431A607B689B6C0093FB68002215
:10AFF0002021786800F057FB0346FB72FB7A002B98
:10B0000035D17B681B681A681D4B13407A685268FB
:10B0100011067A68D26811437A68D26911437A6856
:10B02000126A11437A6812680B4313607B681B68CD
:10B030005A68144B13407A68126911047A6852698D
:10B0400011437A68926911437A6812680B4353601E
:10B050007B681B681A687B681B6842F001021A60F3
:10B060007B6800225A647B68012283F841207B6858
:10B07000002283F84020FB7A18461037BD4680BD79
:10B080002FFFFF00FEF8E0FF80B582B000AF7860D0
:10B090007B68002B01D1012316E07B681B681A68CE
:10B0A0007B681B6822F001021A607868F7F7C8FD18
:10B0B0007B6800225A647B68002283F841207B6809
:10B0C000002283F84020002318460837BD4680BD83
:10B0D00080B588B002AFF860B9607A60FDF738FAE1
:10B0E0003861FB6893F84030DBB2012B01D10223B9
:10B0F00048E0FB68012283F84020FB6893F8413068
:10B10000DBB2012B37D1FB6800225A64FB680222B4
:10B1100083F841207B6800933B6900222021F86876
:10B1200000F0C1FA0346FB75FB7D002B25D1002200
:10B13000B968F86800F0EEFABB685B6A002B15D1BD
:10B140007B6800933B6901220221F86800F0ABFAAA
:10B150000346FB75FB7D002B0FD1FB681B680222A9
:10B16000DA60FB68012283F8412006E0FB680122D7
:10B1700083F8412001E00223FB75FB68002283F87D
:10B180004020FB7D18461837BD4680BD80B58AB08B
:10B1900002AFF860B9607A600023FB77FDF7D8F959
:10B1A000B861FB681B6820337B61FB6893F8403013
:10B1B000DBB2012B01D102237BE0FB68012283F883
:10B1C0004020FB6893F84130DBB2012B6AD1FB6869
:10B1D00000225A64BB68002B5BD0FB68122283F804
:10B1E0004120FB681B681B695A1CFB68DA62FB681C
:10B1F0001B681B695A1CFB689A62FB68BA685A6232
:10B20000FB681B685A69FB681B6822F040625A6140
:10B210001BE07B680093BB6901220421F86800F001
:10B2200042FA0346FB77FB7F002B13D1FB685B6A76
:10B230001A787B691A70FB685B6A5A1CFB685A6251
:10B24000FB68DB6A5A1EFB68DA62FB68DB6A002B6C
:10B25000DFD100E000BFFB7F002B15D17B6800939E
:10B26000BB6901220221F86800F01DFA0346FB7752
:10B27000FB7F002B08D1FB681B680222DA60F868AC
:10B2800000F096F90346FB77FB68012283F8412022
:10B290000AE0FB685B6C43F00802FB685A64012318
:10B2A000FB7701E00223FB77FB68002283F8402054
:10B2B000FB7F18462037BD4680BD80B58AB002AFFF
:10B2C000F860B9607A600023FB77FDF741F9B86157
:10B2D000FB681B689B697B61FB681B6820333B61D3
:10B2E000FB6893F84030DBB2012B01D1022382E0EE
:10B2F000FB68012283F84020FB6893F84130DBB201
:10B30000012B71D1FB6800225A64BB68002B62D00C
:10B31000FB68222283F84120FB681B681B695A1CCA
:10B32000FB689A63FB681B681B695A1CFB685A63BD
:10B33000FB68BA681A63FB681B685B6923F04062AC
:10B34000FB681B6842F080625A61FB681B687A697F
:10B350009A611CE07B680093BB6901220621F868B2
:10B3600000F0A1F90346FB77FB7F002B14D1FB68AB
:10B370001B6B3A691278D2B21A70FB681B6B5A1CAD
:10B38000FB681A63FB689B6B5A1EFB689A63FB6839
:10B390009B6B002BDED100E000BFFB7F002B15D1A3
:10B3A0007B680093BB6901220221F86800F07BF9F9
:10B3B0000346FB77FB7F002B08D1FB681B6802224A
:10B3C000DA60F86800F0F4F80346FB77FB680122C6
:10B3D00083F841200AE0FB685B6C43F00802FB68DD
:10B3E0005A640123FB7701E00223FB77FB6800220C
:10B3F00083F84020FB7F18462037BD4680BD80B5CE
:10B4000088B002AFF860B9607A603B60FDF7A0F8E1
:10B410003861FB6893F84030DBB2012B01D1022385
:10B4200060E0FB68012283F84020FB6893F841301C
:10B43000DBB2012B4FD1FB6800225A64FB68422229
:10B4400083F841203B6800933B6900222021F86883
:10B4500000F029F90346FB75FB7D002B3DD1FB680D
:10B460001B687A6812689A62FB681B687A6852687F
:10B470005A62FB681B687A689268DA62FB681B682C
:10B480001B6823F440027B681B691A43FB681B6836
:10B4900042F480021A607B68DA68BB689A624FF0F7
:10B4A0000062B968F86800F035F93B6800933B69C1
:10B4B00001220821F86800F0F6F80346FB75FB7DD1
:10B4C000002B0AD1FB681B680822DA60FB680122A6
:10B4D00083F8412001E00223FB75FB68002283F81A
:10B4E0004020FB7D18461837BD4680BD80B588B02A
:10B4F00002AFF860B9607A60FDF72AF83861FB683E
:10B5000093F84030DBB2012B01D102234CE0FB6801
:10B51000012283F84020FB6893F84130DBB2012B15
:10B520003BD1FB6800225A64FB68822283F84120E9
:10B53000FB689B6C00933B6900222021F86800F0B7
:10B54000B2F80346FB75FB7D002B28D1FB681B6816
:10B550001B6823F008017B685A68FB681B680A4374
:10B560001A607B685B68082B10D1FB681B687A68DF
:10B5700012681A63FB681B681022DA60FB681B689C
:10B580001A68FB681B6842F480121A604FF0406230
:10B59000B968F86800F0BEF801E00223FB75FB68AB
:10B5A000002283F84020FB7D18461837BD4680BD39
:10B5B00080B586B002AF78600023FB73FCF7C8FF4C
:10B5C000B8607B6893F84130DBB203F00203002BD4
:10B5D00056D07B68002283F840207B681B681B687C
:10B5E00003F00403002B17D07B681B681A687B6884
:10B5F0001B6822F004021A607B68DB6B1846FDF7BB
:10B600005FFB0346FB73FB7B002B05D07B685B6C09
:10B6100043F004027B685A647B681B681A687B6885
:10B620001B6842F002021A607B689B6C0093BB6847
:10B6300001220221786800F036F80346FB73FB7B99
:10B64000002B0ED17B681B680222DA607B689B6C42
:10B650000093BB6800222021786800F024F803469C
:10B66000FB73FB7B002B0BD17B681B685A697B68E3
:10B670001B6822F040625A617B68012283F84120F6
:10B68000FB7B18461037BD4680BD80B483B000AF49
:10B69000786039607B683A689A6400BF0C37BD46B1
:10B6A0005DF8047B704780B584B000AFF860B96086
:10B6B0003B601346FB711AE0BB69B3F1FF3F16D044
:10B6C000FCF746FF02463B68D31ABA699A4202D396
:10B6D000BB69002B0BD1FB68042283F84120FB6877
:10B6E0005B6C43F00102FB685A6401230EE0FB68C7
:10B6F0001B689A68BB681340002B14BF012300230A
:10B70000DBB21A46FB799A42D6D10023184610378D
:10B71000BD4680BD80B485B000AFF860B9607A6086
:10B72000BB685B6A002B09D07B68B3F1406F05D022
:10B73000BB689A6AFB681B68013A1A61BB689B691F
:10B74000002B00F0B980BB681B6A002B5FD0FB6840
:10B750001B68BA689268DA61BB68DB69002B31D07C
:10B76000BB68DA6ABB681B6B1A43BB685B6B1A4326
:10B77000BB685B6A1A43BB685B699B041A43BB687E
:10B780001B691A43BB681B6A1A43BB68DB681A4310
:10B79000BB68DB691A43BB689B691A43BB681B68BB
:10B7A00042EA0301FB681B687A680A435A617B68B6
:10B7B000B3F1406F00F02E81FB681B68BA685268D5
:10B7C0009A6127E1BB68DA6ABB681B6B1A43BB68E6
:10B7D0005B6B1A43BB685B6A1A43BB685B699B047B
:10B7E0001A43BB681B691A43BB681B6A1A43BB68D0
:10B7F000DB691A43BB689B691A43BB681B6842EA52
:10B800000301FB681B687A680A435A6102E1BB685E
:10B81000DB69002B2ED0BB68DA6ABB681B6B1A434E
:10B82000BB685B6B1A43BB685B6A1A43BB685B69A6
:10B830009B041A43BB681B6A1A43BB68DB681A4344
:10B84000BB68DB691A43BB689B691A43BB681B680A
:10B8500042EA0301FB681B687A680A435A617B6805
:10B86000B3F1406F00F0D680FB681B68BA6852687D
:10B870009A61CFE0BB68DA6ABB681B6B1A43BB688E
:10B880005B6B1A43BB685B6A1A43BB685B699B04CA
:10B890001A43BB681B6A1A43BB68DB691A43BB685F
:10B8A0009B691A43BB681B6842EA0301FB681B687B
:10B8B0007A680A435A61ADE0BB681B6A002B58D016
:10B8C000FB681B68BA689268DA61BB68DB69002BA9
:10B8D0002DD0BB68DA6ABB681B6B1A43BB685B6B15
:10B8E0001A43BB685B6A1A43BB685B699B041A43D3
:10B8F000BB681B691A43BB681B6A1A43BB68DB68D9
:10B900001A43BB68DB691A43BB689B6942EA0301BF
:10B91000FB681B687A680A435A617B68B3F1406F21
:10B9200078D0FB681B68BA6852689A6172E0BB689D
:10B93000DA6ABB681B6B1A43BB685B6B1A43BB6854
:10B940005B6A1A43BB685B699B041A43BB681B694B
:10B950001A43BB681B6A1A43BB68DB691A43BB689E
:10B960009B6942EA0301FB681B687A680A435A61D3
:10B9700050E0BB68DB69002B2AD0BB68DA6ABB6881
:10B980001B6B1A43BB685B6B1A43BB685B6A1A4349
:10B99000BB685B699B041A43BB681B6A1A43BB689C
:10B9A000DB681A43BB68DB691A43BB689B6942EAE0
:10B9B0000301FB681B687A680A435A617B68B3F12C
:10B9C000406F27D0FB681B68BA6852689A6121E013
:10B9D000BB685B6A002B1DD0BB68DA6ABB681B6B57
:10B9E0001A43BB685B6B1A43BB685B6A1A43BB684C
:10B9F0005B699B041A43BB681B6A1A43BB68DB691B
:10BA00001A43BB689B6942EA0301FB681B687A68BA
:10BA10000A435A6100BF1437BD465DF8047B704786
:10BA200080B586B000AF78600023FB757B68002B83
:10BA300001D1012391E27B681B6803F00103002B15
:10BA400000F08780964B9B6803F00C03042B0CD00E
:10BA5000934B9B6803F00C03082B12D1904B5B684F
:10BA600003F48003B3F5800F0BD18D4B1B6803F4F7
:10BA70000033002B6CD07B685B68002B68D10123FE
:10BA80006BE27B685B68B3F5803F06D1844B1B6833
:10BA9000834A43F4803313602EE07B685B68002B9D
:10BAA0000CD17F4B1B687E4A23F4803313607C4BA0
:10BAB0001B687B4A23F4802313601DE07B685B686E
:10BAC000B3F5A02F0CD1764B1B68754A43F4802345
:10BAD0001360734B1B68724A43F4803313600BE0AE
:10BAE0006F4B1B686E4A23F4803313606C4B1B68EA
:10BAF0006B4A23F4802313607B685B68002B13D0B0
:10BB0000FCF726FD386108E0FCF722FD02463B69A0
:10BB1000D31A642B01D903231FE2614B1B6803F482
:10BB20000033002BF0D014E0FCF712FD386108E080
:10BB3000FCF70EFD02463B69D31A642B01D903239F
:10BB40000BE2574B1B6803F40033002BF0D100E0ED
:10BB500000BF7B681B6803F00203002B69D0504BC9
:10BB60009B6803F00C03002B0BD04D4B9B6803F03C
:10BB70000C03082B1CD14A4B5B6803F48003002B99
:10BB800016D1474B1B6803F00203002B05D07B68DE
:10BB9000DB68012B01D00123DFE1414B1B6823F05F
:10BBA000F8027B681B69DB003D4913430B6040E0F2
:10BBB0007B68DB68002B23D0394B1B68384A43F085
:10BBC00001031360FCF7C4FC386108E0FCF7C0FC1B
:10BBD00002463B69D31A022B01D90323BDE1304B46
:10BBE0001B6803F00203002BF0D02D4B1B6823F0E1
:10BBF000F8027B681B69DB00294913430B6018E0DE
:10BC0000274B1B68264A23F001031360FCF7A0FCB6
:10BC1000386108E0FCF79CFC02463B69D31A022B12
:10BC200001D9032399E11E4B1B6803F00203002B8B
:10BC3000F0D17B681B6803F00803002B38D07B68C9
:10BC40005B69002B19D0164B5B6F154A43F001035B
:10BC50005367FCF77DFC386108E0FCF779FC02468D
:10BC60003B69D31A022B01D9032376E10C4B5B6F9E
:10BC700003F00203002BF0D01AE0094B5B6F084A77
:10BC800023F001035367FCF763FC38610AE0FCF71B
:10BC90005FFC02463B69D31A022B03D903235CE104
:10BCA00000380240914B5B6F03F00203002BEED192
:10BCB0007B681B6803F00403002B00F0A4808B4B0F
:10BCC0001B6C03F08053002B0DD1884B1B6C874AF3
:10BCD00043F080531364854B1B6C03F08053BB60AF
:10BCE000BB680123FB75824B1B6803F48073002B38
:10BCF00018D17F4B1B687E4A43F480731360FCF7B6
:10BD000027FC386108E0FCF723FC02463B69D31AA4
:10BD1000642B01D9032320E1754B1B6803F4807366
:10BD2000002BF0D07B689B68012B06D16F4B1B6FFB
:10BD30006E4A43F0010313672DE07B689B68002B7C
:10BD40000CD16A4B1B6F694A23F001031367674BE1
:10BD50001B6F664A23F0040313671CE07B689B6833
:10BD6000052B0CD1614B1B6F604A43F00403136732
:10BD70005E4B1B6F5D4A43F0010313670BE05B4BA7
:10BD80001B6F5A4A23F001031367584B1B6F574A26
:10BD900023F0040313677B689B68002B15D0FCF726
:10BDA000D7FB38610AE0FCF7D3FB02463B69D31AA4
:10BDB00041F28832934201D90323CEE04B4B1B6FF3
:10BDC00003F00203002BEED014E0FCF7C1FB386156
:10BDD0000AE0FCF7BDFB02463B69D31A41F2883208
:10BDE000934201D90323B8E0404B1B6F03F00203D9
:10BDF000002BEED1FB7D012B05D13C4B1B6C3B4A4C
:10BE000023F0805313647B689B69002B00F0A480AF
:10BE1000364B9B6803F00C03082B6BD07B689B6947
:10BE2000022B49D1314B1B68304A23F080731360D9
:10BE3000FCF78EFB386108E0FCF78AFB02463B69A1
:10BE4000D31A022B01D9032387E0284B1B6803F088
:10BE50000073002BF0D17B68DA697B681B6A1A4398
:10BE60007B685B6A9B011A437B689B6A5B08013BAA
:10BE70001B041A437B68DB6A1B0613431B4A43F00F
:10BE800000535360194B1B68184A43F080731360CA
:10BE9000FCF75EFB386108E0FCF75AFB02463B69A1
:10BEA000D31A022B01D9032357E0104B1B6803F070
:10BEB0000073002BF0D04FE00C4B1B680B4A23F0B3
:10BEC00080731360FCF744FB386108E0FCF740FB2B
:10BED00002463B69D31A022B01D903233DE0034BF1
:10BEE0001B6803F00073002BF0D135E000380240EE
:10BEF000007000401B4B5B68FB607B689B69012BFB
:10BF000028D0FB6803F480027B68DB699A4221D168
:10BF1000FB6803F03F027B681B6A9A421AD1FA68F9
:10BF200047F6C07313407A68526A9201934211D166
:10BF3000FB6803F440327B689B6A5B08013B1B048F
:10BF40009A4207D1FB6803F070627B68DB6A1B06CC
:10BF50009A4201D0012300E0002318461837BD465D
:10BF600080BD00BF0038024080B584B000AF78606B
:10BF700039600023FB607B68002B01D10123D0E0F6
:10BF80006A4B1B6803F00F033A689A4210D9674B5B
:10BF90001B6823F00F0265493B6813430B60634B3A
:10BFA0001B6803F00F033A689A4201D00123B8E0FE
:10BFB0007B681B6803F00203002B20D07B681B68A2
:10BFC00003F00403002B05D0594B9B68584A43F4F7
:10BFD000E05393607B681B6803F00803002B05D0D7
:10BFE000534B9B68524A43F460439360504B9B68A9
:10BFF00023F0F0027B689B684D4913438B607B689C
:10C000001B6803F00103002B40D07B685B68012BA9
:10C0100007D1474B1B6803F40033002B15D10123D4
:10C020007FE07B685B68022B07D1414B1B6803F004
:10C030000073002B09D1012373E03D4B1B6803F013
:10C040000203002B01D101236BE0394B9B6823F0E5
:10C0500003027B685B68364913438B60FCF778FA10
:10C06000F8600AE0FCF774FA0246FB68D31A41F262
:10C070008832934201D9032353E02D4B9B6803F090
:10C080000C027B685B689B009A42EBD1274B1B68D4
:10C0900003F00F033A689A4210D2244B1B6823F036
:10C0A0000F0222493B6813430B60204B1B6803F0CF
:10C0B0000F033A689A4201D0012332E07B681B6883
:10C0C00003F00403002B08D0194B9B6823F4E052C3
:10C0D0007B68DB68164913438B607B681B6803F041
:10C0E0000803002B09D0124B9B6823F460427B6845
:10C0F0001B69DB000E4913438B6000F021F80246F8
:10C100000B4B9B681B0903F00F030A49CB5C22FA17
:10C1100003F3094A1360094B1B681846F6F78AFFB8
:10C12000002318461037BD4680BD00BF003C0240CA
:10C1300000380240E0E00208240000205000002007
:10C14000B0B584B000AF002179600021F960002112
:10C1500039600021B9605249896801F00C01082951
:10C160000DD0082900F29480002902D0042903D0C0
:10C170008EE04C4BBB608EE04B4BBB608BE0484984
:10C18000496801F03F0179604549496801F480013F
:10C19000002924D042494968890908464FF0000126
:10C1A00040F2FF144FF0000500EA040201EA050323
:10C1B0003D4901FB03F0002101FB02F144183A491B
:10C1C000A2FB0101631819467B681A464FF0000371
:10C1D000F4F776F802460B461346FB604AE0304B14
:10C1E0005B689B091A464FF0000340F2FF104FF0C6
:10C1F000000102EA000403EA0105204629464FF047
:10C2000000024FF000034B0143EAD06342011046A5
:10C210001946001B61EB05014FF000024FF00003CF
:10C220008B0143EA90638201121A63EB01034FF022
:10C2300000004FF00001D90041EA5271D0000246DF
:10C240000B46121945EB03034FF000004FF00001BD
:10C25000990241EA9251900202460B461046194655
:10C260007B681A464FF00003F4F72AF802460B46A3
:10C270001346FB600A4B5B681B0C03F0030301339E
:10C280005B003B60FA683B68B2FBF3F3BB6002E023
:10C29000044BBB6000BFBB6818461037BD46B0BD3D
:10C2A000003802400024F40040787D0180B400AFE3
:10C2B000034B1B681846BD465DF8047B704700BF02
:10C2C0002400002080B500AFFFF7F0FF0246054BC9
:10C2D0009B689B0A03F007030349CB5C22FA03F334
:10C2E000184680BD00380240F0E0020880B483B0F8
:10C2F00000AF786039607B680F221A60124B9B6830
:10C3000003F003027B685A600F4B9B6803F0F00256
:10C310007B689A600C4B9B6803F4E0527B68DA60A0
:10C32000094B9B68DB0803F4E0527B681A61074BFA
:10C330001B6803F00F023B681A6000BF0C37BD4654
:10C340005DF8047B704700BF00380240003C0240AB
:10C3500080B588B000AF786000237B6100233B612B
:10C360000023FB600023FB610023BB617B681B682B
:10C3700003F00103002B12D0694B9B68684A23F439
:10C3800000039360664B9A687B685B6B6449134358
:10C390008B607B685B6B002B01D10123FB617B68A9
:10C3A0001B6803F40023002B17D05D4BD3F88C30AF
:10C3B00023F440127B68DB6B59491343C1F88C307E
:10C3C0007B68DB6BB3F5801F01D10123FB617B68C8
:10C3D000DB6B002B01D10123BB617B681B6803F47D
:10C3E0008013002B17D04E4BD3F88C3023F440022F
:10C3F0007B681B6C4A491343C1F88C307B681B6C0B
:10C40000B3F5800F01D10123FB617B681B6C002B0E
:10C4100001D10123BB617B681B6803F08073002B93
:10C4200001D00123FB617B681B6803F02003002B14
:10C4300000F08B803A4B1B6C394A43F080531364F5
:10C44000374B1B6C03F08053BB60BB68354B1B68DC
:10C45000344A43F480731360FCF77AF8786108E09B
:10C46000FCF776F802467B69D31A642B01D90323C3
:10C4700057E32C4B1B6803F48073002BF0D0284B40
:10C480001B6F03F440733B613B69002B35D07B6825
:10C490001B6B03F440733A699A422ED0204B1B6FFA
:10C4A00023F440733B611E4B1B6F1D4A43F48033E2
:10C4B00013671B4B1B6F1A4A23F480331367184A08
:10C4C0003B691367164B1B6F03F00103012B14D15B
:10C4D000FCF73EF878610AE0FCF73AF802467B691F
:10C4E000D31A41F28832934201D9032319E30C4B4A
:10C4F0001B6F03F00203002BEED07B681B6B03F471
:10C500004073B3F5407F11D1054B9B6823F4F812BB
:10C510007B68196B044B0B40014913438B600BE0A4
:10C520000038024000700040FFFCFF0FB14B9B68D9
:10C53000B04A23F4F8139360AE4B1A6F7B681B6B01
:10C54000C3F30B03AB4913430B677B681B6803F012
:10C550001003002B10D0A74BD3F88C30A54A23F042
:10C560008073C2F88C30A34BD3F88C207B689B6B14
:10C57000A0491343C1F88C307B681B6803F48043E7
:10C58000002B0AD09B4BD3F8903023F440327B68C9
:10C590005B6E98491343C1F890307B681B6803F4C5
:10C5A0000043002B0AD0934BD3F8903023F4402261
:10C5B0007B689B6E8F491343C1F890307B681B6882
:10C5C00003F48033002B0AD08A4BD3F8903023F445
:10C5D00040127B68DB6E87491343C1F890307B685B
:10C5E0001B6803F40033002B0AD0824BD3F8903041
:10C5F00023F440027B681B6F7E491343C1F89030DF
:10C600007B681B6803F04003002B0AD0794BD3F8FA
:10C61000903023F003027B685B6C76491343C1F8CA
:10C6200090307B681B6803F08003002B0AD0714BAD
:10C63000D3F8903023F00C027B689B6C6D49134358
:10C64000C1F890307B681B6803F48073002B0AD01C
:10C65000684BD3F8903023F030027B68DB6C65497F
:10C660001343C1F890307B681B6803F40073002B00
:10C670000AD0604BD3F8903023F0C0027B681B6D6A
:10C680005C491343C1F890307B681B6803F48063F6
:10C69000002B0AD0574BD3F8903023F440727B68BC
:10C6A0005B6D54491343C1F890307B681B6803F4F9
:10C6B0000063002B0AD04F4BD3F8903023F4406234
:10C6C0007B689B6D4B491343C1F890307B681B68B6
:10C6D00003F48053002B0AD0464BD3F8903023F458
:10C6E00040527B68DB6D43491343C1F890307B684F
:10C6F0001B6803F40053002B0AD03E4BD3F8903054
:10C7000023F440427B681B6E3A491343C1F89030D2
:10C710007B681B6803F48003002B0AD0354BD3F8E9
:10C72000903023F080627B689B6F32491343C1F8DD
:10C7300090307B681B6803F40013002B11D02D4B45
:10C74000D3F8903023F000627B68DB6F29491343F4
:10C75000C1F890307B68DB6FB3F1006F01D101232A
:10C76000BB617B681B6803F00803002B01D0012329
:10C77000BB617B681B6803F48023002B0AD01D4B30
:10C78000D3F8903023F040727B685B6F19491343F4
:10C79000C1F890307B681B6803F40003002B0BD0BA
:10C7A000144BD3F8903023F080527B68D3F880305C
:10C7B00010491343C1F89030FB69012B06D07B6808
:10C7C0001B6803F00073002B00F0D980094B1B6835
:10C7D000084A23F080631360FBF7BAFE78610BE030
:10C7E000FBF7B6FE02467B69D31A642B04D90323F8
:10C7F00097E100BF003802406C4B1B6803F00063F8
:10C80000002BEDD17B681B6803F00103002B21D0C6
:10C810007B685B6B002B1DD1644BD3F884301B0C01
:10C8200003F003033B61614BD3F884301B0E03F02C
:10C830000F03FB607B685B689A013B691B041A432A
:10C84000FB681B061A437B689B681B075749134309
:10C85000C1F884307B681B6803F40023002B04D0EC
:10C860007B68DB6BB3F5801F0AD07B681B6803F421
:10C870008013002B2ED07B681B6CB3F5800F29D161
:10C880004A4BD3F884301B0C03F003033B61474B46
:10C89000D3F884301B0F03F00703FB607B685B68F1
:10C8A0009A013B691B041A437B68DB681B061A4329
:10C8B000FB681B073D491343C1F884303B4BD3F859
:10C8C0008C3023F01F027B685B6A013B37491343BE
:10C8D000C1F88C307B681B6803F08073002B1DD07F
:10C8E000324BD3F884301B0E03F00F033B612F4B08
:10C8F000D3F884301B0F03F00703FB607B685B6891
:10C900009A017B681B691B041A433B691B061A4387
:10C91000FB681B0725491343C1F884307B681B68FB
:10C9200003F00073002B11D07B685B689A017B6871
:10C930001B691B041A437B68DB681B061A437B6870
:10C940009B681B0719491343C1F88430174B1B68B8
:10C95000164A43F080631360FBF7FAFD786108E044
:10C96000FBF7F6FD02467B69D31A642B01D903233A
:10C97000D7E00E4B1B6803F00063002BF0D0BB69BF
:10C98000012B40F0CD80094B1B68084A23F08053EF
:10C990001360FBF7DDFD78610AE0FBF7D9FD024685
:10C9A0007B69D31A642B03D90323BAE00038024011
:10C9B0005E4B1B6803F00053B3F1005FEDD07B6862
:10C9C0001B6803F40023002B03D07B68DB6B002B78
:10C9D00009D07B681B6803F48013002B2ED07B6882
:10C9E0001B6C002B2AD1514BD3F888301B0C03F061
:10C9F00003033B614D4BD3F888301B0F03F0070353
:10CA0000FB607B685B699A013B691B041A437B6886
:10CA10009B691B061A43FB681B0744491343C1F873
:10CA20008830424BD3F88C3023F4F8527B689B6AF1
:10CA3000013B1B023D491343C1F88C307B681B68E6
:10CA400003F40013002B22D07B68DB6FB3F1006F7F
:10CA50001DD1364BD3F888301B0E03F00F033B611A
:10CA6000324BD3F888301B0F03F00703FB607B6861
:10CA70005B699A017B681B6A1B041A433B691B06AE
:10CA80001A43FB681B0729491343C1F888307B68A8
:10CA90001B6803F00803002B28D0244BD3F8883000
:10CAA0001B0E03F00F033B61204BD3F888301B0CA7
:10CAB00003F00303FB607B685B699A01FB681B045E
:10CAC0001A433B691B061A437B68DB691B0717493E
:10CAD0001343C1F88830154BD3F88C3023F440321F
:10CAE0007B68DB6A11491343C1F88C300F4B1B681C
:10CAF0000E4A43F080531360FBF72AFD786108E08B
:10CB0000FBF726FD02467B69D31A642B01D9032368
:10CB100007E0064B1B6803F00053B3F1005FEFD151
:10CB2000002318462037BD4680BD00BF00380240B4
:10CB300080B582B000AF78607B68002B01D1012303
:10CB400022E07B6893F83430DBB2002B05D17B68A0
:10CB500000221A777868F6F79DF87B68032283F83D
:10CB60003420786800F014F80346002B01D001232C
:10CB70000AE07B6800229A637B6800221A637B6864
:10CB8000012283F83420002318460837BD4680BDB3
:10CB9000B0B58EB004AF78600023BB600023FB60AB
:10CBA00000233B6100237B610023BB617623FB6193
:10CBB0007B681D686C4607F1140393E8070084E85E
:10CBC000070007F108030ECB284602F019FB0346C5
:10CBD00087F8273097F82730002B01D0012356E043
:10CBE0007B681B685A687B681B6822F480725A60F5
:10CBF0007B681B68184602F04DFB7B681B685A680F
:10CC00007B681B6842F480725A60786800F0F2FF1B
:10CC100038623B6A002B0BD07B68012283F83420FA
:10CC20007B689A6B3B6A1A437B689A6301232EE008
:10CC3000786800F013FF38623B6A002B0BD07B68EA
:10CC4000012283F834207B689A6B3B6A1A437B6825
:10CC50009A6301231BE07B681B684FF40071184640
:10CC600002F0ACFB38623B6A002B0FD07B681B687C
:10CC7000094A9A637B689A6B3B6A1A437B689A639A
:10CC80007B68012283F83420012300E0002318464A
:10CC90002837BD46B0BD00BFFF05400080B58CB051
:10CCA00000AFF860B9607A603B607B68BB62BB68CC
:10CCB000002B07D1FB689B6B43F00062FB689A6313
:10CCC0000123C3E0FB6893F83430DBB2012B40F062
:10CCD000BC80FB6800229A63BA6A3B681A44FB680E
:10CCE000DB6D9A4207D9FB689B6B43F00072FB68CF
:10CCF0009A630123AAE0FB68032283F83420FB68CF
:10CD00001B680022DA62FB681B68DA6BFB681B6831
:10CD100042F49572DA63FB681B6C4E4ADA63FB6877
:10CD20001B6C4D4ADA64FB681B6C00221A65FB68B9
:10CD30001B6C00229A60FB681B6C1B681B6823F04D
:10CD4000C001FB681B6C9A68FB681B6C1B680A437C
:10CD50001A60FB68186CFB681B6880331946BA6858
:10CD60003B685B029B08FBF74BFF0346002B17D089
:10CD7000FB681B68DA6BFB681B6822F49572DA6348
:10CD8000FB681B68354A9A63FB689B6B43F08042E3
:10CD9000FB689A63FB68012283F83420012355E085
:10CDA000FB681B68DA6AFB681B6842F00802DA62FB
:10CDB000FB685B6C012B02D0BB6A5B02BB624FF06D
:10CDC000FF333B613B685B027B619023BB610223C5
:10CDD000FB6100233B6201237B62FB681B6807F158
:10CDE00010021146184602F0BDFA3B68012B0AD921
:10CDF000FB6882221A63FB681B68B96A184602F056
:10CE000021FBF86209E0FB6881221A63FB681B685A
:10CE1000B96A184602F0F4FAF862FB6A002B12D0E5
:10CE2000FB681B680D4A9A63FB689A6BFB6A1A439E
:10CE3000FB689A63FB68012283F83420FB680022B8
:10CE40001A63012302E0002300E002231846303772
:10CE5000BD4680BD6BD80008DDD80008FF05400046
:10CE600080B58CB000AFF860B9607A603B607B68D9
:10CE7000BB62BB68002B07D1FB689B6B43F0006271
:10CE8000FB689A630123C6E0FB6893F83430DBB299
:10CE9000012B40F0BF80FB6800229A63BA6A3B68AE
:10CEA0001A44FB68DB6D9A4207D9FB689B6B43F021
:10CEB0000072FB689A630123ADE0FB68032283F8EC
:10CEC0003420FB681B680022DA62FB681B68DA6B9F
:10CED000FB681B6842F01A02DA63FB68DB6B504A9E
:10CEE000DA63FB68DB6B4F4ADA64FB68DB6B0022BA
:10CEF0001A65FB685B6C012B02D0BB6A5B02BB62EC
:10CF00003B68012B0AD9FB68A0221A63FB681B68E7
:10CF1000B96A184602F0DAFAF86209E0FB68902272
:10CF20001A63FB681B68B96A184602F0ADFAF8622A
:10CF3000FB6A002B12D0FB681B683B4A9A63FB68B4
:10CF40009A6BFB6A1A43FB689A63FB68012283F8B9
:10CF50003420FB6800221A6301235CE0FB681B6835
:10CF6000DA6AFB681B6842F00802DA62FB68DB6B76
:10CF700040229A60FB68DB6B1B681B6823F0C001D2
:10CF8000FB68DB6B9A68FB68DB6B1B680A431A6003
:10CF9000FB68D86BB968FB681B6880331A463B682E
:10CFA0005B029B08FBF72CFE0346002B1AD0FB68A4
:10CFB0001B68DA6BFB681B6822F01A02DA63FB68F5
:10CFC0001B68194A9A63FB689B6B43F08042FB68BD
:10CFD0009A63FB68012283F83420FB6800221A63FD
:10CFE000012318E04FF0FF333B613B685B027B613C
:10CFF0009023BB610023FB6100233B6201237B6222
:10D00000FB681B6807F110021146184602F0AAF9E6
:10D01000002300E0022318463037BD4680BD00BF24
:10D0200041D80008DDD80008FF05400080B584B075
:10D0300000AF78607B681B6BFB607B681B685B6B79
:10D0400003F40043002B08D0FB6803F00803002B17
:10D0500003D0786800F0EDFF53E17B681B685B6BE1
:10D0600003F48073002B00F08D807B681B684FF405
:10D0700080729A637B681B68D96B7B681A68A34BC4
:10D080000B40D3637B681B68DA6A7B681B6822F0FD
:10D090000102DA62FB6803F00803002B39D0FB6859
:10D0A00003F00203002B04D1FB6803F02003002BE4
:10D0B00011D07B681B68184602F02AFAB860BB687A
:10D0C000002B08D07B689A6BBB681A437B689A6315
:10D0D000786800F021F97B681B6840F23A529A6345
:10D0E0007B68012283F834207B6800221A63FB6886
:10D0F00003F00103002B04D1FB6803F00203002BB3
:10D1000003D07868F6F7B8F9FBE07868F6F7AAF983
:10D11000F7E0FB6803F08003002B00F0F280FB686F
:10D1200003F02003002B11D07B681B68184602F027
:10D13000EFF9B860BB68002B08D07B689A6BBB68BE
:10D140001A437B689A63786800F0E6F8FB6803F09E
:10D150000103002B40F0D580FB6803F00203002B95
:10D1600040F0CF807B681B68DA6A7B681B6822F01E
:10D170000802DA627B68012283F834207868F6F7C7
:10D1800071F9BEE07B681B685B6B03F48043002B86
:10D1900008D0FB6803F00803002B03D0786800F088
:10D1A00099FFAEE07B681B685B6B03F03A03002BD2
:10D1B00000F0A7807B681B685B6B03F00203002B09
:10D1C00005D07B689B6B43F002027B689A637B68A7
:10D1D0001B685B6B03F00803002B05D07B689B6B1F
:10D1E00043F008027B689A637B681B685B6B03F003
:10D1F0002003002B05D07B689B6B43F020027B68EB
:10D200009A637B681B685B6B03F01003002B05D0EF
:10D210007B689B6B43F010027B689A637B681B689A
:10D2200040F23A529A637B681B68DA6B7B681B6832
:10D2300022F49D72DA637B681B68184602F068F975
:10D2400002467B689B6B1A437B689A63FB6803F01A
:10D250000803002B0AD07B68012283F834207B6806
:10D2600000221A63786800F057F84AE0FB6803F080
:10D270008003002B45D0FB6803F01003002B04D182
:10D28000FB6803F02003002B11D07B68DB6B204A86
:10D290001A657B68DB6B1846FBF782FD0346002BA3
:10D2A0002FD07B68DB6B184600F06AFB29E0FB6837
:10D2B00003F00103002B04D1FB6803F00203002BF1
:10D2C00011D07B681B6C134A1A657B681B6C18466F
:10D2D000FBF766FD0346002B13D07B681B6C1846DA
:10D2E00000F085FB0DE07B6800229A637B680122D9
:10D2F00083F834207B6800221A637868F6F7A8F870
:10D30000FFE700BF1037BD4680BD00BFC53EFFFF31
:10D3100081D90008EFD9000880B483B000AF7860ED
:10D3200000BF0C37BD465DF8047B704780B483B006
:10D3300000AF786039607B685B6E9B0FDAB23B6848
:10D340001A707B685B6E9B0EDBB203F00F03DAB2E0
:10D350003B685A707B685B6E1B0EDBB203F0030305
:10D36000DAB23B689A707B685B6E1B0CDAB23B6882
:10D37000DA707B685B6E1B0ADAB23B681A717B68F5
:10D380005B6EDAB23B685A717B689B6E1B0D9AB27A
:10D390003B68DA807B689B6E1B0CDBB203F00F03EB
:10D3A000DAB23B681A727B689B6EDB0BDBB203F070
:10D3B0000103DAB23B685A727B689B6E9B0BDBB24F
:10D3C00003F00103DAB23B689A727B689B6E5B0BD9
:10D3D000DBB203F00103DAB23B68DA727B689B6E62
:10D3E0001B0BDBB203F00103DAB23B681A733B6834
:10D3F00000225A737B685B6C002B63D17B689B6E49
:10D400009A0040F6FC7313407A68D26E920F1A436A
:10D410003B681A617B68DB6EDB0EDBB203F007034F
:10D42000DAB23B681A757B68DB6E1B0EDBB203F069
:10D430000703DAB23B685A757B68DB6E5B0DDBB2C3
:10D4400003F00703DAB23B689A757B68DB6E9B0CCE
:10D45000DBB203F00703DAB23B68DA757B68DB6E98
:10D46000DB0BDBB203F00703DAB23B681A763B68EA
:10D470001B695A1C7B685A653B681B7EDBB203F054
:10D4800007030233012202FA03F37A68526D02FBAA
:10D4900003F27B685A653B681B7ADBB203F00F032B
:10D4A00001229A407B689A657B685B6D7A68926D11
:10D4B000520A02FB03F27B68DA657B684FF4007264
:10D4C0001A6631E07B685B6C012B1DD17B689B6E1B
:10D4D0001B0403F47C127B68DB6E1B0C1A433B6855
:10D4E0001A613B681B6901339A027B685A657B6845
:10D4F0005A6D7B68DA657B684FF400729A657B68C9
:10D500009A6D7B681A660FE07B681B68584A9A63BD
:10D510007B689B6B43F080527B689A637B68012237
:10D5200083F8342001239DE07B68DB6E9B0BDBB22C
:10D5300003F00103DAB23B685A767B68DB6EDB09E5
:10D54000DBB203F07F03DAB23B689A767B68DB6E6E
:10D55000DBB203F07F03DAB23B68DA767B681B6FDD
:10D56000DB0FDAB23B681A777B681B6F5B0FDBB2AD
:10D5700003F00303DAB23B685A777B681B6F9B0E9C
:10D58000DBB203F00703DAB23B689A777B681B6F64
:10D590009B0DDBB203F00F03DAB23B68DA777B68EE
:10D5A0001B6F5B0DDBB203F00103DAB23B6883F85B
:10D5B00020203B68002283F821207B681B6F1B0C16
:10D5C000DBB203F00103DAB23B6883F822207B6808
:10D5D0001B6FDB0BDBB203F00103DAB23B6883F8AD
:10D5E00023207B681B6F9B0BDBB203F00103DAB2D5
:10D5F0003B6883F824207B681B6F5B0BDBB203F076
:10D600000103DAB23B6883F825207B681B6F1B0B94
:10D61000DBB203F00103DAB23B6883F826207B68B3
:10D620001B6F9B0ADBB203F00303DAB23B6883F89B
:10D6300027207B681B6F1B0ADBB203F00303DAB2FF
:10D640003B6883F828207B681B6F5B08DBB203F024
:10D650007F03DAB23B6883F829203B68012283F814
:10D660002A20002318460C37BD465DF8047B70471E
:10D67000FF05400080B483B000AF786039607B68FC
:10D680005A6C3B681A607B689A6C3B685A607B688E
:10D69000DA6C3B689A607B681A6D3B68DA607B687D
:10D6A0005A6D3B681A617B689A6D3B685A617B686A
:10D6B000DA6D3B689A617B681A6E3B68DA61002319
:10D6C00018460C37BD465DF8047B7047B0B58EB088
:10D6D00004AF78603960002387F827307B68032225
:10D6E00083F834207B685B6C032B2ED03B68B3F54A
:10D6F000805F06D17B689B6B43F080527B689A63A6
:10D7000029E03B68B3F5006F0AD1786800F028FB88
:10D7100038627B689A6B3B6A1A437B689A631AE0AB
:10D720003B68002B0AD1786800F065FB38627B68A3
:10D730009A6B3B6A1A437B689A630CE07B689B6B2D
:10D7400043F000627B689A6305E07B689B6B43F063
:10D7500080527B689A637B689B6B002B0BD07B6845
:10D760001B68264A9A637B68012283F834200123D0
:10D7700087F827301FE07B685B68BB607B689B682D
:10D78000FB607B68DB683B613B687B617B685B6956
:10D79000BB617B689B69FB617B681D686C4607F118
:10D7A000140393E8070084E8070007F108030ECB91
:10D7B000284601F025FD7B681B684FF40071184670
:10D7C00001F0FCFD38623B6A002B0CD07B681B68C3
:10D7D0000A4A9A637B689A6B3B6A1A437B689A632E
:10D7E000012387F827307B68012283F8342097F8DB
:10D7F000273018462837BD46B0BD00BFFF054000A2
:10D8000080B586B000AF78600023FB6007F10C03A1
:10D810001946786800F07CFA78617B69002B05D0A6
:10D820007B689A6B7B691A437B689A63FB685B0A27
:10D8300003F00F033B613B6918461837BD4680BDB6
:10D8400080B485B000AF78607B689B6BFB60FB6841
:10D850001B68DA6BFB681B6842F48072DA6300BFF6
:10D860001437BD465DF8047B704780B584B000AFC7
:10D8700078607B689B6BFB60FB681B6B822B11D114
:10D88000FB681B68184601F043FEB860BB68002BBC
:10D8900008D0FB689A6BBB681A43FB689A63F86808
:10D8A000FFF73AFDFB681B68DA6AFB681B6822F029
:10D8B0000802DA62FB681B6840F23A529A63FB681E
:10D8C000012283F83420FB6800221A63F868F5F718
:10D8D000D3FD00BF1037BD4680BD000080B586B0C7
:10D8E00000AF78607B689B6B7B617868FBF704FC1A
:10D8F0000346022B3ED07B691B6C5B6D3B617B69F1
:10D90000DB6B5B6DFB603B69012B02D0FB68012B7D
:10D910002DD17B691B68194A9A637B691B68DA6B96
:10D920007B691B6822F49D72DA637B699B6B43F011
:10D9300080427B699A637869FFF762FFB860BB68D1
:10D94000062B02D0BB68052B0AD17B691B681846E1
:10D9500001F0DEFD02467B699B6B1A437B699A638B
:10D960007B69012283F834207B6900221A6378697D
:10D97000FFF7D2FC00BF1837BD4680BDFF05400051
:10D9800080B584B000AF78607B689B6BFB60FB6800
:10D990001B6840F23A529A63F868FFF731FFB860AB
:10D9A000FB68012283F83420FB6800221A63BB68FD
:10D9B000062B02D0BB68052B0AD1FB681B681846F2
:10D9C00001F0A6FD0246FB689B6B1A43FB689A6355
:10D9D000FB689B6B002B03D1F868F5F739FD02E07B
:10D9E000F868FFF799FC00BF1037BD4680BD80B5D1
:10D9F00084B000AF78607B689B6BFB60FB681B6842
:10DA000040F23A529A63F868FFF7FAFEB860FB6892
:10DA1000012283F83420FB6800221A63BB68062BBE
:10DA200002D0BB68052B0AD1FB681B68184601F0C1
:10DA30006FFD0246FB689B6B1A43FB689A63FB68A9
:10DA40009B6B002B03D1F868F5F702FD02E0F86844
:10DA5000FFF762FC00BF1037BD4680BDB0B594B083
:10DA600004AF78600123FB817B681B68184601F0D6
:10DA700020FC0346002B02D14FF08063B6E07B68A8
:10DA80005B6C032B2FD07B681B68184601F04BFEA4
:10DA9000F863FB6B002B01D0FB6BA7E07B681B6876
:10DAA0000021184601F04BFC02467B685A677B68F0
:10DAB0001B680421184601F042FC02467B689A6705
:10DAC0007B681B680821184601F039FC02467B6818
:10DAD000DA677B681B680C21184601F030FC0246AF
:10DAE0007B68C3F880207B685B6C032B0DD07B6860
:10DAF0001B6807F10E021146184601F051FEF8634B
:10DB0000FB6B002B01D0FB6B70E07B685B6C032B25
:10DB100036D0FB891A467B681A657B681A687B6871
:10DB20001B6D1B041946104601F01BFEF863FB6BCE
:10DB3000002B01D0FB6B59E07B681B680021184665
:10DB400001F0FDFB02467B685A667B681B68042176
:10DB5000184601F0F4FB02467B689A667B681B68F6
:10DB60000821184601F0EBFB02467B68DA667B6809
:10DB70001B680C21184601F0E2FB02467B681A671D
:10DB80007B681B680421184601F0D9FB03461A0D77
:10DB90007B68DA6407F1100319467868FFF7C6FB63
:10DBA0000346002B02D04FF080531FE07B681968BA
:10DBB0007B681B6D1B041A464FF00003084601F0FA
:10DBC000C9FCF863FB6B002B01D0FB6B0EE07B689C
:10DBD0001D687B686C4603F1100207CA84E80700E1
:10DBE00004330ECB284601F00BFB002318464037C8
:10DBF000BD46B0BD80B586B000AF78600023BB6085
:10DC000000237B6100233B617B681B68184601F0A1
:10DC1000C4FCF860FB68002B01D0FB6872E07B68F5
:10DC20001B68184601F0D7FCF860FB68002B0DD08C
:10DC30007B6800229A647B681B68184601F0ADFC83
:10DC4000F860FB68002B04D0FB685BE07B68012276
:10DC50009A647B689B6C012B37D17B681B68002121
:10DC6000184601F0D7FCF860FB68002B2DD04FF070
:10DC7000805347E07B681B680021184601F0CAFC0E
:10DC8000F860FB68002B01D0FB683BE07B681B68F9
:10DC90001E49184601F0E0FCF860FB68002B02D03A
:10DCA0004FF080532EE07B681B680021184601F07E
:10DCB00046FB78617B69DB0F012B01D1012300E07A
:10DCC00000233B61BB680133BB60BB684FF6FE724B
:10DCD000934202D83B69002BCCD0BB684FF6FE7252
:10DCE000934202D94FF080730CE07B6903F08043CC
:10DCF000002B03D07B6801225A6402E07B6800227B
:10DD00005A64002318461837BD4680BD000010C174
:10DD100080B584B000AF786039603B68002B02D1D9
:10DD20004FF0006318E07B681A687B681B6D1B046A
:10DD30001946104601F055FDF860FB68002B01D034
:10DD4000FB6809E07B681B680021184601F0F7FAC0
:10DD500002463B681A60002318461037BD4680BD56
:10DD600080B586B000AF78600023FB6000233B6184
:10DD70007B681B680021184601F0E1FA034603F0B6
:10DD80000073B3F1007F02D14FF400632FE007F17D
:10DD90000C031946786800F079F878617B69002BEC
:10DDA00001D07B6923E03B6903F48023002B1CD066
:10DDB0007B681A687B681B6D1B041946104601F0CE
:10DDC00029FC78617B69002B01D07B690FE07B68BF
:10DDD0001B680221184601F063FC78617B69002B07
:10DDE00001D07B6903E0002301E04FF08063184617
:10DDF0001837BD4680BD80B586B000AF786000237F
:10DE0000FB6000233B617B681B680021184601F022
:10DE100096FA034603F00073B3F1007F02D14FF48A
:10DE200000632FE007F10C031946786800F02EF824
:10DE300078617B69002B01D07B6923E03B6903F4A7
:10DE40008033002B1CD07B681A687B681B6D1B0419
:10DE50001946104601F0DEFB78617B69002B01D08A
:10DE60007B690FE07B681B680021184601F018FCF5
:10DE700078617B69002B01D07B6903E0002301E01E
:10DE80004FF0806318461837BD4680BD90B58FB0FF
:10DE900000AF78603960FAF75BFB386300237B637F
:10DEA0000023BB600023FB603B68FB627B681B6850
:10DEB0000821184601F082FAB862BB6A002B01D033
:10DEC000BB6AB2E07B681A687B681B6D1B0419464D
:10DED000104601F09FFBB862BB6A002B01D0BB6A01
:10DEE000A3E04FF0FF333B6108237B613023BB612C
:10DEF0000223FB6100233B6201237B627B681B687A
:10DF000007F110021146184601F02CFA7B681B68D5
:10DF1000184601F0E7FBB862BB6A002B2AD0BB6A47
:10DF200083E07B681B685B6B03F40013002B0FD04E
:10DF30007B6819687B6B9B0007F10802D4180846C0
:10DF400001F08AF9034623607B6B01337B6306E0B3
:10DF50007B681B685B6B03F40053002B12D0FAF74D
:10DF6000F7FA02463B6BD31AB3F1FF3F02D14FF0F1
:10DF700000435AE07B681B685B6B03F02A03002BAD
:10DF8000CFD000E000BF7B681B685B6B03F0080329
:10DF9000002B05D07B681B6808229A63082344E0A5
:10DFA0007B681B685B6B03F00203002B05D07B686A
:10DFB0001B6802229A63022337E07B681B685B6B55
:10DFC00003F02003002B05D07B681B6820229A6396
:10DFD00020232AE07B681B6840F23A529A63FB6870
:10DFE0001A06FB681B0203F47F031A43FB681B0A33
:10DFF00003F47F431A43FB681B0E1A43FB6A1A6043
:10E00000FB6A0433FB62BB681A06BB681B0203F49D
:10E010007F031A43BB681B0A03F47F431A43BB68A0
:10E020001B0E1A43FB6A1A60002318463C37BD4694
:10E0300090BD80B586B000AF78607B689B6AFB605E
:10E040007B68DB6A3B613B69002B3FD000237B612F
:10E0500033E07B681B68184601F0FEF8B860BB68C7
:10E06000DAB2FB681A70FB680133FB603B69013B65
:10E070003B61BB681B0ADAB2FB681A70FB680133AC
:10E08000FB603B69013B3B61BB681B0CDAB2FB6880
:10E090001A70FB680133FB603B69013B3B61BB6865
:10E0A0001B0EDAB2FB681A70FB680133FB603B6938
:10E0B000013B3B617B6901337B617B69072BC8D9DD
:10E0C0007B68FA689A627B683A69DA6200BF18373F
:10E0D000BD4680BD80B586B000AF78607B681B6AA6
:10E0E000FB607B685B6A3B613B69002B43D000238C
:10E0F0007B6137E0FB681B78BB60FB680133FB602A
:10E100003B69013B3B61FB681B781A02BB68134308
:10E11000BB60FB680133FB603B69013B3B61FB6813
:10E120001B781A04BB681343BB60FB680133FB60B8
:10E130003B69013B3B61FB681B781A06BB681343D4
:10E14000BB60FB680133FB603B69013B3B617B6863
:10E150001B6807F108021146184601F08AF87B692E
:10E1600001337B617B69072BC4D97B68FA681A622B
:10E170007B683A695A6200BF1837BD4680BD80B5DA
:10E1800082B000AF786039607B68002B01D1012339
:10E1900025E07B6893F82C30DBB2002B06D17B683E
:10E1A000002283F82D207868F4F73AFF7B6802227A
:10E1B00083F82C207B681A687B6804331946104664
:10E1C00000F0F4FE7B6818687B685B681A46396863
:10E1D00000F05EFF7B68012283F82C2000231846A4
:10E1E0000837BD4680BD80B584B000AFF860B96027
:10E1F0007A60FB6893F82C30DBB2022B01D102234A
:10E2000018E0FB68022283F82C20FB681B687A6800
:10E21000B968184600F0BCFFBB681B68022B04D12C
:10E22000FB68052283F82C2003E0FB68012283F8B9
:10E230002C20002318461037BD4680BD80B582B023
:10E2400000AF786039607B6893F82C30DBB2022B2A
:10E2500001D102230EE07B68022283F82C207B6828
:10E260001B683968184600F0B7FF7B68012283F805
:10E270002C20002318460837BD4680BD80B582B0EB
:10E2800000AF78607B68002B01D1012349E07B68F7
:10E2900093F83D30DBB2002B06D17B68002283F877
:10E2A0003C20786800F041F87B68022283F83D202A
:10E2B0007B681A687B6804331946104600F0CCFA74
:10E2C0007B68012283F848207B68012283F83E2086
:10E2D0007B68012283F83F207B68012283F840207D
:10E2E0007B68012283F841207B68012283F8422069
:10E2F0007B68012283F843207B68012283F8442055
:10E300007B68012283F845207B68012283F8462040
:10E310007B68012283F847207B68012283F83D2037
:10E32000002318460837BD4680BD80B483B000AFD7
:10E33000786000BF0C37BD465DF8047B7047000075
:10E3400080B485B000AF78607B6893F83D30DBB275
:10E35000012B01D0012354E07B68022283F83D2089
:10E360007B681B68DA687B681B6842F00102DA6030
:10E370007B681B68264A934222D07B681B68B3F1F6
:10E38000804F1DD07B681B68224A934218D07B685F
:10E390001B68214A934213D07B681B681F4A934233
:10E3A0000ED07B681B681E4A934209D07B681B68AD
:10E3B0001C4A934204D07B681B681B4A934215D1C8
:10E3C0007B681B689A68194B1340FB60FB68062B3F
:10E3D00015D0FB68B3F5803F11D07B681B681A68C5
:10E3E0007B681B6842F001021A6008E07B681B68CA
:10E3F0001A687B681B6842F001021A6000E000BFE7
:10E40000002318461437BD465DF8047B704700BFF3
:10E41000000001400004004000080040000C0040E3
:10E4200000040140004001400018004007000100C6
:10E4300080B582B000AF78607B68002B01D10123EA
:10E4400049E07B6893F83D30DBB2002B06D17B6856
:10E45000002283F83C207868F4F72CFD7B680222C8
:10E4600083F83D207B681A687B68043319461046A0
:10E4700000F0F2F97B68012283F848207B680122D2
:10E4800083F83E207B68012283F83F207B680122CD
:10E4900083F840207B68012283F841207B680122B9
:10E4A00083F842207B68012283F843207B680122A5
:10E4B00083F844207B68012283F845207B68012291
:10E4C00083F846207B68012283F847207B6801227D
:10E4D00083F83D20002318460837BD4680BD80B52F
:10E4E00082B000AF78607B681B681B6903F0020391
:10E4F000022B22D17B681B68DB6803F00203022B2E
:10E500001BD17B681B686FF002021A617B680122D5
:10E510001A777B681B689B6903F00303002B03D009
:10E52000786800F07BF905E0786800F06DF97868AC
:10E5300000F07EF97B6800221A777B681B681B69F4
:10E5400003F00403042B22D17B681B68DB6803F013
:10E550000403042B1BD17B681B686FF004021A6153
:10E560007B6802221A777B681B689B6903F44073FF
:10E57000002B03D0786800F051F905E0786800F0CE
:10E5800043F9786800F054F97B6800221A777B68B9
:10E590001B681B6903F00803082B22D17B681B68EA
:10E5A000DB6803F00803082B1BD17B681B686FF046
:10E5B00008021A617B6804221A777B681B68DB6992
:10E5C00003F00303002B03D0786800F027F905E07F
:10E5D000786800F019F9786800F02AF97B68002261
:10E5E0001A777B681B681B6903F01003102B22D17C
:10E5F0007B681B68DB6803F01003102B1BD17B6862
:10E600001B686FF010021A617B6808221A777B681A
:10E610001B68DB6903F44073002B03D0786800F0BB
:10E62000FDF805E0786800F0EFF8786800F000F990
:10E630007B6800221A777B681B681B6903F0010363
:10E64000012B0ED17B681B68DB6803F00103012BF3
:10E6500007D17B681B686FF001021A617868F3F7D5
:10E66000F1FF7B681B681B6903F08003802B0ED1D0
:10E670007B681B68DB6803F08003802B07D17B6815
:10E680001B686FF080021A61786800F07BFC7B6881
:10E690001B681B6903F48073B3F5807F0ED17B6820
:10E6A0001B68DB6803F08003802B07D17B681B6845
:10E6B0006FF480721A61786800F06EFC7B681B68EA
:10E6C0001B6903F04003402B0ED17B681B68DB689D
:10E6D00003F04003402B07D17B681B686FF04002BA
:10E6E0001A61786800F0AEF87B681B681B6903F05C
:10E6F0002003202B0ED17B681B68DB6803F020030E
:10E70000202B07D17B681B686FF020021A617868A4
:10E7100000F02EFC00BF0837BD4680BD80B584B038
:10E7200000AFF860B9607A60FB6893F83C30012B69
:10E7300001D1022364E0FB68012283F83C207B685E
:10E74000142B57D801A252F823F000BFA1E700080C
:10E75000F5E70008F5E70008F5E70008AFE700086F
:10E76000F5E70008F5E70008F5E70008BDE7000851
:10E77000F5E70008F5E70008F5E70008CBE7000833
:10E78000F5E70008F5E70008F5E70008D9E7000815
:10E79000F5E70008F5E70008F5E70008E7E70008F7
:10E7A000FB681B68B968184600F0F6F823E0FB68C0
:10E7B0001B68B968184600F061F91CE0FB681B682B
:10E7C000B968184600F0D2F915E0FB681B68B96813
:10E7D000184600F041FA0EE0FB681B68B96818465D
:10E7E00000F092FA07E0FB681B68B968184600F071
:10E7F000DDFA00E000BFFB68002283F83C20002324
:10E8000018461037BD4680BD80B483B000AF786035
:10E8100000BF0C37BD465DF8047B704780B483B001
:10E8200000AF786000BF0C37BD465DF8047B7047D1
:10E8300080B483B000AF786000BF0C37BD465DF890
:10E84000047B704780B483B000AF786000BF0C37A2
:10E85000BD465DF8047B704780B485B000AF78603A
:10E8600039607B681B68FB607B68404A934213D029
:10E870007B68B3F1804F0FD07B683D4A93420BD049
:10E880007B683C4A934207D07B683B4A934203D063
:10E890007B683A4A934208D1FB6823F07003FB601F
:10E8A0003B685B68FA681343FB607B682F4A9342BE
:10E8B0002BD07B68B3F1804F27D07B682C4A9342E2
:10E8C00023D07B682B4A93421FD07B682A4A93420D
:10E8D0001BD07B68294A934217D07B68284A934211
:10E8E00013D07B68274A93420FD07B68264A934215
:10E8F0000BD07B68254A934207D07B68244A934219
:10E9000003D07B68234A934208D1FB6823F4407309
:10E91000FB603B68DB68FA681343FB60FB6823F02D
:10E9200080023B685B691343FB607B68FA681A608E
:10E930003B689A687B68DA623B681A687B689A620F
:10E940007B680A4A934203D07B680C4A934203D106
:10E950003B681A697B681A637B6801225A6100BFB1
:10E960001437BD465DF8047B704700BF00000140CE
:10E970000004004000080040000C0040000401407A
:10E9800000400140004401400048014000180040A0
:10E99000001C00400020004080B487B000AF7860C9
:10E9A00039607B681B6A23F001027B681A627B680E
:10E9B0001B6A7B617B685B683B617B689B69FB6072
:10E9C000FA682B4B1340FB60FB6823F00303FB60EA
:10E9D0003B681B68FA681343FB607B6923F0020302
:10E9E0007B613B689B687A6913437B617B68214A42
:10E9F000934203D07B68204A93420CD17B6923F079
:10EA000008037B613B68DB687A6913437B617B6940
:10EA100023F004037B617B68164A934203D07B6832
:10EA2000154A934211D13B6923F480733B613B69E2
:10EA300023F400733B613B685B693A6913433B61B4
:10EA40003B689B693A6913433B617B683A695A604A
:10EA50007B68FA689A613B685A687B685A637B688E
:10EA60007A691A6200BF1C37BD465DF8047B7047A7
:10EA70008FFFFEFF000001400004014080B487B01A
:10EA800000AF786039607B681B6A23F010027B68F6
:10EA90001A627B681B6A7B617B685B683B617B6891
:10EAA0009B69FB60FA682E4B1340FB60FB6823F404
:10EAB0004073FB603B681B681B02FA681343FB60F2
:10EAC0007B6923F020037B613B689B681B017A69AB
:10EAD00013437B617B68234A934203D07B68224ABD
:10EAE00093420DD17B6923F080037B613B68DB6837
:10EAF0001B017A6913437B617B6923F040037B61CF
:10EB00007B68184A934203D07B68174A934213D11B
:10EB10003B6923F480633B613B6923F400633B6101
:10EB20003B685B699B003A6913433B613B689B69A7
:10EB30009B003A6913433B617B683A695A607B6882
:10EB4000FA689A613B685A687B689A637B687A695D
:10EB50001A6200BF1C37BD465DF8047B704700BFDA
:10EB6000FF8FFFFE000001400004014080B487B029
:10EB700000AF786039607B681B6A23F480727B6821
:10EB80001A627B681B6A7B617B685B683B617B68A0
:10EB9000DB69FB60FA682D4B1340FB60FB6823F0D8
:10EBA0000303FB603B681B68FA681343FB607B69E7
:10EBB00023F400737B613B689B681B027A691343F3
:10EBC0007B617B68224A934203D07B68214A93424F
:10EBD0000DD17B6923F400637B613B68DB681B021A
:10EBE0007A6913437B617B6923F480637B617B6873
:10EBF000174A934203D07B68164A934213D13B696C
:10EC000023F480533B613B6923F400533B613B6831
:10EC10005B691B013A6913433B613B689B691B01BC
:10EC20003A6913433B617B683A695A607B68FA68CA
:10EC3000DA613B685A687B68DA637B687A691A62D2
:10EC400000BF1C37BD465DF8047B70478FFFFEFF99
:10EC5000000001400004014080B487B000AF78603C
:10EC600039607B681B6A23F480527B681A627B6878
:10EC70001B6A3B617B685B687B617B68DB69FB606F
:10EC8000FA681E4B1340FB60FB6823F44073FB6083
:10EC90003B681B681B02FA681343FB603B6923F463
:10ECA00000533B613B689B681B033A6913433B611C
:10ECB0007B68134A934203D07B68124A934209D17E
:10ECC0007B6923F480437B613B685B699B017A69C4
:10ECD00013437B617B687A695A607B68FA68DA6102
:10ECE0003B685A687B681A647B683A691A6200BF9D
:10ECF0001C37BD465DF8047B704700BFFF8FFFFEE9
:10ED0000000001400004014080B487B000AF78608B
:10ED100039607B681B6A23F480327B681A627B68E7
:10ED20001B6A3B617B685B687B617B685B6DFB603A
:10ED3000FA681B4B1340FB603B681B68FA6813437F
:10ED4000FB603B6923F400333B613B689B681B0419
:10ED50003A6913433B617B68124A934203D07B6854
:10ED6000114A934209D17B6923F480337B613B686C
:10ED70005B691B027A6913437B617B687A695A601D
:10ED80007B68FA685A653B685A687B689A657B6855
:10ED90003A691A6200BF1C37BD465DF8047B7047B4
:10EDA0008FFFFEFF000001400004014080B487B0E7
:10EDB00000AF786039607B681B6A23F480127B683F
:10EDC0001A627B681B6A3B617B685B687B617B685E
:10EDD0005B6DFB60FA681C4B1340FB603B681B6873
:10EDE0001B02FA681343FB603B6923F400133B6189
:10EDF0003B689B681B053A6913433B617B68134A78
:10EE0000934203D07B68124A934209D17B6923F471
:10EE100080237B613B685B699B027A6913437B615A
:10EE20007B687A695A607B68FA685A653B685A68F9
:10EE30007B68DA657B683A691A6200BF1C37BD4699
:10EE40005DF8047B704700BFFF8FFFFE00000140AC
:10EE50000004014080B485B000AF786039607B6801
:10EE600093F83C30012B01D102236DE07B68012235
:10EE700083F83C207B68022283F83D207B681B6876
:10EE80005B68FB607B681B689B68BB607B681B687A
:10EE9000304A934204D07B681B682F4A934208D1C2
:10EEA000FB6823F47003FB603B685B68FA681343FC
:10EEB000FB60FB6823F07003FB603B681B68FA682B
:10EEC0001343FB607B681B68FA685A607B681B68A9
:10EED000204A934222D07B681B68B3F1804F1DD03B
:10EEE0007B681B681D4A934218D07B681B681C4ACC
:10EEF000934213D07B681B681A4A93420ED07B68FA
:10EF00001B68154A934209D07B681B68164A9342D6
:10EF100004D07B681B68154A93420CD1BB6823F070
:10EF20008003BB603B689B68BA681343BB607B6827
:10EF30001B68BA689A607B68012283F83D207B6871
:10EF4000002283F83C20002318461437BD465DF8A4
:10EF5000047B7047000001400004014000040040B1
:10EF600000080040000C0040004001400018004034
:10EF700080B483B000AF786000BF0C37BD465DF849
:10EF8000047B704780B483B000AF786000BF0C375B
:10EF9000BD465DF8047B704780B483B000AF7860F5
:10EFA00000BF0C37BD465DF8047B704780B485B068
:10EFB00000AF786039600023FB600023BB603B68D2
:10EFC0001B68012B27D07B681B68FB60FA682F4BFE
:10EFD0001340FB603B685A683B689B681A433B6878
:10EFE000DB681A433B681B691A433B685B691A4339
:10EFF0003B689B691A433B68DB691A433B681B6AA1
:10F000001A433B685B6A1343FA681343FB607B68EF
:10F01000FA681A6032E07B681B68FB60FB6823F4C7
:10F02000F843FB603B68DA693B681B6A1A433B683C
:10F030005B6A1343FA681343FB607B685B68BB60E1
:10F04000BA68124B1340BB603B685A683B689B68C8
:10F050001A433B68DB681A433B681B691A433B68E9
:10F060005B691A433B689B691343BA681343BB60EF
:10F070007B68FA681A607B68BA685A600023184691
:10F080001437BD465DF8047B704700BF0080FFFF6A
:10F0900080B487B000AFF860B9607A6000237B610C
:10F0A00000233B617B68012B2ED0FB689B687B6152
:10F0B0007B6903F070437B61BB681B685A1EBB68A9
:10F0C0005B68013B1B011A43BB689B68013B1B0249
:10F0D0001A43BB68DB68013B1B031A43BB681B690F
:10F0E000013B1B041A43BB685B69013B1B051A43C8
:10F0F000BB689B69013B1B0613437A6913437B6121
:10F10000FB687A699A6039E0FB689B687B617A6981
:10F110001E4B13407B61BB68DB68013B1A03BB6875
:10F120005B69013B1B0513437A6913437B61FB68F1
:10F13000DB683B613B6903F070433B61BB681B6864
:10F140005A1EBB685B68013B1B011A43BB689B6886
:10F15000013B1B021A43BB681B69013B1B041A439A
:10F16000BB689B69013B1B0613433A6913433B6130
:10F17000FB687A699A60FB683A69DA60002318468E
:10F180001C37BD465DF8047B704700BFFF0F0FFFC3
:10F1900080B485B000AFF860B9607A60FB681A6926
:10F1A0000C4B1340BA681168BA6852681143BA68C8
:10F1B0009268013A52011143BA68D26852020A4376
:10F1C0001A43FB681A61002318461437BD465DF8E0
:10F1D000047B70470000C0FF80B483B000AF78604C
:10F1E00039607B685A693B685B001A437B685A61E7
:10F1F000002318460C37BD465DF8047B70470000BD
:10F2000084B080B485B000AF786007F11C0080E85E
:10F210000E000023FB60FA693B6A1A437B6A1A43BB
:10F22000BB6A1A43FB6A1A433B6B1343FA681343E6
:10F23000FB607B685A68074B1340FA681A437B6887
:10F240005A60002318461437BD465DF8047B04B0AD
:10F25000704700BF0081FFFF80B483B000AF7860CB
:10F260007B68D3F8803018460C37BD465DF8047BC8
:10F27000704780B483B000AF786039603B681A682B
:10F280007B68C3F88020002318460C37BD465DF824
:10F29000047B704780B582B000AF78607B68032242
:10F2A0001A600220F9F760F9002318460837BD46B6
:10F2B00080BD80B483B000AF78607B681B6803F0CA
:10F2C000030318460C37BD465DF8047B7047000009
:10F2D00080B485B000AF786039600023FB603B6884
:10F2E0001A687B689A603B685A683B689B681A4357
:10F2F0003B68DB681A433B681B691343FA68134396
:10F30000FB607B68DA68064B1340FA681A437B6837
:10F31000DA60002318461437BD465DF8047B704759
:10F3200000F0FFFF80B483B000AF78607B681B699A
:10F33000DBB218460C37BD465DF8047B704780B4DD
:10F3400085B000AF786039607B6814331A463B683B
:10F350001344FB60FB681B6818461437BD465DF814
:10F36000047B704780B485B000AF786039600023BB
:10F37000FB603B681A687B685A623B685A687B6826
:10F380009A623B689A683B68DB681A433B681B6972
:10F390001A433B685B691343FA681343FB607B685D
:10F3A000DB6A23F0F702FB681A437B68DA6200230A
:10F3B00018461437BD465DF8047B704780B588B0A9
:10F3C00000AF786039603B68BB601023FB6040236E
:10F3D0003B6100237B614FF48063BB6107F108034D
:10F3E00019467868FFF774FF41F288321021786877
:10F3F00000F046FAF861FB6918462037BD4680BD2B
:10F4000080B588B000AF786039603B68BB6011237D
:10F41000FB6040233B6100237B614FF48063BB6151
:10F4200007F1080319467868FFF752FF41F2883266
:10F430001121786800F024FAF861FB69184620373A
:10F44000BD4680BD80B588B000AF786039603B684C
:10F45000BB601223FB6040233B6100237B614FF4C0
:10F460008063BB6107F1080319467868FFF730FF36
:10F4700041F288321221786800F002FAF861FB69E3
:10F4800018462037BD4680BD80B588B000AF786093
:10F4900039603B68BB601823FB6040233B6100235D
:10F4A0007B614FF48063BB6107F1080319467868FC
:10F4B000FFF70EFF41F288321821786800F0E0F97A
:10F4C000F861FB6918462037BD4680BD80B588B01D
:10F4D00000AF786039603B68BB601923FB60402354
:10F4E0003B6100237B614FF48063BB6107F108033C
:10F4F00019467868FFF7ECFE41F2883219217868E6
:10F5000000F0BEF9F861FB6918462037BD4680BDA2
:10F5100080B588B000AF78600023BB600C23FB602F
:10F5200040233B6100237B614FF48063BB6107F1A3
:10F53000080319467868FFF7CBFE054A0C21786866
:10F5400000F09EF9F861FB6918462037BD4680BD82
:10F5500000E1F50580B58AB000AFF860C7E9002387
:10F560003B683B6107237B614023BB610023FB6158
:10F570004FF480633B6207F110031946F868FFF708
:10F58000A7FE41F288320721F86800F079F9786225
:10F590007B6A18462837BD4680BD80B588B000AF6D
:10F5A00078600023BB600023FB6000233B610023E5
:10F5B0007B614FF48063BB6107F1080319467868EB
:10F5C000FFF786FE786800F02FF9F861FB691846AE
:10F5D0002037BD4680BD80B588B000AF78604FF45D
:10F5E000D573BB600823FB6040233B6100237B6134
:10F5F0004FF48063BB6107F1080319467868FFF791
:10F6000067FE786800F026FBF861FB691846203732
:10F61000BD4680BD80B588B000AF786039603B687A
:10F62000BB603723FB6040233B6100237B614FF4C9
:10F630008063BB6107F1080319467868FFF748FE4D
:10F6400041F288323721786800F01AF9F861FB69D5
:10F6500018462037BD4680BD80B588B000AF7860C1
:10F6600039603A680D4B1343BB602923FB6040238C
:10F670003B6100237B614FF48063BB6107F10803AA
:10F6800019467868FFF724FE786800F02FFAF861D1
:10F69000FB6918462037BD4680BD00BF00001080C2
:10F6A00080B588B000AF786039603B68BB600623E6
:10F6B000FB6040233B6100237B614FF48063BB61AF
:10F6C00007F1080319467868FFF702FE41F2883215
:10F6D0000621786800F0D4F8F861FB6918462037F5
:10F6E000BD4680BD80B588B000AF78600023BB60A8
:10F6F0003323FB6040233B6100237B614FF4806335
:10F70000BB6107F1080319467868FFF7E1FD41F294
:10F7100088323321786800F0B3F8F861FB69184645
:10F720002037BD4680BD80B588B000AF786000232B
:10F73000BB600223FB60C0233B6100237B614FF46D
:10F740008063BB6107F1080319467868FFF7C0FDC5
:10F75000786800F083F9F861FB6918462037BD46E8
:10F7600080BD80B588B000AF786039603B68BB6011
:10F770000923FB60C0233B6100237B614FF480635E
:10F78000BB6107F1080319467868FFF7A1FD7868A7
:10F7900000F064F9F861FB6918462037BD4680BD6A
:10F7A00080B588B000AF786039600023BB60032368
:10F7B000FB6040233B6100237B614FF48063BB61AE
:10F7C00007F1080319467868FFF782FD3A680321BC
:10F7D000786800F0C9F9F861FB6918462037BD4622
:10F7E00080BD80B588B000AF786039603B68BB6091
:10F7F0000D23FB6040233B6100237B614FF480635A
:10F80000BB6107F1080319467868FFF761FD41F213
:10F8100088320D21786800F033F8F861FB691846EA
:10F820002037BD4680BD000080B485B000AF786051
:10F83000114B1B68114AA2FB03235B0A41F2883279
:10F8400002FB03F3FB60FB685A1EFA60002B02D137
:10F850004FF0004309E07B685B6B03F08003002BF3
:10F86000F1D07B68C5229A63002318461437BD4641
:10F870005DF8047B704700BF24000020D34D621068
:10F8800080B588B000AFF8600B467A60FB72704BB1
:10F890001B68704AA2FB03235A0A7B6802FB03F32E
:10F8A000FB61FB695A1EFA61002B02D14FF0004345
:10F8B000C9E0FB685B6BBB61BB6903F04503002BD0
:10F8C000EFD0BB6903F40063002BEAD1FB685B6BEC
:10F8D00003F00403002B04D0FB6804229A63042382
:10F8E000B1E0FB685B6B03F00103002B04D0FB6805
:10F8F00001229A630123A6E0FB68C5229A63F86897
:10F90000FFF710FD03461A46FB7A934201D001230C
:10F9100099E00021F868FFF712FD78617A694E4B93
:10F920001340002B01D100238DE07B69002B02DA0C
:10F930004FF0007387E07B6903F08043002B01D018
:10F94000402380E07B6903F00053002B01D080232B
:10F9500079E07B6903F08053002B02D04FF4807371
:10F9600071E07B6903F00063002B02D04FF4007359
:10F9700069E07B6903F08063002B02D04FF4806361
:10F9800061E07B6903F08073002B02D04FF40063C9
:10F9900059E07B6903F40003002B02D04FF480533D
:10F9A00051E07B6903F48003002B02D04FF4005335
:10F9B00049E07B6903F40013002B02D04FF480432D
:10F9C00041E07B6903F48013002B02D04FF4004325
:10F9D00039E07B6903F48023002B02D04FF400331D
:10F9E00031E07B6903F40033002B02D04FF4802315
:10F9F00029E07B6903F48033002B02D04FF400230D
:10FA000021E07B6903F40043002B02D04FF4801304
:10FA100019E07B6903F48043002B02D04FF40013FC
:10FA200011E07B6903F40053002B02D04FF48003F4
:10FA300009E07B6903F00803002B02D04FF40003B8
:10FA400001E04FF4803318462037BD4680BD00BF2B
:10FA500024000020D34D621008E0FFFD80B485B083
:10FA600000AF78601F4B1B681F4AA2FB03235B0A91
:10FA700041F2883202FB03F3FB60FB685A1EFA6016
:10FA8000002B02D14FF0004326E07B685B6BBB602C
:10FA9000BB6803F04503002BEFD0BB6803F40063A1
:10FAA000002BEAD17B685B6B03F00403002B04D0CE
:10FAB0007B6804229A6304230EE07B685B6B03F08F
:10FAC0000103002B04D07B6801229A63012303E029
:10FAD0007B68C5229A63002318461437BD465DF83B
:10FAE000047B704724000020D34D621080B485B0A1
:10FAF00000AF78601A4B1B681A4AA2FB03235B0A0B
:10FB000041F2883202FB03F3FB60FB685A1EFA6085
:10FB1000002B02D14FF000431BE07B685B6BBB60A6
:10FB2000BB6803F04503002BEFD0BB6803F4006310
:10FB3000002BEAD17B685B6B03F00403002B04D03D
:10FB40007B6804229A63042303E07B68C5229A63DE
:10FB5000002318461437BD465DF8047B704700BF8C
:10FB600024000020D34D621080B588B000AFF8604B
:10FB70000B467A60FB72354B1B68354AA2FB0323A8
:10FB80005B0A41F2883202FB03F3FB61FB695A1EF8
:10FB9000FA61002B02D14FF0004352E0FB685B6B2F
:10FBA000BB61BB6903F04503002BEFD0BB6903F4D5
:10FBB0000063002BEAD1FB685B6B03F00403002BAE
:10FBC00004D0FB6804229A6304233AE0FB685B6B71
:10FBD00003F00103002B04D0FB6801229A63012388
:10FBE0002FE0F868FFF79EFB03461A46FB7A934224
:10FBF00001D0012325E0FB68C5229A630021F86843
:10FC0000FFF79DFB78617B6903F46043002B06D10D
:10FC10007B691B0C9AB27B681A80002311E07B6918
:10FC200003F48043002B02D04FF4005309E07B69BA
:10FC300003F40043002B02D04FF4805301E04FF453
:10FC4000803318462037BD4680BD00BF2400002009
:10FC5000D34D621080B485B000AF7860224B1B6832
:10FC6000224AA2FB03235B0A41F2883202FB03F320
:10FC7000FB60FB685A1EFA60002B02D14FF0004374
:10FC80002CE07B685B6BBB60BB6803F04503002B1B
:10FC9000EFD0BB6803F40063002BEAD17B685B6B99
:10FCA00003F00403002B04D07B6804229A6304232E
:10FCB00014E07B685B6B03F00103002B04D07B68CE
:10FCC00001229A63012309E07B685B6B03F0400328
:10FCD000002B02D07B6840229A6300231846143719
:10FCE000BD465DF8047B704724000020D34D6210B0
:10FCF00080B487B000AFF860B9601346FB71012390
:10FD0000FB750023BB751F4B5B7ADBB2002B31D137
:10FD10001C4B5B7ADBB21A461A4B00219954194BE3
:10FD20005B7ADBB2174A9B001344FA685A60154BA2
:10FD30005B7ADBB21A46134B1344FA791A72114BF1
:10FD40005B7ADBB25A1CD1B20E4A5172BB75BB7DD5
:10FD50003033DAB2BB681A70BB6801333A221A70CA
:10FD6000BB6802332F221A70BB68033300221A705B
:10FD70000023FB75FB7D18461C37BD465DF8047BF0
:10FD8000704700BF4C53002080B582B000AF786050
:10FD90003960002239687868FFF7AAFF03461846E1
:10FDA0000837BD4680BD80B485B000AF0346FB80F8
:10FDB0000023FB60B7F90630842B05D0B7F9062085
:10FDC000FB6813440333FB60FB6818461437BD46D9
:10FDD0005DF8047B704780B483B000AFEFF3058318
:10FDE0007B607B68002B14BF01230023DBB2184625
:10FDF0000C37BD465DF8047B704780B500AF02F05C
:10FE00000FF80023184680BD80B500AF02F0A0FCBB
:10FE10000346012B01D1002300E00123184680BDD9
:10FE200080B500AFFFF7D7FF0346002B03D002F0E9
:10FE300027F9034602E002F013F90346184680BD95
:10FE4000F0B589B004AF786039607B685B69002BDE
:10FE500020D07B689B69002B1CD07B685C687B682A
:10FE60001D687B681E697B68B3F908301846FFF788
:10FE70009AFF01467B685B697A68926902920193F6
:10FE800000913B6832462946204601F0DDFD0346DD
:10FE9000FB601CE07B685C687B681D687B681B6995
:10FEA0009EB27B68B3F908301846FFF77CFF024624
:10FEB00007F10C03019300923B6832462946204625
:10FEC00001F025FE0346012B01D0002300E0FB6872
:10FED00018461437BD46F0BD80B400AF064B4FF056
:10FEE00080521A60BFF34F8FBFF36F8F0023184605
:10FEF000BD465DF8047B704704ED00E080B584B03A
:10FF000000AF78607B68FB60FB68002B01D0FB686A
:10FF100000E00123184601F04DFF0023184610377A
:10FF2000BD4680BD80B586B002AF786039607B6821
:10FF30005B68002B0FD03B68012B0AD17B685B68A4
:10FF40000322009200220021012000F0B5FE0346AA
:10FF500016E0002314E03B68012B10D1032200219E
:10FF6000012000F02BFFF860FB68002B05D0002378
:10FF700000220021F86800F083FFFB6800E0002306
:10FF800018461037BD4680BD80B584B000AF78609C
:10FF900039600023BB607B68002B01D180233AE0ED
:10FFA0000023FB603B68B3F1FF3F03D14FF0FF3309
:10FFB000FB6009E03B68002B06D03B68FB60FB68F8
:10FFC000002B01D10123FB60FFF705FF0346002B47
:10FFD00017D007F108031A460021786801F086FB64
:10FFE0000346012B01D0FF2315E0BB68002B11D085
:10FFF0000B4B4FF080521A60BFF34F8FBFF36F8FE0
:020000040801F1
:1000000008E0F968786801F05DFA0346012B01D039
:10001000FF2300E0002318461037BD4680BD00BF17
:1000200004ED00E080B584B000AF78600023FB6091
:100030000023BB60FFF7CFFE0346002B16D007F16D
:1000400008031946786801F0C1F80346012B01D076
:10005000FF2317E0BB68002B13D00C4B4FF08052EE
:100060001A60BFF34F8FBFF36F8F0AE000230022A7
:100070000021786800F004FF0346012B01D0FF2324
:10008000FB60FB6818461037BD4680BD04ED00E0FC
:1000900090B585B002AF786039607B689B68002BB3
:1000A00011D07B68DB68002B0DD07B6818687B68FB
:1000B00059687B689A687B68DB680024009400F0CC
:1000C000FBFD034608E07B6818687B685B680022DC
:1000D000194600F073FE034618460C37BD4690BD26
:1000E00080B586B000AFF860B9607A6000233B61EC
:1000F0007B687B617B69002B01D101237B61FFF76A
:100100006AFE0346002B18D007F1100207F1080120
:100110000023F86800F0BAFF0346012B01D0FF234B
:1001200018E03B69002B14D00C4B4FF080521A6042
:10013000BFF34F8FBFF36F8F0BE007F10801002370
:100140007A69F86800F09CFE0346012B01D0FF237A
:1001500000E0002318461837BD4680BD04ED00E0DE
:1001600090B58BB000AFF860B9607A60BB68FB6196
:100170000023BB61BB68002B0AD180237B61FB6835
:100180001C4607F1140393E8070084E8070054E0D5
:1001900000233B6200237B627B68B3F1FF3F03D106
:1001A0004FF0FF337B6209E07B68002B06D07B6851
:1001B0007B627B6A002B01D101237B62FFF70BFE80
:1001C0000346002B1CD007F1200207F1140304336F
:1001D0001946B86801F08AFA0346012B02D11023B0
:1001E0007B6101E000237B613B6A002B1DD0154B36
:1001F0004FF080521A60BFF34F8FBFF36F8F14E040
:1002000007F1140304337A6A1946B86801F074F8E8
:100210000346012B02D110237B6106E07B6A002B91
:1002200001D1002300E040237B61FB681C4607F1FD
:10023000140393E8070084E80700F8682C37BD46EC
:1002400090BD00BF04ED00E080B58AB000AF7860DB
:100250000023FB6101F058FE5B4B1B68002B01D1B2
:1002600000F01AF9594B1A687B681340002B40F0D4
:1002700092807B68002B1FD008227B6813447B6030
:100280007B6803F00703002B16D07B6823F007037D
:1002900008337B607B6803F00703002B0CD04FF022
:1002A000500372B683F31188BFF36F8FBFF34F8F84
:1002B00062B67B6100BFFEE77B68002B6BD0444BCE
:1002C0001B687A689A4266D8424B3B62414B1B6876
:1002D0007B6204E07B6A3B627B6A1B687B627B6AB1
:1002E0005B687A689A4203D97B6A1B68002BF1D15C
:1002F000354B1B687A6A9A424DD03B6A1B680822CC
:100300001344FB617B6A1A683B6A1A607B6A5A680D
:100310007B68D21A08235B009A4221D97A6A7B68EB
:100320001344BB61BB6903F00703002B0CD04FF0F3
:10033000500372B683F31188BFF36F8FBFF34F8FF3
:1003400062B63B6100BFFEE77B6A5A687B68D21ADF
:10035000BB695A607B6A7A685A60B86900F0FEF837
:100360001B4B1A687B6A5B68D31A194A1360184BD7
:100370001A68194B1B689A4203D2154B1B68164A20
:1003800013607B6A5A68114B1B681A437B6A5A6078
:100390007B6A00221A6001F0C5FDFB6903F00703C8
:1003A000002B0CD04FF0500372B683F31188BFF3CB
:1003B0006F8FBFF34F8F62B6FB6000BFFEE7FB6934
:1003C00018462837BD4680BD605301206C5301207C
:1003D00064530120585301206853012080B586B032
:1003E00000AF78607B687B617B68002B4CD0082372
:1003F0005B427A6913447B617B693B613B695A6864
:10040000234B1B681340002B0CD14FF0500372B6E6
:1004100083F31188BFF36F8FBFF34F8F62B6FB601A
:1004200000BFFEE73B691B68002B0CD04FF0500368
:1004300072B683F31188BFF36F8FBFF34F8F62B62D
:10044000BB6000BFFEE73B695A68114B1B68134055
:10045000002B19D03B691B68002B15D13B695A68EA
:100460000B4B1B68DB431A403B695A6001F04CFDA3
:100470003B695A68074B1B681344064A1360386986
:1004800000F06CF801F04EFD00BF1837BD4680BD8E
:100490006C5301206453012080B485B000AF4FF449
:1004A0008033BB60274BFB60FB6803F00703002B26
:1004B0000CD0FB680733FB60FB6823F00703FB608D
:1004C000BA68FB68D31A1F4A1344BB60FB687B60A1
:1004D0001D4A7B6813601C4B00225A607B68BA6817
:1004E0001344FB600822FB689B1AFB60FB6823F047
:1004F0000703FB60FB68154A1360144B1B6800225E
:100500005A60124B1B6800221A607B683B603B6894
:10051000FA68D21A3B685A600C4B1A683B681A603A
:100520003B685B680A4A13603B685B68094A136072
:10053000094B4FF000421A6000BF1437BD465DF80A
:10054000047B70475853002058530120605301200A
:1005500068530120645301206C53012080B485B09E
:1005600000AF7860284BFB6002E0FB681B68FB6013
:10057000FB681B687A689A42F7D8FB68BB60FB6827
:100580005B68BA6813447A689A4208D1FB685A6873
:100590007B685B681A44FB685A60FB687B607B6819
:1005A000BB607B685B68BA681A44FB681B689A4248
:1005B00018D1FB681A68154B1B689A420DD07B68EE
:1005C0005A68FB681B685B681A447B685A60FB6862
:1005D0001B681A687B681A6008E00C4B1A687B6815
:1005E0001A6003E0FB681A687B681A60FA687B6827
:1005F0009A4202D0FB687A681A6000BF1437BD4681
:100600005DF8047B704700BF585301206053012000
:1006100080B483B000AF78607B6803F108027B6828
:100620005A607B684FF0FF329A607B6803F10802E2
:100630007B68DA607B6803F108027B681A617B687B
:1006400000221A6000BF0C37BD465DF8047B70477E
:1006500080B483B000AF78607B6800221A6100BF6D
:100660000C37BD465DF8047B704780B485B000AFA1
:10067000786039607B685B68FB603B68FA685A6049
:10068000FB689A683B689A60FB689B683A685A60A6
:10069000FB683A689A603B687A681A617B681B68F5
:1006A0005A1C7B681A6000BF1437BD465DF8047B96
:1006B000704780B485B000AF786039603B681B68D4
:1006C000BB60BB68B3F1FF3F03D17B681B69FB6074
:1006D0000CE07B680833FB6002E0FB685B68FB6052
:1006E000FB685B681B68BA689A42F6D2FB685A6876
:1006F0003B685A603B685B683A689A603B68FA6896
:100700009A60FB683A685A603B687A681A617B684D
:100710001B685A1C7B681A6000BF1437BD465DF821
:10072000047B704780B485B000AF78607B681B693C
:10073000FB607B685B687A6892689A607B689B68FC
:100740007A6852685A60FB685B687A689A4203D19B
:100750007B689A68FB685A607B6800221A61FB68B4
:100760001B685A1EFB681A60FB681B681846143722
:10077000BD465DF8047B704780B485B000AFF8607B
:10078000B9607A60FB68043BFB60FB684FF08072E5
:100790001A60FB68043BFB60BB6823F00102FB6846
:1007A0001A60FB68043BFB600C4AFB681A60FB683C
:1007B000143BFB607A68FB681A60FB68043BFB60D3
:1007C000FB686FF002021A60FB68203BFB60FB686D
:1007D00018461437BD465DF8047B7047E1070108F1
:1007E00080B485B000AF00237B60144B1B68B3F16D
:1007F000FF3F0CD04FF0500372B683F31188BFF364
:100800006F8FBFF34F8F62B6FB6000BFFEE74FF004
:10081000500372B683F31188BFF36F8FBFF34F8F0E
:1008200062B6BB6000BF00BF7B68002BFCD000BF7E
:1008300000BF1437BD465DF8047B704758000020A8
:10084000074B19680868B0E8F04F80F30988BFF3D8
:100850006F8F4FF0000080F311887047AFF3008076
:100860007853012000BF00BF08480068006880F38B
:1008700008884FF0000080F3148862B661B6BFF3B9
:100880004F8FBFF36F8F00DF00BF00BF08ED00E0A8
:1008900080B584B000AF374BFB60FB681B78DBB2E0
:1008A0007B60FB68FF221A70FB681B78DBB2FB7071
:1008B000FB78DBB203F05003DAB22F4B1A702F4BE8
:1008C00007221A6009E02D4B1B68013B2B4A13607D
:1008D000FB78DBB25B00DBB2FB70FB78DBB203F0D2
:1008E0008003802BEFD0254B1B68C3F10703042B3B
:1008F0000CD04FF0500372B683F31188BFF36F8FA3
:10090000BFF34F8F62B6BB6000BFFEE71B4B1B6897
:100910001B021A4A1360194B1B6803F4E063174A61
:1009200013607B68DAB2FB681A70154B1B68144AB7
:1009300043F470031360124B1B68114A43F0704379
:10094000136000F0DDF80F4B00221A6000F0FCF895
:100950000D4B1B680C4A43F040431360FFF784FFC4
:1009600001F098FCFFF73CFF002318461037BD4606
:1009700080BD00BF00E400E07053012074530120EB
:1009800020ED00E05800002034EF00E080B483B098
:1009900000AF4FF0500372B683F31188BFF36F8F2F
:1009A000BFF34F8F62B67B6000BF104B1B680133F3
:1009B0000E4A13600D4B1B68012B11D10C4B1B68A9
:1009C000DBB2002B0CD04FF0500372B683F31188CA
:1009D000BFF36F8FBFF34F8F62B63B6000BFFEE780
:1009E00000BF0C37BD465DF8047B704758000020FF
:1009F00004ED00E080B483B000AF134B1B68002B04
:100A00000CD14FF0500372B683F31188BFF36F8F90
:100A1000BFF34F8F62B67B6000BFFEE70A4B1B68D7
:100A2000013B094A1360084B1B68002B05D10023CA
:100A30003B603B6883F3118800BF00BF0C37BD46A5
:100A40005DF8047B704700BF5800002000000000E4
:100A5000EFF30980BFF36F8F154B1A681EF0100F6C
:100A600008BF20ED108A20E9F04F10602DE9090041
:100A70004FF0500072B680F31188BFF34F8FBFF371
:100A80006F8F62B601F006FC4FF0000080F3118812
:100A900009BC19680868B0E8F04F1EF0100F08BFD5
:100AA000B0EC108A80F30988BFF36F8F704700BFE6
:100AB0007853012000BF00BF80B582B000AF4FF077
:100AC000500372B683F31188BFF36F8FBFF34F8F5C
:100AD00062B67B6000BF01F0E5FA0346002B03D04D
:100AE000064B4FF080521A6000233B603B6883F353
:100AF000118800BF00BF0837BD4680BD04ED00E08F
:100B000080B400AF0B4B00221A600B4B00221A601E
:100B10000A4B1B680A4AA2FB03239B09094A013BB3
:100B20001360044B07221A6000BFBD465DF8047BCA
:100B3000704700BF10E000E018E000E02400002053
:100B4000D34D621014E000E0DFF80C00016841F4BE
:100B500070010160704700BF88ED00E080B485B08F
:100B600000AFEFF30583FB60FB680F2B16D9194A22
:100B7000FB6813441B78FB72174B1B78FA7A9A4276
:100B80000CD24FF0500372B683F31188BFF36F8F0E
:100B9000BFF34F8F62B67B6000BFFEE70F4B1B6851
:100BA00003F4E0620E4B1B689A420CD94FF05003DD
:100BB00072B683F31188BFF36F8FBFF34F8F62B6A6
:100BC0003B6000BFFEE700BF1437BD465DF8047B05
:100BD000704700BFF0E300E0705301200CED00E02F
:100BE0007453012080B584B000AF786039607B68B1
:100BF000FB60FB68002B0CD14FF0500372B683F3FF
:100C00001188BFF36F8FBFF34F8F62B6BB6000BF19
:100C1000FEE7FFF7BBFEFB681A68FB68DB6BF96851
:100C2000096C01FB03F31A44FB689A60FB6800221D
:100C30009A63FB681A68FB685A60FB681A68FB686D
:100C4000DB6B013BF968096C01FB03F31A44FB6899
:100C5000DA60FB68FF2283F84420FB68FF2283F8F8
:100C600045203B68002B14D1FB681B69002B1AD070
:100C7000FB681033184601F0A1FB0346002B12D08D
:100C80000C4B4FF080521A60BFF34F8FBFF36F8F42
:100C900009E0FB6810331846FFF7BAFCFB68243301
:100CA0001846FFF7B5FCFFF7A5FE012318461037DD
:100CB000BD4680BD04ED00E080B58EB002AFF860A7
:100CC000B9607A603B60FB68002B0CD14FF0500399
:100CD00072B683F31188BFF36F8FBFF34F8F62B685
:100CE000BB6200BFFEE73B68002B0CD14FF0500306
:100CF00072B683F31188BFF36F8FBFF34F8F62B665
:100D00007B6200BFFEE77B68002B02D0BB68002B34
:100D100001D0012300E00023002B0CD14FF0500341
:100D200072B683F31188BFF36F8FBFF34F8F62B634
:100D30003B6200BFFEE77B68002B02D1BB68002B43
:100D400001D1012300E00023002B0CD14FF0500310
:100D500072B683F31188BFF36F8FBFF34F8F62B604
:100D6000FB6100BFFEE748237B617B69482B0CD009
:100D70004FF0500372B683F31188BFF36F8FBFF348
:100D80004F8F62B6BB6100BFFEE77B693B68FB62C9
:100D9000FB6A002B0DD0FB6A012283F8462097F8EE
:100DA0003820FB6A009313467A68B968F86800F047
:100DB00047F8FB6A18463037BD4680BD80B58AB01B
:100DC00002AFF860B9601346FB71FB68002B0CD1D1
:100DD0004FF0500372B683F31188BFF36F8FBFF3E8
:100DE0004F8F62B63B6100BFFEE7BB68002B02D1AC
:100DF0000023FB6104E0FB68BA6802FB03F3FB61BC
:100E0000FB6948331846FFF71FFAB861BB69002B2E
:100E100011D0BB697B617B6948337B61BB69002270
:100E200083F84620FA79BB69009313467A69B9685A
:100E3000F86800F005F8BB6918462037BD4680BD4C
:100E400080B584B000AFF860B9607A60FB70BB68B1
:100E5000002B03D1BB69BA691A6002E0BB697A68EA
:100E60001A60BB69FA68DA63BB69BA681A6401215F
:100E7000B869FFF7B7FE00BF1037BD4680BD000060
:100E800080B58EB000AFF860B9607A603B60002337
:100E90007B63FB683B633B6B002B0CD14FF0500333
:100EA00072B683F31188BFF36F8FBFF34F8F62B6B3
:100EB000BB6200BFFEE7BB68002B03D13B6B1B6C22
:100EC000002B01D1012300E00023002B0CD14FF0B7
:100ED000500372B683F31188BFF36F8FBFF34F8F48
:100EE00062B67B6200BFFEE73B68022B03D13B6B1F
:100EF000DB6B012B01D1012300E00023002B0CD17F
:100F00004FF0500372B683F31188BFF36F8FBFF3B6
:100F10004F8F62B63B6200BFFEE701F019FC03464B
:100F2000002B02D17B68002B01D1012300E00023BC
:100F3000002B0CD14FF0500372B683F31188BFF32E
:100F40006F8FBFF34F8F62B6FB6100BFFEE7FFF705
:100F50001DFD3B6B9A6B3B6BDB6B9A4202D33B688C
:100F6000022B29D13A68B968386B00F05DFCF86251
:100F70003B6B5B6A002B10D03B6B2433184601F0AF
:100F80001DFA0346002B13D03F4B4FF080521A60DE
:100F9000BFF34F8FBFF36F8F0AE0FB6A002B07D0C0
:100FA000394B4FF080521A60BFF34F8FBFF36F8FF2
:100FB000FFF720FD012363E07B68002B03D1FFF7DF
:100FC00019FD00235CE07B6B002B06D107F11403B5
:100FD000184601F057FA01237B63FFF70BFD00F081
:100FE00093FFFFF7D3FC3B6B93F844305BB2B3F154
:100FF000FF3F03D13B6B002283F844203B6B93F807
:1010000045305BB2B3F1FF3F03D13B6B002283F865
:101010004520FFF7EFFC3A1D07F11403114618466F
:1010200001F046FA0346002B24D1386B00F0F4FCA3
:101030000346002B18D03B6B10337A6811461846D4
:1010400001F096F9386B00F07FFC00F06BFF03466F
:10105000002B7FF47CAF0C4B4FF080521A60BFF333
:101060004F8FBFF36F8F72E7386B00F06DFC00F0AD
:1010700059FF6CE7386B00F067FC00F053FF00236A
:1010800018463837BD4680BD04ED00E080B58EB00F
:1010900000AFF860B9607A603B60FB683B633B6B14
:1010A000002B0CD14FF0500372B683F31188BFF3BD
:1010B0006F8FBFF34F8F62B67B6200BFFEE7BB68E6
:1010C000002B03D13B6B1B6C002B01D1012300E0F3
:1010D0000023002B0CD14FF0500372B683F311881C
:1010E000BFF36F8FBFF34F8F62B63B6200BFFEE767
:1010F0003B68022B03D13B6BDB6B012B01D101233E
:1011000000E00023002B0CD14FF0500372B683F3A4
:101110001188BFF36F8FBFF34F8F62B6FB6100BFC3
:10112000FEE7FFF71BFDEFF311824FF0500372B69D
:1011300083F31188BFF36F8FBFF34F8F62B6BA612D
:101140007B61BB69FB623B6B9A6B3B6BDB6B9A42CF
:1011500002D33B68022B2CD13B6B93F8453087F8C8
:101160002B303A68B968386B00F05EFB97F92B308A
:10117000B3F1FF3F12D13B6B5B6A002B16D03B6B88
:101180002433184601F01AF90346002B0ED07B6871
:10119000002B0BD07B6801221A6007E097F82B30F8
:1011A0000133DBB25AB23B6B83F8452001237B63EA
:1011B00001E000237B63FB6A3B613B6983F3118899
:1011C00000BF7B6B18463837BD4680BD80B58EB0FA
:1011D00000AF786039607B683B633B6B002B0CD1C0
:1011E0004FF0500372B683F31188BFF36F8FBFF3D4
:1011F0004F8F62B63B6200BFFEE73B6B1B6C002B60
:101200000CD04FF0500372B683F31188BFF36F8F89
:10121000BFF34F8F62B6FB6100BFFEE73B6B1B68FD
:10122000002B03D13B6B9B68002B01D1012300E015
:101230000023002B0CD14FF0500372B683F31188BA
:10124000BFF36F8FBFF34F8F62B6BB6100BFFEE786
:10125000FFF784FCEFF311824FF0500372B683F373
:101260001188BFF36F8FBFF34F8F62B67A613B6116
:101270007B69FB623B6B9B6BBB623B6BDB6BBA6A54
:101280009A422BD23B6B93F8453087F82730BB6AE4
:101290005A1C3B6B9A6397F92730B3F1FF3F12D189
:1012A0003B6B5B6A002B16D03B6B2433184601F076
:1012B00085F80346002B0ED03B68002B0BD03B6813
:1012C00001221A6007E097F827300133DBB25AB2E7
:1012D0003B6B83F8452001237B6301E000237B63A4
:1012E000FB6AFB60FB6883F3118800BF7B6B1846C9
:1012F0003837BD4680BD000080B58CB000AFF860C7
:10130000B9607A600023FB62FB68BB62BB6A002B9A
:101310000CD14FF0500372B683F31188BFF36F8F77
:10132000BFF34F8F62B63B6200BFFEE7BB68002B86
:1013300003D1BB6A1B6C002B01D1012300E0002309
:10134000002B0CD14FF0500372B683F31188BFF31A
:101350006F8FBFF34F8F62B6FB6100BFFEE701F0F6
:10136000F7F90346002B02D17B68002B01D1012342
:1013700000E00023002B0CD14FF0500372B683F332
:101380001188BFF36F8FBFF34F8F62B6BB6100BF91
:10139000FEE7FFF7FBFABB6A9B6B7B627B6A002B65
:1013A0001FD0B968B86A00F0A9FA7B6A5A1EBB6AF6
:1013B0009A63BB6A1B69002B0FD0BB6A10331846B7
:1013C00000F0FCFF0346002B07D03D4B4FF080524E
:1013D0001A60BFF34F8FBFF36F8FFFF70BFB012333
:1013E00069E07B68002B03D1FFF704FB002362E078
:1013F000FB6A002B06D107F11003184601F042F8F2
:101400000123FB62FFF7F6FA00F07EFDFFF7BEFA5C
:10141000BB6A93F844305BB2B3F1FF3F03D1BB6AC0
:10142000002283F84420BB6A93F845305BB2B3F1E5
:10143000FF3F03D1BB6A002283F84520FFF7DAFAA9
:101440003A1D07F110031146184601F031F8034622
:10145000002B23D1B86A00F0C9FA0346002B17D03D
:10146000BB6A24337A681146184600F081FFB86AD7
:1014700000F06AFA00F056FD0346002B89D1104BAC
:101480004FF080521A60BFF34F8FBFF36F8F80E72A
:10149000B86A00F059FA00F045FD7AE7B86A00F042
:1014A00053FA00F03FFDB86A00F0A0FA0346002BA3
:1014B0003FF46FAF002318463037BD4680BD00BFF4
:1014C00004ED00E080B58EB000AF78603960002395
:1014D0007B637B68FB6200233B63FB6A002B0CD1C0
:1014E0004FF0500372B683F31188BFF36F8FBFF3D1
:1014F0004F8F62B63B6200BFFEE7FB6A1B6C002B9E
:101500000CD04FF0500372B683F31188BFF36F8F86
:10151000BFF34F8F62B6FB6100BFFEE701F018F921
:101520000346002B02D13B68002B01D1012300E0D0
:101530000023002B0CD14FF0500372B683F31188B7
:10154000BFF36F8FBFF34F8F62B6BB6100BFFEE783
:10155000FFF71CFAFB6A9B6BBB62BB6A002B24D0B3
:10156000BB6A5A1EFB6A9A63FB6A1B68002B04D194
:1015700001F0B4FA0246FB6A9A60FB6A1B69002B11
:101580000FD0FB6A1033184600F018FF0346002BFB
:1015900007D0554B4FF080521A60BFF34F8FBFF307
:1015A0006F8FFFF727FA012399E03B68002B13D1D7
:1015B0003B6B002B0CD04FF0500372B683F31188B5
:1015C000BFF36F8FBFF34F8F62B67B6100BFFEE743
:1015D000FFF710FA002382E07B6B002B06D107F1A6
:1015E0000C03184600F04EFF01237B63FFF702FA5D
:1015F00000F08AFCFFF7CAF9FB6A93F844305BB24B
:10160000B3F1FF3F03D1FB6A002283F84420FB6A59
:1016100093F845305BB2B3F1FF3F03D1FB6A002280
:1016200083F84520FFF7E6F93A4607F10C03114627
:10163000184600F03DFF0346002B32D1F86A00F057
:10164000D5F90346002B26D0FB6A1B68002B09D175
:10165000FFF79CF9FB6A9B68184601F097F838631E
:10166000FFF7C8F9FB6A24333A681146184600F0C0
:101670007FFEF86A00F068F900F054FC0346002B86
:101680007FF466AF184B4FF080521A60BFF34F8F54
:10169000BFF36F8F5CE7F86A00F056F900F042FC88
:1016A00056E7F86A00F050F900F03CFCF86A00F0E8
:1016B0009DF90346002B3FF44BAF3B6B002B0DD045
:1016C000FFF764F9F86A00F097F87862FB6A9B68A4
:1016D000796A184601F064F9FFF78CF9002318467F
:1016E0003837BD4680BD00BF04ED00E080B58EB048
:1016F00000AFF860B9607A60FB683B633B6B002B1E
:101700000CD14FF0500372B683F31188BFF36F8F83
:10171000BFF34F8F62B63B6200BFFEE7BB68002B92
:1017200003D13B6B1B6C002B01D1012300E0002394
:10173000002B0CD14FF0500372B683F31188BFF326
:101740006F8FBFF34F8F62B6FB6100BFFEE7FFF7FD
:1017500005FAEFF311824FF0500372B683F311884C
:10176000BFF36F8FBFF34F8F62B6BA617B61BB6906
:10177000FB623B6B9B6BBB62BB6A002B2FD03B6B4E
:1017800093F8443087F82730B968386B00F0B6F822
:10179000BB6A5A1E3B6B9A6397F92730B3F1FF3F40
:1017A00012D13B6B1B69002B16D03B6B10331846D4
:1017B00000F004FE0346002B0ED07B68002B0BD0FC
:1017C0007B6801221A6007E097F827300133DBB20B
:1017D0005AB23B6B83F8442001237B6301E0002372
:1017E0007B63FB6A3B613B6983F3118800BF7B6BC2
:1017F00018463837BD4680BD80B485B000AF7860EC
:101800007B685B6A002B06D07B681B6B1B68C3F18F
:101810000703FB6001E00023FB60FB6818461437F8
:10182000BD465DF8047B704780B586B000AFF860B8
:10183000B9607A6000237B61FB689B6B3B61FB684E
:101840001B6C002B0DD1FB681B68002B4DD1FB6876
:101850009B68184601F01AF87861FB6800229A60CC
:1018600043E07B68002B19D1FB685868FB681B6C50
:101870001A46B96819F0ACFCFB685A68FB681B6C27
:101880001A44FB685A60FB685A68FB689B689A4276
:101890002BD3FB681A68FB685A6026E0FB68D8689F
:1018A000FB681B6C1A46B96819F092FCFB68DA6891
:1018B000FB681B6C5B421A44FB68DA60FB68DA6801
:1018C000FB681B689A4207D2FB689A68FB681B6C2E
:1018D0005B421A44FB68DA607B68022B05D13B69E6
:1018E000002B02D03B69013B3B613B695A1CFB6802
:1018F0009A637B6918461837BD4680BD80B582B0B3
:1019000000AF786039607B681B6C002B18D07B6857
:10191000DA687B681B6C1A447B68DA607B68DA687B
:101920007B689B689A4203D37B681A687B68DA609D
:101930007B68D9687B681B6C1A46386819F048FCCC
:1019400000BF0837BD4680BD80B584B000AF786069
:10195000FFF71CF87B6893F84530FB7311E07B6858
:101960005B6A002B12D07B682433184600F026FDFA
:101970000346002B01D000F001FEFB7B013BDBB2F4
:10198000FB7397F90F30002BE9DC00E000BF7B68A8
:10199000FF2283F84520FFF72DF8FEF7F7FF7B685D
:1019A00093F84430BB7311E07B681B69002B12D0A5
:1019B0007B681033184600F001FD0346002B01D070
:1019C00000F0DCFDBB7B013BDBB2BB7397F90E3053
:1019D000002BE9DC00E000BF7B68FF2283F8442095
:1019E000FFF708F800BF1037BD4680BD80B584B052
:1019F00000AF7860FEF7CAFF7B689B6B002B02D1BB
:101A00000123FB6001E00023FB60FEF7F3FFFB68AE
:101A100018461037BD4680BD80B584B000AF7860F1
:101A2000FEF7B4FF7B689A6B7B68DB6B9A4202D14E
:101A30000123FB6001E00023FB60FEF7DBFFFB6896
:101A400018461037BD4680BD80B58EB004AFF86033
:101A5000B9607A603B607B6B002B0CD14FF0500378
:101A600072B683F31188BFF36F8FBFF34F8F62B6E7
:101A70003B6200BFFEE7BB6B002B0CD14FF0500365
:101A800072B683F31188BFF36F8FBFF34F8F62B6C7
:101A9000FB6100BFFEE7B8233B613B69B82B0CD06C
:101AA0004FF0500372B683F31188BFF36F8FBFF30B
:101AB0004F8F62B6BB6100BFFEE73B69BB6B002B7B
:101AC0001ED07B6B002B1BD0BB6B7B627B6A7A6B5F
:101AD0001A637B6A022283F8B520002303937B6A92
:101AE000029307F1140301933B6B00933B687A6800
:101AF000B968F86800F050F8786A00F0F1F801E091
:101B000000237B617B6918462837BD4680BD80B5C0
:101B10008CB004AFF860B9603B601346FB80FB8873
:101B20009B001846FEF790FB78617B69002B0ED076
:101B3000B820FEF789FBF861FB69002B03D0FB6935
:101B40007A691A6305E07869FEF748FC01E0002332
:101B5000FB61FB69002B17D0FB69002283F8B520DD
:101B6000FA8800230393FB690293FB6A0193BB6A23
:101B700000933B68B968F86800F00EF8F86900F067
:101B8000AFF80123BB6102E04FF0FF33BB61BB69DB
:101B900018462037BD4680BD80B588B000AFF860DC
:101BA000B9607A603B603B6B1A6B79686FF04043B9
:101BB0000B449B001344BB61BB6923F00703BB616B
:101BC000BB6903F00703002B0CD04FF0500372B633
:101BD00083F31188BFF36F8FBFF34F8F62B67B61C2
:101BE00000BFFEE7BB68002B1FD00023FB6112E0A3
:101BF000BA68FB69134419783A6BFB6913443433B0
:101C00000A461A70BA68FB6913441B78002B06D089
